S01400005354345F52433030375F32382E73726563E1
S3150800800000000220195E0208695E0208695E02081D
S31508008010695E0208695E0208695E020800000000DF
S31508008020000000000000000000000000695E020871
S31508008030695E020800000000695E0208655D0208C4
S31508008040695E0208695E0208695E0208695E0208DE
S31508008050695E0208695E0208695E0208695E0208CE
S31508008060695E0208695E0208695E0208695E0208BE
S31508008070695E0208695E0208695E0208695E0208AE
S31508008080695E0208695E0208695E0208695E02089E
S31508008090695E0208695E0208695E0208715D020887
S315080080A0695E0208695E0208695E0208695E02087E
S315080080B0E95D0208015E0208695E0208695E020857
S315080080C0695E0208695E0208695E0208695E02085E
S315080080D0695E0208B55D0208695E0208695E020803
S315080080E09D5D0208695E0208695E0208695E02080B
S315080080F0695E0208695E0208695E0208695E02082E
S31508008100695E0208695E0208695E0208695E02081D
S31508008110695E0208695E0208695E0208695E02080D
S31508008120695E0208695E0208C55D0208695E0208A2
S31508008130695E02080000000000000000695E02088F
S31508008140695E0208695E0208695E0208695E0208DD
S31508008150695E0208695E0208D95D0208695E02085E
S31508008160695E0208695E0208695E0208695E0208BD
S31508008170695E0208695E0208695E0208000000007E
S3150800818000000000695E0208000000000000000010
S31508008190695E02080000000000000000695E02082F
S315080081A0000000000000000000000000695E0208F0
S315080081B0695E0208695E0208695E0208695E02086D
S309080081C0695E0208DC
S315080081D010B5054C237833B9044B13B10448AFF3F3
S315080081E000800123237010BD200A00200000000033
S315080081F09C8802080C4B43B10C480D4910B5AFF3E7
S3150800820000800C48036823B910BD0A48036833B9CF
S315080082107047094B002BF7D0BDE810401847064BAE
S31508008220002BF5D0184700BF000000009C88020804
S31508008230240A00201C0A00200000000081F00041EA
S3150800824002E000BF83F0004330B54FEA41044FEA2D
S31508008250430594EA050F08BF90EA020F1FBF54EAC8
S31508008260000C55EA020C7FEA645C7FEA655C00F064
S31508008270E2804FEA5454D4EB5555B8BF6D420CDD35
S315080082802C4480EA020281EA030382EA000083EAB8
S31508008290010180EA020281EA0303362D88BF30BD58
S315080082A011F0004F4FEA01314FF4801C4CEA1131AE
S315080082B002D0404261EB410113F0004F4FEA03330D
S315080082C04CEA133302D0524263EB430394EA050F98
S315080082D000F0A780A4F10104D5F1200E0DDB02FA07
S315080082E00EFC22FA05F2801841F1000103FA0EF29B
S315080082F0801843FA05F359410EE0A5F120050EF161
S31508008300200E012A03FA0EFC28BF4CF0020C43FA91
S3150800831005F3C01851EBE37101F0004507D54FF09E
S31508008320000EDCF1000C7EEB00006EEB0101B1F5EE
S31508008330801F1BD3B1F5001F0CD349085FEA300034
S315080083404FEA3C0C04F101044FEA445212F5800F3F
S3150800835080F09A80BCF1004F08BF5FEA500C50F1DC
S31508008360000041EB045141EA050130BD5FEA4C0CBF
S31508008370404141EB010111F4801FA4F10104E9D148
S3150800838091F0000F04BF01460020B1FA81F308BF3F
S315080083902033A3F10B03B3F120020CDA0C3208DD0B
S315080083A002F1140CC2F10C0201FA0CF021FA02F1E6
S315080083B00CE002F11402D8BFC2F1200C01FA02F156
S315080083C020FA0CFCDCBF41EA0C019040E41AA2BF7B
S315080083D001EB0451294330BD6FEA04041F3C1CDA43
S315080083E00C340EDC04F11404C4F1200220FA04F063
S315080083F001FA02F340EA030021FA04F345EA03010D
S3150800840030BDC4F10C04C4F1200220FA02F001FACE
S3150800841004F340EA0300294630BD21FA04F0294650
S3150800842030BD94F0000F83F4801306BF81F48011E9
S315080084300134013D4EE77FEA645C18BF7FEA655C5C
S3150800844029D094EA050F08BF90EA020F05D054EA2E
S31508008450000C04BF1946104630BD91EA030F1EBF33
S315080084600021002030BD5FEA545C05D14000494137
S3150800847028BF41F0004130BD14F580043CBF01F52A
S31508008480801130BD01F0004545F0FE4141F4700110
S315080084904FF0000030BD7FEA645C1ABF19461046EB
S315080084A07FEA655C1CBF0B46024650EA013406BFEC
S315080084B052EA033591EA030F41F4002130BD00BFAB
S315080084C090F0000F04BF0021704730B54FF4806468
S315080084D004F132044FF000054FF0000150E700BFE9
S315080084E090F0000F04BF0021704730B54FF4806448
S315080084F004F1320410F0004548BF40424FF0000135
S315080085003EE700BF42004FEAE2014FEA31014FEA77
S3150800851002701FBF12F07F4393F07F4F81F06051C6
S31508008520704792F0000F14BF93F07F4F704730B535
S315080085304FF4607401F0004521F0004120E700BFC8
S3150800854050EA010208BF704730B54FF000050AE04F
S3150800855050EA010208BF704730B511F0004502D550
S31508008560404261EB41014FF4806404F132045FEA52
S31508008570915C3FF4DCAE4FF003025FEADC0C18BFF7
S3150800858003325FEADC0C18BF033202EBDC02C2F1ED
S31508008590200300FA03FC20FA02F001FA03FE40EA7F
S315080085A00E0021FA02F11444C1E600BF70B54FF07F
S315080085B0FF0C4CF4E06C1CEA11541DBF1CEA135561
S315080085C094EA0C0F95EA0C0F00F0DEF82C4481EAC9
S315080085D0030621EA4C5123EA4C5350EA013518BFE9
S315080085E052EA033541F4801143F4801338D0A0FBD6
S315080085F002CE4FF00005E1FB02E506F00042E0FB83
S3150800860003E54FF00006E1FB03569CF0000F18BF88
S315080086104EF0010EA4F1FF04B6F5007F64F5407430
S3150800862004D25FEA4E0E6D4146EB060642EAC621C3
S3150800863041EA55514FEAC52040EA5E504FEACE2E30
S31508008640B4F1FD0C88BFBCF5E06F1ED8BEF1004F33
S3150800865008BF5FEA500E50F1000041EB045170BDAF
S3150800866006F0004646EA010140EA020081EA0301F3
S31508008670B4EB5C04C2BFD4EB0C0541EA045170BDEF
S3150800868041F480114FF0000E013C00F3AB8014F169
S31508008690360FDEBF002001F0004170BDC4F10004B2
S315080086A0203C35DA0C341BDC04F11404C4F1200533
S315080086B000FA05F320FA04F001FA05F240EA02008E
S315080086C001F0004221F0004110EBD37021FA04F6C4
S315080086D042EB06015EEA430E08BF20EAD37070BD7E
S315080086E0C4F10C04C4F1200500FA04F320FA05F0DD
S315080086F001FA04F240EA020001F0004110EBD370DF
S3150800870041F100015EEA430E08BF20EAD37070BD4E
S31508008710C4F1200500FA05F24EEA020E20FA04F327
S3150800872001FA05F243EA020321FA04F001F00041D6
S3150800873021FA04F220EA020000EBD3705EEA430E47
S3150800874008BF20EAD37070BD94F0000F0FD101F076
S315080087500046400041EB010111F4801F08BF013CAF
S31508008760F7D041EA060195F0000F18BF704703F0ED
S315080087700046520043EB030313F4801F08BF013D74
S31508008780F7D043EA0603704794EA0C0F0CEA135530
S3150800879018BF95EA0C0F0CD050EA410618BF52EAEA
S315080087A04306D1D181EA030101F000414FF00000F0
S315080087B070BD50EA410606BF1046194652EA4306FE
S315080087C019D094EA0C0F02D150EA013613D195EA72
S315080087D00C0F05D152EA03361CBF104619460AD1BA
S315080087E081EA030101F0004141F0FE4141F47001C4
S315080087F04FF0000070BD41F0FE4141F4780170BDB4
S3150800880070B54FF0FF0C4CF4E06C1CEA11541DBF18
S315080088101CEA135594EA0C0F95EA0C0F00F0A7F81A
S31508008820A4EB050481EA030E52EA03354FEA013147
S3150800883000F088804FEA03334FF0805545EA13135A
S3150800884043EA12634FEA022245EA111545EA106522
S315080088504FEA00260EF000419D4208BF964244F1B9
S31508008860FD0404F5407402D25B084FEA3202B61AD8
S3150800887065EB03055B084FEA32024FF480104FF4AC
S31508008880002CB6EB020E75EB030E22BFB61A754620
S3150800889040EA0C005B084FEA3202B6EB020E75EBB3
S315080088A0030E22BFB61A754640EA5C005B084FEA1B
S315080088B03202B6EB020E75EB030E22BFB61A7546E8
S315080088C040EA9C005B084FEA3202B6EB020E75EBF3
S315080088D0030E22BFB61A754640EADC0055EA060EB4
S315080088E018D04FEA051545EA16754FEA06164FEAF7
S315080088F0C30343EA52734FEAC2025FEA1C1CC0D1A3
S3150800890011F4801F0BD141EA00014FF000004FF02F
S31508008910004CB6E711F4801F04BF01430020B4F1F0
S31508008920FD0C88BFBCF5E06F3FF6AFAEB5EB030CA8
S3150800893004BFB6EB020C5FEA500C50F1000041EBA5
S31508008940045170BD0EF0004E4EEA113114EB5C0472
S31508008950C2BFD4EB0C0541EA045170BD41F4801145
S315080089604FF0000E013C90E645EA060E8DE60CEA4D
S31508008970135594EA0C0F08BF95EA0C0F3FF43BAF6A
S3150800898094EA0C0F0AD150EA01347FF434AF95EA21
S315080089900C0F7FF425AF104619462CE795EA0C0F05
S315080089A006D152EA03353FF4FDAE1046194622E7D2
S315080089B050EA410618BF52EA43067FF4C5AE50EAAC
S315080089C041047FF40DAF52EA43057FF4EBAE12E79C
S315080089D04FF0FF3C06E000BF4FF0010C02E000BF7D
S315080089E04FF0010C4DF804CD4FEA410C7FEA6C5C60
S315080089F04FEA430C18BF7FEA6C5C1BD001B050EA03
S31508008A00410C0CBF52EA430C91EA030F02BF90EAED
S31508008A10020F0020704710F1000F91EA030F58BFAC
S31508008A20994208BF90422CBFD8176FEAE37040F00E
S31508008A30010070474FEA410C7FEA6C5C02D150EAAC
S31508008A40013C07D14FEA430C7FEA6C5CD6D152EA67
S31508008A50033CD3D05DF8040B704700BF844610462C
S31508008A6062468C461946634600E000BF01B5FFF72B
S31508008A70B7FF002848BF10F1000F01BD4DF808EDFB
S31508008A80FFF7F4FF0CBF012000205DF808FB00BFCC
S31508008A904DF808EDFFF7EAFF34BF012000205DF826
S31508008AA008FB00BF4DF808EDFFF7E0FF94BF012073
S31508008AB000205DF808FB00BF4DF808EDFFF7CEFF74
S31508008AC094BF012000205DF808FB00BF4DF808EDB3
S31508008AD0FFF7C4FF34BF012000205DF808FB00BF84
S31508008AE04FEA410C7FEA6C5C02D150EA013C0AD19C
S31508008AF04FEA430C7FEA6C5C02D152EA033C02D18E
S31508008B004FF0000070474FF0010070474FEA4102EE
S31508008B1012F5001215D211D56FF47873B3EB6252C1
S31508008B2012D94FEAC12343F0004343EA505311F0E8
S31508008B30004F23FA02F018BF404270474FF000007A
S31508008B40704750EA013005D111F0004008BF6FF0B8
S31508008B50004070474FF00000704700BF4A0011D22E
S31508008B6012F5001211D20DD56FF47873B3EB625279
S31508008B700ED44FEAC12343F0004343EA505323FA85
S31508008B8002F070474FF00000704750EA013002D1FA
S31508008B904FF0FF3070474FF0000070474FEA410230
S31508008BA0B2F1E04324BFB3F5001CDCF1FE5C0DD93D
S31508008BB001F0004C4FEAC0024CEA5070B2F1004F87
S31508008BC040EB830008BF20F00100704711F0804F8A
S31508008BD021D113F13872BCBF01F00040704741F44F
S31508008BE080114FEA5252C2F11802C2F1200C10FA53
S31508008BF00CF320FA02F018BF40F001004FEAC12337
S31508008C004FEAD32303FA0CFC40EA0C0023FA02F3DA
S31508008C104FEA4303CCE77FEA625307D150EA0133B0
S31508008C201EBF4FF0FE4040F44000704701F0004080
S31508008C3040F0FE4040F40000704700BF034613F8BA
S31508008C40012B002AFBD1181A0138704700000000D2
S31508008C5001F0FF01102A2BDB10F0070F08D010F8DF
S31508008C60013B013A8B422DD010F0070F42B3F6D1E3
S31508008C70F0B441EA012141EA014122F007047FF0FC
S31508008C8000070023F0E80256083C85EA010586EA53
S31508008C90010685FA47F5A3FA87F586FA47F6A5FA8F
S31508008CA087F68EB9EED1F0BC01F0FF0102F007029B
S31508008CB032B110F8013B013A83EA010313B1F8D146
S31508008CC00020704701387047002D06BF3546033827
S31508008CD0073815F0010F07D1013015F4807F02BF60
S31508008CE0013015F4C03F0130F0BC0138704700BFB1
S31508008CF070470120704790F85000704790F8790047
S31508008D007047E02914BF00200120704740F65C2315
S31508008D10994209D043690BB9038BD3B140F24C533E
S31508008D20994208D00020704742F2E810824214BFE8
S31508008D30002001207047B2F51A7F0CD040F22F436D
S31508008D409A420AD040F2D530824214BF0020012050
S31508008D507047002070470120704701207047019A2C
S31508008D60C3BB80F85D10D37803F00301032920D034
S31508008D7013F0020F2ED092F90230002BB4BF022353
S31508008D80032303EB43030344917801F00F0183F8AF
S31508008D905110918883F85210937990F878209A4266
S31508008DA0B8BF80F8783090F85E30013380F85E30CE
S31508008DB0704792F90210002904DB13F0020F09D05C
S31508008DC00323DEE790F85610012363F3870180F842
S31508008DD05610D6E77047A0F10400FFF7C0BFF8B5F4
S31508008DE005460146002214464FF0080C4FF00F0EB8
S31508008DF0012736E005F1640405F1740601E0B44282
S31508008E0007D054F8040B0028F9D003689B689847E4
S31508008E10F5E7002385F8413085F8423085F8463075
S31508008E2085F8473085F87C3085F85030012285F87A
S31508008E305E202B6685F8783085F87930F8BD81F89C
S31508008E40524081F853403E4603EB43032B4493F8C4
S31508008E50530066F3870083F8530001320331042A6E
S31508008E60C8D0134681F8514012F0FF0FE7D181F8B8
S31508008E7052C081F853407646E6E7000010B504462E
S31508008E801B4B03F1080202603C334360002380F861
S31508008E90413080F8433080F8463080F84830C16465
S31508008EA080F85030012280F85E20036680F878301A
S31508008EB080F8793043668366C3660367FFF78FFFDA
S31508008EC0E06C68B1836F6BB101231A4602F11E018B
S31508008ED050F8211039B10133DBB21A460F2BF5DDF4
S31508008EE0204610BD00221E3240F82240F8E700BF97
S31508008EF0B88802082DE9F04788B004460E4617469A
S31508008F001D46FFF76CFF94F8503023B1D925284643
S31508008F1008B0BDE8F087D4F84C80D8F800301B6854
S31508008F20002140469847814600283AD0D0F800A04C
S31508008F30BAF1000F37D004F151030360857103AB12
S31508008F400093122300221146E06C02F00AFCC9F8CD
S31508008F5000A0054640B10D280CBF0546E12523684B
S31508008F609B6820469847D2E7D8F800305D683B46AC
S31508008F70002231464046A84784F85000A8B19DF81B
S31508008F80133084F852309DF81D3084F85430BDF8FB
S31508008F901430A4F87630BDF81630A4F87430E025FD
S31508008FA0B5E7D625B3E7D725B1E7D425AFE710B59A
S31508008FB00446FFF714FFE06C03689B6894F85010AA
S31508008FC09847002010BDF0B585B0054604AB402291
S31508008FD023F8022D00F1C90690F8572090F8501092
S31508008FE090F8780001900096E86C02F0C3F918B181
S31508008FF005F16404743515E0BDF80E30002BF7D082
S3150800900005F1640405F1740701E0BC42F0D054F898
S31508009010040B0028F9D003681B6831469847F4E723
S31508009020A54207D054F8040B0028F9D003685B68FA
S315080090309847F5E705B0F0BD30B589B0B0F8863089
S3150800904023F00103A0F8863090F8515090F850406C
S31508009050C06C00230793069105920492039302932A
S315080090600193009320232A46214602F0C2FA09B04A
S3150800907030BD10B501460023A0F88630032280F8DB
S3150800908089200C2480F88A4080F88B308931FFF7D4
S31508009090D3FF10BD08B5B0F8863023F01003A0F84A
S315080090A086301A2380F889300C2380F88A30012309
S315080090B080F88B30C36843B1032380F88C300422D0
S315080090C000F18901FFF7B8FF08BD022380F88C304C
S315080090D0F5E708B50146B0F8863023F02003A0F876
S315080090E08630092380F88930102380F88A300023D7
S315080090F080F88B3003228931FFF79EFF08BD08B53B
S315080091000146B0F8863023F04003A0F886300123E4
S3150800911080F88930102380F88A30002380F88B3055
S3150800912003228931FFF788FF08BD08B50146B0F864
S31508009130863023F00203A0F88630092380F88930A8
S31508009140042380F88A30072380F88B30037F80F861
S315080091508C30437F80F88D30837F80F88E30C37FD4
S3150800916080F88F3090F8203080F8903090F82130D1
S3150800917080F89130002380F892300A228931FFF76F
S315080091805BFF08BD08B50146B0F8863023F0080332
S31508009190A0F88630192380F88930042380F88A30AD
S315080091A00A2380F88B30037F80F88C30437F80F861
S315080091B08D30837F80F88E30C37F80F88F3090F8AB
S315080091C0203080F8903090F8213080F891300123D3
S315080091D080F89230002380F8933080F8943080F835
S315080091E095300D228931FFF727FF08BDF8B50746E8
S315080091F00E46132380F889300C2380F88A300846F7
S31508009200FFF71CFD013087F88B000024E5B23046D5
S31508009210FFF714FD631CA84206D9725D57FA84F459
S3150800922084F88C201C46F1E757FA84F4002384F866
S315080092308C303046FFF702FD021D92B207F1890114
S315080092403846FFF7F9FEF8BD08B50146B0F886308E
S3150800925023F08003A0F88630012380F889300423A0
S3150800926080F88A30052380F88B30332380F88C30D9
S315080092708B2380F88D309E2380F88E30302380F83B
S315080092808F300A2380F8903008228931FFF7D4FE00
S3150800929008BD08B50146022380F88930042380F802
S315080092A08A30002380F88B3003228931FFF7C4FE09
S315080092B008BD08B5B0F8862022F48172A0F8862089
S315080092C0052280F88920042280F88A200D2280F859
S315080092D08B200A7880F88C204A7880F88D208A7846
S315080092E080F88E20CA7880F88F200A7980F8902036
S315080092F04A7980F89120182280F89220CC2280F8AA
S315080093009320012280F89420002280F8952080F886
S31508009310962080F8972080F89820102200F189017D
S31508009320FFF78AFE08BD08B500F11C01FFF7C1FF6B
S3150800933008BDF8B506460D2380F88930042380F861
S315080093408A30172380F88B30037F80F88C30437F70
S3150800935080F88D30837F80F88E30C37F80F88F3019
S3150800936090F8203080F8903090F8213080F89130CD
S3150800937090F8433063B3062380F8923090F87A3039
S31508009380D3B100F1140300F193021A3013F8011B4C
S3150800939002F8011B8342F9D106F1980306F1A201EE
S315080093A0002203F8012F9942FBD11A2206F18901FE
S315080093B03046FFF741FEF8BD00F11C0300F19302A9
S315080093C0223013F8011B02F8011B8342F9D1E3E7A7
S315080093D007693846FFF732FC86F892000024E5B2A2
S315080093E03846FFF72BFC631CA84206D97A5D56FA65
S315080093F084F484F893201C46F1E72C460F2DD4DC20
S315080094000023344484F893300135EDB22C460F2DF1
S31508009410F7DDCAE708B501460E2380F8893004232C
S3150800942080F88A30062380F88B30037F80F88C30EA
S31508009430437F80F88D30837F80F88E30C37F80F835
S315080094408F3090F8203080F8903090F8213080F8EE
S31508009450913009228931FFF7EFFD08BD08B50146AD
S315080094600C2380F88930042380F88A30062380F894
S315080094708B30037F80F88C30437F80F88D30837F74
S3150800948080F88E30C37F80F88F3090F8203080F8CF
S31508009490903090F8213080F8913009228931FFF711
S315080094A0CBFD08BDF0B585B0044604AB402223F8D1
S315080094B0022D90F8542090F8501090F878000190FA
S315080094C004F189000090E06C01F054FF10F0FB00F5
S315080094D068D194F88930013B162B63D8DFE813F07E
S315080094E045006400DB002201F6005F01040162000A
S315080094F06200620062006200620017006200620099
S31508009500620062006200620062004A015B0194F830
S315080095108E30002B46D1B4F8860040F00103A4F83B
S315080095208630B4F88C3041F20102934214D041F2ED
S315080095300902934236D104F1140304F18F0204F1AF
S315080095401A0512F8011B03F8011BAB42F9D140F0CA
S315080095502100A4F8860025E094F88F3084F840307E
S3150800956040F04100A4F886001CE094F88830042BEB
S3150800957013DD94F8433013B994F848306BB10023DF
S3150800958084F8883084F8413084F8433084F84630CB
S3150800959084F848300A2384F8803094F888300133F8
S315080095A084F8883005B0F0BD94F88B30002BF9D0DC
S315080095B09E46002BF6D0DB00DBB294F843704FF0E2
S315080095C0000C2FE084F87E1084F87D60002384F870
S315080095D07F30012384F87B300CEB4C0204EB42020B
S315080095E08C3204F11C0304F1220012F8011B03F863
S315080095F0011B9842F9D1B4F8863043F08003A4F8E9
S315080096008630CFE794F848502DB111F0050F02D0F7
S3150800961016F0C80F1CD10130C0B284460333DBB242
S31508009620704531DAE21892F88D6092F88E1092F849
S315080096308F20002FE6D0002AE4D111F0050FEAD0DA
S3150800964016F00C0FBED194F84850002DE0D1E2E791
S3150800965084F87E1084F87D6084F87F200CEB4C0338
S3150800966004EB43038C3304F11C0204F1220013F8C3
S31508009670011B02F8011B8242F9D1B4F8863043F087
S315080096808003A4F886308DE784F87E1084F87D6020
S3150800969084F87F2086E7B4F8863043F48072A4F80D
S315080096A0862094F88B206AB994F88D20120202F469
S315080096B0706294F88C100A43628343F48173A4F8A9
S315080096C086306FE7062384F880306BE794F88B3092
S315080096D0002B7FF467AFB4F8863023F0020343F01B
S315080096E00403A4F886305DE794F88B30002B7FF4EA
S315080096F059AF94F8923084F8223063B104F122030A
S3150800970004F1920104F13F0011F8012F03F8012F2B
S315080097100AB18342F8D1B4F8863043F00803A4F8B6
S3150800972086303FE704F11C0304F18B0204F12200A2
S3150800973012F8011B03F8011B8342F9D194F8912012
S3150800974084F87D2094F8923084F87E3094F893104B
S3150800975084F87F1013F0050F05D012F0C80F1CBF50
S31508009760012384F84730B4F8863043F01003A4F890
S31508009770863017E794F843302BB923693BB1204666
S31508009780FFF7D7FD0EE72046FFF7D3FD0AE7204689
S31508009790FFF740FE06E72046FFF760FE02E794F86B
S315080097A0433013B194F841306BB194F84830002B2C
S315080097B03FF4F8AE94F84630002B7FF4F3AE01235D
S315080097C084F84630EEE6012384F84130EAE608B527
S315080097D00146112380F88930042380F88A30022351
S315080097E080F88B30438B80F88C30C3F3032380F8E2
S315080097F08D3005228931FFF71FFC08BD10B5B0F87A
S31508009800862022F00402A0F88620062280F8892005
S31508009810042480F88A40032480F88B4080F88C1052
S31508009820C1F3032180F88D10132180F88E1000F102
S315080098308901FFF701FC10BD08B50146242380F80D
S3150800984089300C2380F88A30032380F88B30042370
S3150800985080F88C30082380F88D30002380F88E300D
S3150800986006228931FFF7E8FB08BD000070B50446FB
S3150800987090F88030102B1CD8DFE813F01100250073
S315080098804E005900640075007E008F00A400B300E6
S31508009890C500E100F60054011B006A017B01B0F81F
S315080098A0823001339BB2A0F88230B0F8842093420C
S315080098B000DC70BDFFF7DDFB012384F88030002350
S315080098C0A4F8823070BDB0F8823001339BB2A0F89C
S315080098D08230B0F8862012F0010F14D1B0F8842037
S315080098E09342E6DD02EB82035B009BB2B3F5FA6FA7
S315080098F0C8BF4FF4FA63A0F88430002380F880309C
S31508009900A0F8823070BD0023A0F88230022380F8C8
S315080099108030FFF791FF70BDB0F8863013F0010F65
S31508009920C7D0032380F88030FFF7D3FB70BDB0F8AB
S31508009930863013F0200FBCD0FFF7E1FB042384F830
S31508009940803070BDB0F8863013F0400FB1D0C168D2
S3150800995029B1FFF74BFC052384F8803070BD062338
S3150800996080F8803070BDB0F8863013F0010FA0D0B3
S31508009970062380F8803070BD90F8483013B990F807
S31508009980433033B12046FFF75FFC072384F8803065
S3150800999070BD0A2380F8803070BDB0F8863013F0A9
S315080099A0800F86D0FFF775FC94F87B301BB9082327
S315080099B084F8803070BD2046FFF7E4FB0C2384F85A
S315080099C0803070BDB0F8863013F0010F3FF471AFE8
S315080099D0002380F87B30FFF7A6FC092384F8803043
S315080099E070BDB0F8863013F4807F3FF462AF13F091
S315080099F0020F05D0FFF7EBFE0A2384F8803070BD0E
S31508009A00FFF791FC70BD90F84130002B7FF451AF01
S31508009A1090F84330002B7FF44CAF90F84630002B7B
S31508009A207FF447AF90F84830002B7FF442AFFFF73A
S31508009A3031FB012323720B2384F8803070BDB0F804
S31508009A40863013F0100F07D113F0040F3FF431AF2F
S31508009A50102380F8803070BD00230372FFF792FB55
S31508009A600C2384F8803070BDB0F8863013F0080FE8
S31508009A703FF41FAF00F122050822524928461CF080
S31508009A80A1FE90B9012384F84230002384F84430BB
S31508009A9084F8453084F87A3016224B4928461CF05B
S31508009AA091FE80B9012384F84430B4F87E30252B22
S31508009AB022D094F8433073B394F87B305BB3082311
S31508009AC084F8803070BD1622404928461CF07AFE7C
S31508009AD038B9012384F87A3084F8443084F845305C
S31508009AE0E3E713223A4928461CF06CFE0028DCD12D
S31508009AF0012384F87A30D8E794F87D30082BD8D13A
S31508009B001322344928461CF05DFE0028D1D10123D2
S31508009B1084F87C30CDE72046FFF707FB0D2384F851
S31508009B20803070BDB0F8863013F0020F3FF4C1AE36
S31508009B3090F87C3013B1012380F846300023637215
S31508009B40A372E372A4F886300F2384F8803070BDC0
S31508009B50B0F8823001339BB2B3F57A7F02DCA0F805
S31508009B60823070BD0023A0F882300A2380F8803046
S31508009B7070BDB0F8863013F0040F3FF49AAE002596
S31508009B80A0F8865040263246294689301CF0D7FC74
S31508009B903246294604F1C9001CF0D1FC84F843502A
S31508009BA084F8425084F8415084F87B5084F8485031
S31508009BB084F8475084F8465084F87C500A2384F881
S31508009BC0803076E6100203081C02030834020308F4
S31508009BD04C0203086002030890F879300BB900209C
S31508009BE0704710B5044602F0F7FC236EC01A002829
S31508009BF00EDB02F0F1FC94F8783018442066204613
S31508009C00FFF750FC2046FFF731FE2046FFF7DBF949
S31508009C10002010BDF0B583B002AF03F10F0424F0A5
S31508009C200704ADEB040D0DF1080C8DF80810C1F30F
S31508009C30032141F020018CF80110191D8CF802103F
S31508009C4009128CF803108CF8043000218CF80510E2
S31508009C50397E8CF80610397F8CF807105BB11E46E2
S31508009C60E646002421467444555C2572013189B2C2
S31508009C700C468E42F7DC90F85A2090F85010C06CCB
S31508009C80CDF800C0083301F096FC10B90437BD467C
S31508009C90F0BD642002F0A6FCF8E770B582B0BDF806
S31508009CA01850022680F8096180F80A21042280F8F3
S31508009CB00B21002280F80C2180F80D512D1280F816
S31508009CC00E511D7880F80F515B7880F8103101929B
S31508009CD001230093082300F20912FFF79BFF02B045
S31508009CE070BD70B582B0069D032680F8096180F8BC
S31508009CF00A21082280F80B21002280F80C211E7800
S31508009D0080F80D615B7880F80E312B7880F80F317A
S31508009D106B7880F810319DF81C3080F8113180F886
S31508009D20122180F8132180F814210192012300934F
S31508009D300C2300F20912FFF76DFF02B070BD30B5B3
S31508009D4083B0042580F8095180F80A21082280F892
S31508009D500B21002280F80C211D7880F80D515B78C4
S31508009D6080F80E3180F80F2180F81021012380F841
S31508009D701131022580F81251FF2580F8135180F819
S31508009D801451019200930C2300F20912FFF742FFC7
S31508009D9003B030BD70B582B0052580F8095180F84A
S31508009DA00A210A2280F80B21002280F80C211D784E
S31508009DB080F80D515B7880F80E3180F80F2180F815
S31508009DC0102180F8112180F81221012380F813311F
S31508009DD0022580F81451A02680F8156180F81651DE
S31508009DE0019200930E2300F20912FFF713FF02B047
S31508009DF070BD70B582B0069D062680F8096180F8A8
S31508009E000A21042280F80B21002280F80C211E78F2
S31508009E1080F80D615B7880F80E312B7880F80F3169
S31508009E206B7880F81031019201230093082300F221
S31508009E300912FFF7EFFE02B070BD70B582B0069D3D
S31508009E40072680F8096180F80A21042280F80B2188
S31508009E50002280F80C211E7880F80D615B7880F866
S31508009E600E312B7880F80F316B7880F8103101921B
S31508009E7001230093082300F20912FFF7CBFE02B074
S31508009E8070BD10B58AB001238DF820300AAA0023C8
S31508009E9002F8073D8B1D13F8014D02F8014F8B425E
S31508009EA0F9D190F8512090F85010C06C0023079310
S31508009EB008AC069408240594049403930323029398
S31508009EC0F523019309230093212301F092FB0AB09D
S31508009ED010BD10B58CB005238DF8243010238DF8ED
S31508009EE02B3001238DF82C3002238DF82D301223C8
S31508009EF08DF82E304B1E09AA053113F8014F02F8CA
S31508009F00014F8B42F9D190F8512090F85010C06C4F
S31508009F100023079309AC06940B2405940494039331
S31508009F20032302930523019309230093212301F0B8
S31508009F3060FB0CB010BD00002DE9F04792B0044656
S31508009F401F4690F85480002380F85430C66C336856
S31508009F501B6890F8501030469847002800F0EF80AC
S31508009F6081464FF4967002F03DFB94F8503000227B
S31508009F701146E06C01F046FC054638B1002389F825
S31508009F80063023689B6820469847D9E0002389F85D
S31508009F90063033681B6894F85010304698470028F6
S31508009FA000F0D280877104F151094B46012294F8DA
S31508009FB05010E06C00F0A9FF05460028E1D1B4F87E
S31508009FC0762040F24C539A4246D04746B8F1000FE5
S31508009FD000F08B805D4EDFF87881DFF878A1636F3B
S31508009FE0B3420CBFCDF80CA0CDF80C80231D04930A
S31508009FF000228DF82820ADF82A208DF83C208DF80F
S3150800A0003D208DF83E208DF844200BABCDF8153059
S3150800A01007939DF814108DF821108DF820100993D8
S3150800A02094F8501003AB00932B46E06C01F0C1FB8B
S3150800A030002840F0828094F85E20032A59DC013516
S3150800A040EDB2BD42CBDB00231A4694F85010E06C03
S3150800A05001F0D8FBD12594E7B4F87430B3F51A7F2C
S3150800A06007D040F22F42934203D040F2D5329342B2
S3150800A070ABD1642002F0B6FA012394F8512094F883
S3150800A0805010E06C01F0D5FB054600287FF479AF47
S3150800A09063690BB9238B6BB1B4F87430B3F51A7FC7
S3150800A0A003D040F22F42934219D104F114012046FD
S3150800A0B0FFF7E7FE002394F8512094F85010E06C5F
S3150800A0C001F0B7FB00231A4694F85010E06C01F033
S3150800A0D099FB23689B6820469847D12530E004F110
S3150800A0E014012046FFF7F5FEE4E794F85E20032AFC
S3150800A0F0A9DD4B4694F85010E06C00F006FF0546C3
S3150800A10000287FF43EAF94F85D3094F8512094F817
S3150800A1105010E06C01F08DFB054600287FF431AF46
S3150800A1206423A4F884300023A4F8823084F88030AD
S3150800A1302372012384F8793002E0054621E7D62503
S3150800A140284612B0BDE8F087D625F9E7E8215C0A6B
S3150800A1500C0203080002030870B582B004460E46D6
S3150800A160154690F83030042B00F2E480DFE803F05F
S3150800A170030D1E254A0002230372D0F80920026146
S3150800A18043750375012380F830302A46314604F1B9
S3150800A190100002F0C5F90346002874D0D4F8093037
S3150800A1A01A7884F831205B7884F8323004F1220377
S3150800A1B0C4F80930032384F8303094F83230023B6F
S3150800A1C01F2B16D8DFE803F01315104315151515C0
S3150800A1D01515151515151515151515151515151521
S3150800A1E01515151515151546002384F8333007235C
S3150800A1F02372D4F809302361237A637523750423FF
S3150800A20084F8303094F83230042B3FD0052B6AD0CE
S3150800A210022B24D0237F002B00F08580012B40F0F1
S3150800A2208D80E28B002A00F087802B886BB1013A7B
S3150800A230E2833368013333602B88013B9BB22B8062
S3150800A240E28B002A78D0002BF1D100231BE00523EE
S3150800A2502372CEE794F83130023B2372C9E72A46C7
S3150800A260314604F1100002F05BF9034658B194F840
S3150800A270253084F8343004F12003C4F8093000236B
S3150800A28084F830300123184602B070BD2A4631469C
S3150800A29004F1100002F044F903460028F3D094F8BC
S3150800A2A02530E02BE7D194F82630012BE3D194F83A
S3150800A2B038309BB194F82730002BDCD0012384F882
S3150800A2C0333094F8223084F8363094F8233084F802
S3150800A2D0373094F8273084F83530CCE794F82730AF
S3150800A2E0012BC8D1EAE72A46314604F1100002F0EC
S3150800A2F017F903460028C6D094F83330002BBAD095
S3150800A30060680028B7D094F8373094F8362094F867
S3150800A3103410056804F12006019694F83560009615
S3150800A3202D68A847A7E794F83130023BE383012359
S3150800A330237776E70123A6E700232377E38B002B11
S3150800A34099D000239FE710B582B00446ADF80610F1
S3150800A3500092BDF806303BB10DF10602694620466B
S3150800A360FFF7FAFE0028F4D102B010BD70B582B02E
S3150800A37004460E46154690F83030042B00F2E48069
S3150800A380DFE803F0030D1E254A0002230372D0F806
S3150800A3900920026143750375012380F830302A4687
S3150800A3A0314604F1100002F0BBF80346002874D0C9
S3150800A3B0D4F809301A7884F831205B7884F832307A
S3150800A3C004F12203C4F80930032384F8303094F8E2
S3150800A3D03230023B1F2B16D8DFE803F01315104363
S3150800A3E0151515151515151515151515151515150F
S3150800A3F0151515151515151515151546002384F883
S3150800A400333007232372D4F809302361237A63751E
S3150800A4102375042384F8303094F83230042B3FD067
S3150800A420052B6AD0022B24D0237F002B00F08580D1
S3150800A430012B40F08D80E28B002A00F087802B8864
S3150800A4406BB1013AE2833368013333602B88013BF1
S3150800A4509BB22B80E28B002A78D0002BF1D1002307
S3150800A4601BE005232372CEE794F83130023B2372B2
S3150800A470C9E72A46314604F1100002F051F80346AE
S3150800A48058B194F8253084F8343004F12003C4F820
S3150800A4900930002384F830300123184602B070BD15
S3150800A4A02A46314604F1100002F03AF8034600281D
S3150800A4B0F3D094F82530FF2BE7D194F82630012BFA
S3150800A4C0E3D194F838309BB194F82730002BDCD0D0
S3150800A4D0012384F8333094F8223084F8363094F81F
S3150800A4E0233084F8373094F8273084F83530CCE7B1
S3150800A4F094F82730012BC8D1EAE72A46314604F1F9
S3150800A500100002F00DF803460028C6D094F8333040
S3150800A510002BBAD060680028B7D094F8373094F882
S3150800A520362094F83410056804F12006019694F84C
S3150800A530356000962D68A847A7E794F83130023BA6
S3150800A540E3830123237776E70123A6E7002323770E
S3150800A550E38B002B99D000239FE710B582B0044601
S3150800A560ADF806100092BDF806303BB10DF10602B3
S3150800A57069462046FFF7FAFE0028F4D102B010BD5E
S3150800A58010B50446436803B1984723689B6920467B
S3150800A590984710BD70477047704708B50022427546
S3150800A5A080F82520026180F82A200368DB6998472D
S3150800A5B008BD10B582B004468189027D0132D2B247
S3150800A5C0027500F12803009300F118038068FFF76D
S3150800A5D010FC23689B6820469847092384F82A308C
S3150800A5E002B010BD90F82A30002B4FD1F0B583B0D9
S3150800A5F00446806890F8463033B1437A23B9637DC0
S3150800A60013B994F825302BB1236913F0010F15D12E
S3150800A61003B0F0BD0123437284F82530A068418B4E
S3150800A620A1810022226122751123009304F12603D9
S3150800A630FFF733FB022384F82A30E9E704F12607FB
S3150800A64004F11605227DA1890126019600953B464F
S3150800A650FFF747FB304601F0C5FF227DA18900239D
S3150800A660019300953B46A068FFF73BFB237D3344E7
S3150800A6702375304601F0B6FF2B46227DA189A068D6
S3150800A680FFF75DFB042384F82A30C1E77047000012
S3150800A69070B5064618483060B16089B1486E58B141
S3150800A6A00120044601EB84056D6E35B10130C0B258
S3150800A6B004460328F6DD03E0002401EB84014E6618
S3150800A6C00E493160002186F82410F1613162B068C4
S3150800A6D080F84820B2681361702386F8263086F819
S3150800A6E02710712386F8283086F829103046FFF798
S3150800A6F054FF304670BD00BF7C0203080489020877
S3150800A70010B584B0034690F82420012A84BF00229D
S3150800A71080F8242090F8241041F0700104AA02F869
S3150800A720011D81898068DC7D01949B7D009301234E
S3150800A730FFF770FA04B010BDF0B583B0044690F880
S3150800A7402A30023B072B09D8DFE803F03D4F04A364
S3150800A75010687A8D036913F0020F01D103B0F0BDBA
S3150800A760FFF7CEFF062384F82A30F7E7036913F0CC
S3150800A770100FF3D000F1280700F11805027D818932
S3150800A7800126019600953B468068FFF7AAFA3046EF
S3150800A79001F028FF227DA1890023019300953B46FD
S3150800A7A0A068FFF79EFA237D33442375304601F0EF
S3150800A7B019FF2B46227DA189A068FFF7C0FA082356
S3150800A7C084F82A30CAE7036913F0040FC6D0027D5D
S3150800A7D00132D2B2027500F1160381898068FFF74B
S3150800A7E0AEFA032384F82A30B8E7036913F0020F98
S3150800A7F0B4D0FFF785FF012001F0F4FE227D013277
S3150800A800D2B22275A1891323009304F12803A06804
S3150800A810FFF743FA072384F82A309FE7036913F002
S3150800A820400F9BD0027D0132D2B2027500F11803A7
S3150800A83081898068FFF783FA082384F82A308DE730
S3150800A840036913F0200F89D08268002382F8463006
S3150800A850826882F848300125457503681B69984760
S3150800A86084F82A507AE7036913F0800F3FF476AF2D
S3150800A870027D0132D2B20275818900F12603009366
S3150800A88000F116038068FFF7B4FA052384F82A3026
S3150800A89064E7036913F0080F3FF460AF81898068A5
S3150800A8A0FEF7ACFF4FF6FF73A3810023236184F8FC
S3150800A8B02A3053E770B582B083685A7A52B993F84A
S3150800A8C047203AB1427D2AB990F8252012B90A7A6A
S3150800A8D0022A06D086890A78F3B29A4215D002B0BF
S3150800A8E070BD4C7B0A7B42EA0422112AF2D100226F
S3150800A8F083F8472084680123637280F825308368CB
S3150800A9005B8B838180F82A20E4E74A78331243F088
S3150800A91020039A42E3D10D4604468B79CA7943EA65
S3150800A9200221012908D094F82810994200F00781DD
S3150800A9302046FFF701FFD2E72B7A012BF8D0032B2D
S3150800A9401ED0022B4FD0052B6BD0042B00F0918024
S3150800A950062B00F0B380072BEAD12B7BA27D9A4207
S3150800A96000F0E180227E9A42E2D16A7B637E9A42B7
S3150800A970DED16B7A2375236943F080032361D7E719
S3150800A9806A7C2B7C53EA0223D2D1EA7CAB7C53EA5D
S3150800A9900223CDD1AB7B94F826209A4213D094F8A3
S3150800A9A028209A42C4D1EA7B94F829309A42BFD12A
S3150800A9B06B7A23752B7B23766B7B6376236943F04F
S3150800A9C040032361B4E7E97B94F827209142E6D156
S3150800A9D06B7A23752B7BA3756B7BE375236943F031
S3150800A9E004032361A4E76A7B2B7B43EA0223112B2A
S3150800A9F00CD0132B9CD16B7A2375AB7B2376EB7B20
S3150800AA006376236943F01003236191E76B7A237514
S3150800AA10AB7BA375EB7BE375236943F001032361E5
S3150800AA2086E76A7C2B7C53EA022381D12B7B94F838
S3150800AA3026209A4211D094F828209A427FF478AFBB
S3150800AA406A7B94F829309A427FF472AF6B7A237541
S3150800AA50236943F0200323616AE7697B94F827207A
S3150800AA609142E8D16B7A2375236943F00203236187
S3150800AA705EE72B7B94F826209A4212D094F8282079
S3150800AA809A427FF455AF6A7B94F829309A427FF44C
S3150800AA904FAF04F118036A7A3146A068FFF77AF9CE
S3150800AAA046E7697B94F827209142E7D104F116031B
S3150800AAB06A7A3146A068FFF76DF939E72B7B94F877
S3150800AAC026209A421AD094F828209A427FF430AF6A
S3150800AAD06A7B94F829309A427FF42AAF6A7A2275FB
S3150800AAE004F11803009304F128033146A068FFF720
S3150800AAF0A4F923689B682046984719E7697B94F868
S3150800AB0027209142DFD16A7A227504F11603009351
S3150800AB1004F126033146A068FFF78FF923689B687E
S3150800AB202046984704E7697BE27D91427FF41AAF95
S3150800AB306B7A2375236943F008032361F8E694F8D2
S3150800AB40293093427FF4F4AE2B7AA12B7FF4F0AE32
S3150800AB502E79711E23685B6905F10902C9B2204680
S3150800AB6098476B7A012B10D0022B7FF4E1AE206A4E
S3150800AB7000283FF4DDAEB31E02680A350095156855
S3150800AB80DBB200222146A847D2E6E06900283FF456
S3150800AB90CFAEB31E02680A3500951568DBB20022EF
S3150800ABA02146A847C4E603292CD8DFE801F0020DA0
S3150800ABB01721007A00F00F00072825D030B30128A6
S3150800ABC014BF002001207047007A00F00F000138FA
S3150800ABD0C0B202288CBF002001207047007A00F01E
S3150800ABE00F000338C0B202288CBF0020012070472E
S3150800ABF0007A00F00F000538C0B202288CBF00208A
S3150800AC0001207047002070470120704701207047D7
S3150800AC1008B5032908DD8068C0F31700044B5B5CA0
S3150800AC20D84000F0010008BDFFF7BDFF08BD00BF12
S3150800AC30248902080A4B5B5C01229A4090F843304B
S3150800AC40B0F8441043EA012323EA020180F84310CE
S3150800AC50090AA0F844101A4214BF012000207047C0
S3150800AC6024890208082904D009290CBF007B002082
S3150800AC707047C07A704701440879704770B5044632
S3150800AC8001295BDD1346002A58D01278012A0DD017
S3150800AC90112A56D1032954DDCA1ED2B23C2A28BF2E
S3150800ACA03C22D91C04301BF025FC08E04A1ED2B20F
S3150800ACB03C2A28BF3C22591C04301BF01BFCA26806
S3150800ACC0C2F31702236CC3F317039A4236D022EA5B
S3150800ACD0030384F843301B0AA4F84430236C62F358
S3150800ACE01703236400212046FFF75DFF0646054645
S3150800ACF001212046FFF757FF10B146F00205EDB2D5
S3150800AD0002212046FFF74FFF10B145F00405EDB2CA
S3150800AD1003212046FFF747FF10B145F00805EDB2BD
S3150800AD2094F84E309D4209D025EA030394F843204F
S3150800AD3063F3030284F8432084F84E5094F84D30A8
S3150800AD4003B970BD23681B6804F14601204698477D
S3150800AD50F7E799B110B40C46C37C8B4218D002228F
S3150800AD601346C3EBC30303441B7BA34208D001323B
S3150800AD70D2B213460F2AF4DD002006E008307047E9
S3150800AD8042B10830C2EBC20210445DF8044B70476A
S3150800AD900122F6E70020F8E711F0800F49D130B418
S3150800ADA00546072B47DC7AB9EC7C14B30220044627
S3150800ADB0C4EBC4042C44247B5CB1441CE0B20446B6
S3150800ADC00F28F5DD002037E0C0790728ECD10020F0
S3150800ADD032E088B3A9B972B1C0EBC0032B44412253
S3150800ADE01A73EB790133EB71C0EBC0002844007B82
S3150800ADF022E00120EEE7C0EBC0032B4401221A73C0
S3150800AE00F2E74FF0000461F3C5046AB144F0400468
S3150800AE10EB790133DBB2EB7163F30204C0EBC000DC
S3150800AE2028440473E0B207E06FF3861463F3020460
S3150800AE30F4E700207047002030BC704770B4134B0D
S3150800AE4003600022C2710273012343738273051DD6
S3150800AE5085600271082141710F2161F387028271B1
S3150800AE60024600241E46D47416755475C3EBC301F6
S3150800AE7001448D6001330732102BF4D1002380F88A
S3150800AE80B8301122024B1A7070BC7047980203083A
S3150800AE903C0A002010B491B10C46C37C8B4228D0E2
S3150800AEA002210B46C3EBC30303441B7BA3421AD000
S3150800AEB00131C9B20B460F29F4DD00201CE000F170
S3150800AEC00801F1B10868B8B14C79E4B10378934246
S3150800AED012D0002303300133DBB2A3420BDA017828
S3150800AEE09142F7D108E051B10830C1EBC1010144E4
S3150800AEF0E7E70121F8E700205DF8044B70470020DA
S3150800AF00FAE70020F8E70020F6E723B330B41D4639
S3150800AF1089B1C37C8B421CD002242346C3EBC303EE
S3150800AF2003441B7B8B420ED00134E4B223460F2C1C
S3150800AF30F4DDD62005E0083088B10171056042715C
S3150800AF40002030BC704744B10830C4EBC404204428
S3150800AF50F2E70124F8E7D8207047D620F1E7D62093
S3150800AF60EFE7000070B582B00C4616460C4D00227D
S3150800AF701021284602F0C8F944F002048DF804406E
S3150800AF808DF805604FF0FF33022201A9054803F04A
S3150800AF9097FD01221021284602F0B6F902B070BDCD
S3150800AFA00010024074CE00202DE9F04F83B082468F
S3150800AFB0174601939DF83090012500EB810802F1B0
S3150800AFC01E0B19E057BB0122E8215046FFF7CAFFBE
S3150800AFD0662001F007FBD8F8780003681C684B4622
S3150800AFE0019A3946A0470D282AD1022E2CDC642066
S3150800AFF001F0F8FA0135EDB26E1EF6B2D8F878000F
S3150800B00003685C684B46019A3946A047E028D9D0C0
S3150800B0100D280AD00028DED0044609E05AF82B008D
S3150800B02003685B6901999847D5E7022E04DD044653
S3150800B030204603B0BDE8F08F642001F0D3FAD9E7C3
S3150800B04004460028F4D000E004463FB11E375AF8FB
S3150800B050270003685B6901999847E9E70122E82117
S3150800B0605046FFF77FFF662001F0BCFAE0E70000D4
S3150800B07070B584B004AC04F8091D104D00221021E7
S3150800B080284602F041F90E4E4FF0FF3301222146C1
S3150800B090304603F015FD04A9002301F8013D4FF0E1
S3150800B0A0FF330122304603F0F6FE0122102128461E
S3150800B0B002F02AF99DF80F0004B070BD0010024096
S3150800B0C074CE00202DE9F84F04468A4617469B465B
S3150800B0D001F082FA00F59C5508350026B146B046BF
S3150800B0E04AEA07074FF0F00A01F076FA401B0028F3
S3150800B0F020DA3A4651462046FFF734FFC82601F0C3
S3150800B1006BFA401B00280BDA31462046FFF7B0FFE2
S3150800B11010F0800FF3D08022C8212046FFF722FFC7
S3150800B120F8212046FFF7A4FF00F00F06042E04D0EE
S3150800B1300E2E0CD03046BDE8F88F09F101091FFA2A
S3150800B14089F9BBF1000FCFD0D945CDD1F2E708F187
S3150800B15001085FFA88F8B8F1030FC5D1EAE70000DD
S3150800B1602DE9F04F87B000908B4601929A46109EC3
S3150800B1709DF844300393BAF800904B780293002365
S3150800B180AAF800308B7813F0020F14BF2022102281
S3150800B190E821FFF7E7FE17E0F821009C2046FFF7B5
S3150800B1A067FF80F01000C0F300109BF8023060F3D0
S3150800B1B041038BF8023013F0020F14BF202210222D
S3150800B1C0E8212046FFF7CEFE019B9BF800200021D0
S3150800B1D00098FFF777FF05460628DDD000286AD1D4
S3150800B1E0C821009C2046FFF743FF10F0040F5FD0EC
S3150800B1F030212046FFF73CFF04464845C8BF5FFAA2
S3150800B20089F4BAF80020A9EB020212B222EAE27225
S3150800B210A242A8BF224617460DF11808082308F8C7
S3150800B220013D00221021254802F06EF84FF0FF3349
S3150800B23001224146224803F043FCFFB23A46002168
S3150800B24030461BF07CF94FF0FF333A4631461C482E
S3150800B25003F021FE3E4401221021184802F054F85A
S3150800B2600422C8210098FFF77DFEBAF8003023446F
S3150800B2709BB2AAF80030029A944208DB994506DD8B
S3150800B280039B002BA0D0184601F0ACF99CE7A84612
S3150800B290F8210098FFF7ECFEC0F300109BF8023087
S3150800B2A060F341038BF80230404607B0BDE8F08FE3
S3150800B2B04FF0F008F8E78046F6E700BF00100240B6
S3150800B2C074CE0020F8B50E4689B1C17CB14244D08F
S3150800B2D002252C46C4EBC4040444247BB44235D06E
S3150800B2E00135EDB22C460F2DF4DDD620F8BD00F160
S3150800B2F00805002D38D02968002937D01C4607468E
S3150800B3003146FFF7C7FD206090B383789A080F2A65
S3150800B310A8BF0F2201239340013B069A13803246A9
S3150800B320E0213846FFF71EFED8213846FFF7A0FE73
S3150800B330AB79A3B197F8B82042F002020243D2B221
S3150800B340D8213846FFF70EFE0020F8BD55B100F1AA
S3150800B3500801C5EBC5050D44CBE70125F7E700F065
S3150800B360F902EDE7D620F8BDD620F8BDD720F8BDFE
S3150800B370DB20F8BD30B585B004461D46002303938F
S3150800B380ADF80A300DF10A03009303ABFFF79AFFF5
S3150800B390034610B1184605B030BDBDF80A209DF821
S3150800B3A024300193089B00932B4603992046FFF708
S3150800B3B0D7FE0346EEE70000F0B583B00D46174604
S3150800B3C01C46114E00221021304601F09DFF45F023
S3150800B3D0020502A901F8015D0C4D4FF0FF33012269
S3150800B3E0284603F06DFB4FF0FF333A4621462846C0
S3150800B3F003F066FB3C4401221021304601F084FF2D
S3150800B400204603B0F0BD00BF0010024074CE0020F5
S3150800B4102DE9F04F85B00192009391F8018008F16B
S3150800B420FF33DBB23F2B04D9DA25284605B0BDE841
S3150800B430F08F04460E4601F0CFF800F59C5A0AF143
S3150800B440080AB37803F00103002B14BF80224022B8
S3150800B450E8212046FFF786FD009B002B00F0A98017
S3150800B4604FF0C80BCDF80880BDF80830009A934213
S3150800B47028BF134603935FFA83F80E9B42461021B2
S3150800B4802046FFF799FF424638212046FFF76AFD16
S3150800B490327842F02002F0212046FFF763FD594634
S3150800B4A02046FFF7E5FD10F0800FF8D080225946B8
S3150800B4B02046FFF757FDF8212046FFF7D9FD00F093
S3150800B4C00F054FF000094F4663E001F085F8A0EB41
S3150800B4D00A0000285FDA062D1CD00E2D15D0042D83
S3150800B4E00AD0F8212046FFF7C3FDC0F34010B37811
S3150800B4F060F30003B37098E709F101091FFA89F9A7
S3150800B500019BEBB199451BD1EBE70137FFB2032F3E
S3150800B51016D1E6E7F8212046FFF7AAFD80F02000BD
S3150800B520C0F34010B37860F30003B37003F001036F
S3150800B530002B14BF80224022E8212046FFF712FD87
S3150800B540002238212046FFF70DFD0E9B1A781021A0
S3150800B5502046FFF707FD424638212046FFF702FD41
S3150800B560327842F02002F0212046FFF7FBFC5946CC
S3150800B5702046FFF77DFD10F0800FF8D0802259464F
S3150800B5802046FFF7EFFCF8212046FFF771FD00F093
S3150800B5900F05002D99D10099039A8B1A9BB219466B
S3150800B5A000930E9B184610440E9000297FF45CAF5A
S3150800B5B097E7002595E730B585B004461D46002374
S3150800B5C00393ADF80A300DF10A03009303ABFFF7B6
S3150800B5D079FE034610B1184605B030BDBDF80A20FD
S3150800B5E0089B00932B4603992046FFF711FF034655
S3150800B5F0F1E72DE9F04F8BB0029003921C46BDF897
S3150800B6006090BDF86470DDF868801B9E0023069381
S3150800B610ADF816300DF11603009306ABFFF752FE90
S3150800B620054618B128460BB0BDE8F08F8DF81C40CA
S3150800B6309DF850308DF81D309DF854308DF81E3029
S3150800B6409DF858308DF81F30BDF85C30ADF82030C5
S3150800B650ADF8229007AB08222021029D2846FFF765
S3150800B660ABFEBDF81630039A10212846FFF72AFDCF
S3150800B67005460028D6D104F08004B8F1000F5DD045
S3150800B680002C47D0069A937843F002039370B9F1D9
S3150800B690000F58D04C464FF0000B26E0DDF818A0F6
S3150800B6A0F8210298FFF7E4FC80F02000C0F3401070
S3150800B6B09AF8023060F341038AF8023013E03368DF
S3150800B6C0D3F800A0BDF81410A9EB0403ADF8263092
S3150800B6D00DF1260342463046D047BDF81430E41A29
S3150800B6E0A4B2BB422FDB002C36D0ADF81470BDF8DF
S3150800B6F01620CDF804B0CDF8008005AB069902985F
S3150800B700FFF72EFD05460628C8D000288AD1002E48
S3150800B710D5D1E2E7069A937843F001039370BDF812
S3150800B7201620CDF800803B4606990298FFF770FE72
S3150800B730054600287FF476AF802105E0002CCCBFB3
S3150800B740A021802100E0A021BDF81630039A0298B6
S3150800B750FFF7B8FC054665E7A021002D7FF462AF28
S3150800B760F2E730B589B0002407940C9D0695059339
S3150800B77004930394012302930194062300938023E0
S3150800B780FFF737FF09B030BD30B589B000240794FC
S3150800B7900D9D0695059304930394022302939DF841
S3150800B7A030300193062300938023FFF722FF09B068
S3150800B7B030BDF0B599B005460E4617461C4608AB8F
S3150800B7C0019300940923FFF7DFFF034610B11846DB
S3150800B7D019B0F0BD1E9B079308AB0693402305934B
S3150800B7E0BDF82230049300230393022302930194A5
S3150800B7F00623009380233A4631462846FFF7F9FE8A
S3150800B8000346E4E710B588B0002407940694059427
S3150800B8100494039402940193052300932346FFF7A7
S3150800B820E8FE04464FF4967000F0DCFE204608B0A9
S3150800B83010BD10B588B000240794069405940494A6
S3150800B840039402940193092300932346FFF7D1FE3C
S3150800B85008B010BD002900F01E832DE9F04F99B0FD
S3150800B86017918346C1EBC10303441B7B03F0070210
S3150800B870099213F0400F5FD0012303930F930193AE
S3150800B880039A531EDBB20E2B00F21E820F2A4ADCE5
S3150800B890C2EBC2035B441B7BC3F3C203099A934200
S3150800B8A059D1039B002B3ED0039B1193C3EBC303D3
S3150800B8B05B441B7B03F007020A9213F0400F67D024
S3150800B8C001230493049A531EDBB20E2B00F2068260
S3150800B8D00F2A54DCC2EBC2035B441B7BC3F3C203CF
S3150800B8E00A9A934262D1049B002B48D0049B129378
S3150800B8F0C3EBC3035B441B7B03F007020B9213F0F5
S3150800B900400F00F0D3810F9B059396E1C3EBC3026A
S3150800B9105A44127BC2F3C20209998A421DD00133E6
S3150800B920DBB20F2BF2DD9BF80730099A934204BF6E
S3150800B93003F1FF338BF80730179BC3EBC3025A4456
S3150800B940002313730121517393730BF1040393605E
S3150800B95019B0BDE8F08F039BE1E70393A1E7012344
S3150800B9600393A1E7C3EBC3025A44127BC2F3C20294
S3150800B9700A998A421CD00133DBB20F2BF2DD9BF801
S3150800B98007300A9A934204BF03F1FF338BF8073056
S3150800B990119BC3EBC3035B4400221A734FF00101EA
S3150800B9A059739A730BF104029A6069E7049BE2E7FC
S3150800B9B0049398E70F9B049398E7019B05935DE131
S3150800B9C0019B069314E1019B0793C5E0DDF80490FB
S3150800B9D0CAE1DDF820909BF80730169A934204BF17
S3150800B9E003F1FF338BF80730109BC3EBC3035B44AB
S3150800B9F000221A734FF0010159739A730BF104026E
S3150800BA009A6009F1FF33DBB20E2B00F28F81B9F190
S3150800BA100F0F69DCC9EBC9035B441B7BC3F3C20385
S3150800BA200E9A934200F09C810E9A89E1DDF82090E7
S3150800BA30D1E7019FC8E1019DF0E1019C17E29BF85F
S3150800BA400730B34204BF03F1FF338BF80730C9EB65
S3150800BA50C909D9444FF0000389F80C304FF00103A7
S3150800BA6089F80D304FF0000389F80E300BF1040306
S3150800BA70C9F808306B1EDBB20E2B00F2B7810F2D0A
S3150800BA8009DCC5EBC5035B441B7BC3F3C203434513
S3150800BA9040F0B481BFE19BF80730434504BF03F18A
S3150800BAA0FF338BF80730029BC3EBC3035B440022CA
S3150800BAB01A734FF0010159739A730BF104029A60D5
S3150800BAC07B1EDBB20E2B00F267810F2F09DCC7EB5A
S3150800BAD0C7035B441B7BC3F3C203534540F0648131
S3150800BAE06FE1DDF8209076E79BF807300E9A9342CF
S3150800BAF004BF03F1FF338BF80730159BC3EBC30371
S3150800BB005B4400221A734FF0010159739A730BF1C3
S3150800BB1004029A60079A531EDBB20E2B00F2FC80D1
S3150800BB200F2A2DDCC2EBC2035B441B7BC3F3C203A3
S3150800BB300D9A93420ED00D99079B0133DBB20F2B5A
S3150800BB401EDCC3EBC3025A44127BC2F3C2028A420A
S3150800BB50F3D10793079B9BB1079A1592C2EBC203D1
S3150800BB605B441B7B13F0400FC7D0C2EBC2035B4498
S3150800BB701B7B03F007030E93DDF804A0D14640E7CC
S3150800BB809BF807300D9A934204BF03F1FF338BF8F5
S3150800BB900730149BC3EBC3035B4400221A734FF0B0
S3150800BBA0010159739A730BF104029A60069A531E9F
S3150800BBB0DBB20E2B00F2A6800F2A28DCC2EBC203EA
S3150800BBC05B441B7BC3F3C2030C9A93420ED00C99B9
S3150800BBD0069B0133DBB20F2B19DCC3EBC3025A44B5
S3150800BBE0127BC2F3C2028A42F3D10693069B73B153
S3150800BBF0069B1493C3EBC3035B441B7B03F007024A
S3150800BC000D9213F0400FC4D0019B079382E79BF86F
S3150800BC1007300C9A934204BF03F1FF338BF80730C1
S3150800BC20139BC3EBC3035B4400221A734FF0010155
S3150800BC3059739A730BF104029A60059A531EDBB284
S3150800BC400E2B55D80F2A28DCC2EBC2035B441B7B9C
S3150800BC50C3F3C2030B9A93420ED0059B0133DBB2A2
S3150800BC600F2B1ADCC3EBC3025A44127BC2F3C2027F
S3150800BC700B998A42F2D10593059B73B1059B1393E1
S3150800BC80C3EBC3035B441B7B03F007020C9213F060
S3150800BC90400FC5D0019B069388E79BF807300B9A9F
S3150800BCA0934204BF03F1FF338BF80730129BC3EBB3
S3150800BCB0C3035B4400221A734FF0010159739A7348
S3150800BCC00BF104029A60FDE59BF81330C3F3C20337
S3150800BCD0099A93423FF443AE012320E69BF81330BA
S3150800BCE0C3F3C2030A9A93423FF464AE0F9B42E63B
S3150800BCF09BF81330C3F3C2030B9A93423FF45DAE2D
S3150800BD00019BABE79BF81330C3F3C2030C998B4234
S3150800BD103FF456AE019B5CE79BF81330C3F3C203AE
S3150800BD200D998B423FF44FAE019B06E79BF8133003
S3150800BD30C3F3C2030E9A93423FF448AEDDF804906B
S3150800BD4009F101095FFA89F9B9F10F0F3FF7CCAE8E
S3150800BD50C9EBC9035B441B7BC3F3C2039342EFD110
S3150800BD60B9F1000F3FF4C0AECDF84090C9EBC90356
S3150800BD705B441B7B13F0400F3FF436AEC9EBC90397
S3150800BD805B441B7B03F007031693DDF804A0CDF88C
S3150800BD90209057469A4693E69BF81330C3F3C2039E
S3150800BDA053453FF446AE019F0137FFB20F2F3FF7C9
S3150800BDB010AEC7EBC7035B441B7BC3F3C2035345F3
S3150800BDC0F2D1002F3FF432AE0297C7EBC7035B44AC
S3150800BDD01B7B13F0400F3FF466AEC7EBC7035B440B
S3150800BDE093F80C8008F00708019D43E69BF813308A
S3150800BDF0C3F3C20343453FF41EAE019D0135EDB2C0
S3150800BE000F2D3FF748AEC5EBC5035B441B7BC3F359
S3150800BE10C2034345F2D1002D3FF43DAEA946C5EB1A
S3150800BE20C5035B441B7B13F0400F3FF410AEC5EB14
S3150800BE30C5035B441E7B06F00706019C1BE09BF8C6
S3150800BE401330C3F3C203B3423FF4F7AD019C013488
S3150800BE50E4B20F2C3FF7F3ADC4EBC4035B441B7B82
S3150800BE60C3F3C203B342F2D1002C3FF4E8AD214636
S3150800BE705846FFF7EFFC631EDBB20E2BDFD80F2CFC
S3150800BE803FF7DDADC4EBC4035B441B7BC3F3C203BE
S3150800BE90B342DCD1E8E770472DE9F041412911D0DA
S3150800BEA0C37C8B4237D002221346C3EBC303034439
S3150800BEB01B7B8B421AD00132D2B213460F2AF4DD0D
S3150800BEC0BDE8F0810246012300241E46051DD474F0
S3150800BED016755475C3EBC30101448D6001330732EF
S3150800BEE0102BF4D10023C371BDE8F0818AB1054651
S3150800BEF01746C2EBC20303441B7B13F0400F14D052
S3150800BF00C2EBC20283181E7B06F007060124A04670
S3150800BF102FE0BDE8F0810122E9E7444625E0EB7908
S3150800BF20B34204BF03F1FF33EB71C7EBC707EB1945
S3150800BF3000221A73012159739A7304359D60BDE86E
S3150800BF40F081EB7CC3F3C203B342E6D04446013426
S3150800BF50E4B20F2CE3DCC4EBC4032B441B7BC3F312
S3150800BF60C203B342F3D1002CD9D021462846FFF7A5
S3150800BF7071FC631EDBB20E2BE3D80F2CCFDCC4EBAF
S3150800BF80C4032B441B7BC3F3C203B342DFD1EAE7E6
S3150800BF902DE9F84310F1080600F0AA808468002C01
S3150800BFA000F0A880837311F0800F40F0AB80072A59
S3150800BFB000F3A880C47C44B302252C46C4EBC40411
S3150800BFC00444247B34B10135EDB22C460F2DF5DD42
S3150800BFD0D42590E0002D00F09580C1B9C5EBC505C4
S3150800BFE0054401242C73C27CA24244D002210A468D
S3150800BFF0C2EBC2020244127BA24219D00131C9B275
S3150800C0000A460F29F4DDD62575E00125E5E7002760
S3150800C0103C4661F3C50467F3861462F30204C5EB74
S3150800C020C50505442C73E4B2002CDCD1D42562E0A6
S3150800C030002963D0C1EBC101711861D007468B7125
S3150800C040234600221146FFF7DDFB0546002852D09D
S3150800C050412C12D0FB7CA34234D002221346C3EBF8
S3150800C060C3033B441B7BA3421AD00132D2B2134608
S3150800C0700F2AF4DD3FE00121DCE73A4601230020E0
S3150800C0801E463C1DD07416755075C3EBC301394462
S3150800C0908C6001330732102BF4D10023FB712AE0A0
S3150800C0A04AB39046C2EBC2033B441B7B13F0400FD6
S3150800C0B012D0C2EBC202BB181E7B06F0070601248B
S3150800C0C0A14639E00122ECE74C4631E0FB79B34260
S3150800C0D004BF03F1FF33FB71C8EBC80807EB08037D
S3150800C0E000221A73012159739A73381D986002E069
S3150800C0F0D62500E0D7252846BDE8F883D625FAE7F1
S3150800C100D625F8E7D425F6E7FB7CC3F3C203B3428A
S3150800C110DAD04C460134E4B20F2CD7DCC4EBC403A6
S3150800C1203B441B7BC3F3C203B342F3D1002CCDD0EF
S3150800C13021463846FFF78EFB631EDBB20E2BE3D88B
S3150800C1400F2CC3DCC4EBC4033B441B7BC3F3C20301
S3150800C150B342DFD1EAE72DE9F04F8DB005460291EB
S3150800C1600392994600218DF8181008238DF8193086
S3150800C1700B460F2262F387038DF81A3003681B6893
S3150800C1809847002800F092800446066806AB0360CC
S3150800C19080F8069007AB0093122300221146284622
S3150800C1A0FFF7DFFA26608046002840F08180BDF858
S3150800C1B024300493BDF826B09DF8203005939DF8E9
S3150800C1C021A0044600270EE0CDF80090039B029AB2
S3150800C1D021462846FEF7E8FED12825D10134E4B2E7
S3150800C1E027460F2C24DC05EB8706B06F0028F5D010
S3150800C1F003681B6998470028F0D1B06F03681B6A6B
S3150800C200514698470028E9D0B06F03689B695A469B
S3150800C210049998470028D7D1B06F0368DB69059958
S3150800C22098470028D0D1D9E70F2FD8BF80463FDDE1
S3150800C230444600264F460BE0B06F03689B695A4692
S3150800C2400499984710B30134E4B226460F2C25DC2E
S3150800C25005EB8606B06F0028F5D003681B6998477A
S3150800C2600028F0D1B06F03681B6A5146984700282A
S3150800C270E2D10097039B029A21462846FEF794FED0
S3150800C28000F0F703D12BDED0804611E0B06F0368CB
S3150800C290DB69059998470028D5D1EAE73B46039A12
S3150800C2A002992846FFF774FE804601E04FF0D6084B
S3150800C2B040460DB0BDE8F08F10B50446F821FEF7EC
S3150800C2C0D7FE00F0C00040282DD007D9802811D00D
S3150800C2D0C0280ED10122204B1A7010BD40B9D122B8
S3150800C2E0D8212046FEF73EFE00221B4B1A7010BDD1
S3150800C2F010BD10BDD8212046FEF7BAFE10F0020F79
S3150800C30008D1C922D8212046FEF72CFE0222124B5C
S3150800C3101A7010BDCB22D8212046FEF723FE032231
S3150800C3200D4B1A7010BDD8212046FEF7A1FE10F05D
S3150800C330020F08D1CB22D8212046FEF713FE03228E
S3150800C340054B1A7010BDC922D8212046FEF70AFEF1
S3150800C3500222014B1A7010BD1AD300202DE9F041B4
S3150800C36007464FF400516B4800F0C8FF38B16A4BD6
S3150800C3701B78032B40D8DFE803F01A142926C821B6
S3150800C3803846FEF775FE10F0200F05D10022C821A9
S3150800C3903846FEF7E7FDEAE73846FFF78DFF202225
S3150800C3A0F5E713225D4B1A704FF0000816E05B4B59
S3150800C3B01B7803F0F003102B21D01122574B1A706B
S3150800C3C04FF000080AE04FF0010801E04FF00008BE
S3150800C3D0524B1B7803F0F003102B05D007F17406B7
S3150800C3E007F1B40534460FE000F0F6F84B4BC830B9
S3150800C3F0586020221A70F1E74FF00008EEE74FF078
S3150800C4000008EBE7AC4207D054F8040F0028F9D02F
S3150800C4100368DB689847F5E7404B1B78402B45D007
S3150800C42007D8202B2ED0302B36D0112B17D0BDE8AD
S3150800C430F081512B51D0802B59D0502BF7D1C821E0
S3150800C4403846FEF715FE10F0400FF0D0334C512356
S3150800C450237000F0C1F814306060BDE8F081002355
S3150800C46087F8B83004E003689B689847A64204D06A
S3150800C47056F8040F0028F6D1F8E71222274B1A704F
S3150800C480BDE8F08100F0A8F8244B5B68C31A002BBE
S3150800C490CDDB3022214B1A700122E8213846FEF7FF
S3150800C4A061FD40221D4B1A70BDE8F081E82138462F
S3150800C4B0FEF7DEFD10F0010FB9D1D8213846FEF798
S3150800C4C0D7FD40F00802D2B2D8213846FEF74AFD19
S3150800C4D05022124B1A70BDE8F08100F07DF80F4B20
S3150800C4E05B68C31A002BA2DB80220C4B1A704346EA
S3150800C4F0002211463846FFF72EFE30B1D22896D0D4
S3150800C500A022064B1A70BDE8F0819022034B1A70E0
S3150800C5108DE700BF000802401AD300203C0A00201D
S3150800C5200368D3B130B40479CCB113889BB10B68D6
S3150800C5301D7843791B1B0468E5540379013B037195
S3150800C5401388013B13800B6801330B60047934B1FF
S3150800C5501388002BEBD1002004E0002070474379B4
S3150800C5600371012030BC704710B50446074B1868A4
S3150800C570074BA3FB0030800900F00CFB0022214684
S3150800C5804FF0FF3000F0BCFA002010BD000000207C
S3150800C590D34D621008B50B4B1A6842F400721A6044
S3150800C5A01A6842F480621A601A6842F480721A6045
S3150800C5B0032000F093FA0020FFF7D6FF19F016FAC9
S3150800C5C0002008BD003C0240024A1368013313608C
S3150800C5D0704700BF4CD30020014B1868704700BF56
S3150800C5E04CD3002010B582B00190FFF7F5FF044642
S3150800C5F0FFF7F2FF019B001B9842F9D302B010BD6A
S3150800C60070470000002800F0BC8010B50446036C93
S3150800C61043B1236C13F0100F0AD00120002384F8CD
S3150800C6203C3010BD436480F83C30FFF7E9FFF0E783
S3150800C630236C23F4885323F0020343F00203236494
S3150800C640514B5A6822F440325A605A6861680A4364
S3150800C6505A602268536823F48073536022685368CB
S3150800C660216943EA012353602268536823F0407323
S3150800C670536022685368A1680B4353602268936825
S3150800C68023F40063936022689368E1680B43936020
S3150800C690A26A3E4B9A4251D02268936823F070638F
S3150800C6A0936022689368A16A0B4393602268936833
S3150800C6B023F04053936022689368E16A0B439360C2
S3150800C6C02268936823F00203936022689368A1693D
S3150800C6D043EA41039360236A002B3AD122685368E0
S3150800C6E023F4006353602268D36A23F47003D36289
S3150800C6F02168CB6AE269013A43EA0253CB622268AF
S3150800C700936823F40073936022689368216B43EA65
S3150800C710412393602268936823F4806393602268B8
S3150800C7209368616943EA8123936000206064236CFF
S3150800C73023F0030343F0010323646FE72268936839
S3150800C74023F0706393602268936823F040539360E4
S3150800C750B6E72268536843F4006353602268536857
S3150800C76023F4604353604FF4604393FAA3F3B3FA98
S3150800C77083F221684868636A013B934003434B6030
S3150800C780B1E70120704700BF002301400100000FF8
S3150800C79082B00023019390F83C30012B63D001232B
S3150800C7A080F83C3003689A6812F0010F14D19A6831
S3150800C7B042F001029A60304B1B68304AA2FB032301
S3150800C7C09B0C03EB43030193019B2BB1019B013B9C
S3150800C7D00193019B002BF9D10268936813F0010FAE
S3150800C7E044D0036C23F4E06323F0010343F480731D
S3150800C7F00364536813F4806F05D0036C23F4405325
S3150800C80043F480530364036C13F4805F1ABF436CCC
S3150800C81023F0060300234364002380F83C306FF0BE
S3150800C82022031360164B5B6813F01F0F0AD10368C7
S3150800C8309A6812F0405F1BD19A6842F080429A606B
S3150800C840002011E002680F4B9A4201D000200BE04D
S3150800C8509B6813F0405F0DD10A4A936843F0804302
S3150800C8609360002000E0022002B070470020FBE73A
S3150800C8700020F9E70020F7E70000002083DE1B43CD
S3150800C880002301400020014003689A6812F4806F73
S3150800C89003D09B6813F4807F1CD170B50C460546FF
S3150800C8A0FFF79AFE06462A68136813F0020F1AD194
S3150800C8B0B4F1FF3FF8D024B1FFF78EFE801B844207
S3150800C8C0F1D22B6C43F004032B64002385F83C302B
S3150800C8D0032070BD036C43F020030364002380F833
S3150800C8E03C30012070476FF0120313602B6C43F441
S3150800C8F000732B642B689A6812F0405F17D1AA69F7
S3150800C900BAB9DA6A12F4700F03D09B6813F4806F11
S3150800C91011D12B6C23F480732B642B6C13F4805F7A
S3150800C9200BD12B6C43F001032B64002070BD002053
S3150800C93070BD002070BD002070BD002070BD03686A
S3150800C940D86C704730B482B00023019390F83C301D
S3150800C950012B00F0B680012380F83C300B68092BC8
S3150800C9603AD90568EA689BB203EB43031E3B0724E2
S3150800C97004FA03F322EA0303EB600468E5680B880C
S3150800C98003EB43031E3B8A6802FA03F32B43E36077
S3150800C9904B68062B35D805686A6B03EB8303053BA2
S3150800C9A01F2404FA03F322EA03036B630468656B26
S3150800C9B00A884B6803EB8303053B02FA03F32B4310
S3150800C9C063630268404B9A424BD0002380F83C30A0
S3150800C9D0184602B030BC704705682A699BB203EB5B
S3150800C9E04303072404FA03F322EA03032B610468CA
S3150800C9F025690B8803EB43028B6893402B4323611D
S3150800CA00C6E70C2B16D805682A6B03EB8303233B72
S3150800CA101F2404FA03F322EA03032B630468256B35
S3150800CA200A884B6803EB8303233B02FA03F32B4381
S3150800CA302363C6E70568EA6A03EB8303413B1F24C1
S3150800CA4004FA03F322EA0303EB620468E56A0A8838
S3150800CA504B6803EB8303413B02FA03F32B43E36280
S3150800CA60AFE70B68122B22D00B68184A934201D005
S3150800CA70112BAAD1164A536843F4000353600A6877
S3150800CA80124B9A42A1D1134B1B68134AA2FB0323EC
S3150800CA909B0C03EB83035B000193019B002B94D053
S3150800CAA0019B013B0193019B002BF9D18DE7084AB5
S3150800CAB0536843F4800353600268034B9A42D3D009
S3150800CAC083E7022085E700BF00200140120000101E
S3150800CAD0002301400000002083DE1B43074AD36879
S3150800CAE023F4E0631B041B0C43F0BF6343F40033D9
S3150800CAF0000200F4E0600343D360704700ED00E0F5
S3150800CB0030B4154BDC68C4F30224C4F10703042BC4
S3150800CB1028BF0423251D062D8CBFE51E00250124EC
S3150800CB2004FA03F3013B1940A940AC40013C2240FA
S3150800CB301143002809DB0901C9B200F1604000F57C
S3150800CB40614080F8001330BC704700F00F000901FF
S3150800CB50C9B2024B1954F6E700ED00E014ED00E007
S3150800CB60420900F01F00012303FA00F0014B43F8C5
S3150800CB702200704700E100E0430900F01F0001228F
S3150800CB8002FA00F02033024A42F82300704700BF39
S3150800CB9000E100E00138B0F1807F0AD2064B586008
S3150800CBA0F021064A82F823100020986007221A60AE
S3150800CBB070470120704700BF10E000E000ED00E07C
S3150800CBC0430900F01F00012202FA00F06033024A0E
S3150800CBD042F82300704700BF00E100E00428044A39
S3150800CBE013680CBF43F0040323F004031360704773
S3150800CBF010E000E0704708B5FFF7FCFF08BD00002D
S3150800CC000268D3B2103B0849A1FB03131B09074965
S3150800CC10C95CC165032B22F47F7222F0030288BF28
S3150800CC2004328265806D7047ABAAAAAA38890208C1
S3150800CC3038B50446FFF7D0FC002C00F09480054672
S3150800CC40002384F83430022384F8353022681368C8
S3150800CC5023F00103136023681A6812F0010F0AD043
S3150800CC60FFF7BAFC401B0528F5D920236365032086
S3150800CC7084F8350038BD1A683C4810406168A268D7
S3150800CC800A43E1680A4321690A4361690A43A169BB
S3150800CC900A43E1690A43216A0A430243616A04298D
S3150800CCA016D01A6021684B6923F00703626A13439A
S3150800CCB0042A12D04B612046FFF7A2FFE26D3F23FC
S3150800CCC09340836000206065012384F8353038BDC1
S3150800CCD0E16A206B01430A43E3E7A26AA069D0B977
S3150800CCE0012A0CD032B1022A10D00020002834D1F3
S3150800CCF01343DFE794F82F0000F00100F6E7E06A37
S3150800CD00B0F1C07F14BF00200120EFE794F82F0090
S3150800CD1000F00100EAE7B0F5005F08D0022A1CD946
S3150800CD20032A18D194F82F0000F00100DEE7032A41
S3150800CD300FD8DFE802F01202120794F82F0000F06D
S3150800CD400100D3E7E06AB0F1C07F14BF00200120DC
S3150800CD50CCE70020CAE70020C8E740236365012026
S3150800CD6084F8350038BD012038BD00BF3F8010F07B
S3150800CD7070B490F83440012C42D0856D012480F8B7
S3150800CD80344090F83540E4B2012C05D0002380F8F1
S3150800CD903430022070BC7047022480F835400024E5
S3150800CDA044650668346824F4802434600468636043
S3150800CDB08368402B1FD0036899600368DA60C26DE8
S3150800CDC03F239340AB600268136843F01603136071
S3150800CDD00268536943F080035361036C23B1026808
S3150800CDE0136843F0080313600268136843F00103ED
S3150800CDF013600020CEE703689A600368D960DEE70F
S3150800CE000220C7E790F83530DBB2022B03D0802327
S3150800CE10436501207047052380F83530026813689A
S3150800CE2023F001031360002070470000F0B583B0BB
S3150800CE30044600230193724B1E68876D3D68C26DD8
S3150800CE40082393402B4210D003681A6812F0040F87
S3150800CE500BD01A6822F004021A60C26D08239340A8
S3150800CE60BB60436D43F001034365E26D654B934038
S3150800CE701D4209D02268526912F0800F04D0BB60A7
S3150800CE80636D43F002036365E26D5F4B93401D4299
S3150800CE9009D02268126812F0020F04D0BB60636DD5
S3150800CEA043F004036365E26D102393401D4224D0CA
S3150800CEB02268126812F0080F1FD0BB6023681A6830
S3150800CEC012F4802F0DD01B6813F4002F04D1236CA5
S3150800CED09BB12046984710E0A36C73B1204698474B
S3150800CEE00BE01A6812F4807F03D11A6822F0080250
S3150800CEF01A60236C0BB120469847E26D20239340B5
S3150800CF001D4255D02268126812F0100F50D0BB602F
S3150800CF1094F83530DBB2052B0ED023681A6812F464
S3150800CF20802F33D01B6813F4002F2AD1636C002B93
S3150800CF303ED0204698473BE02268136823F0160344
S3150800CF4013602268536923F080035361236CA3B1ED
S3150800CF502268136823F008031360E26D3F239340A9
S3150800CF60BB60002384F83430012384F83530236D00
S3150800CF70002B43D02046984740E0A36C002BE7D10E
S3150800CF80EBE7E36BA3B12046984711E01A6812F461
S3150800CF90807F09D11A6822F010021A60002384F8EB
S3150800CFA03430012384F83530E36B0BB120469847BB
S3150800CFB0636D1BB3636D13F0010F1BD0052384F853
S3150800CFC035302268136823F0010313600F4AA2FB69
S3150800CFD00632920A019B013301939A4204D32368CD
S3150800CFE01B6813F0010FF5D1002384F834300123B0
S3150800CFF084F83530E36C0BB12046984703B0F0BD92
S3150800D000000000200100800004008000B5814E1B4E
S3150800D0102DE9F04F83B00025664FDFF8A4E1664E90
S3150800D020DFF8A091DFF8A0A156E0EC0800EB840435
S3150800D030D4F820C005F007024FEA820B0F2202FA45
S3150800D0400BF22CEA020C0A6902FA0BF242EA0C020B
S3150800D05022624DE0846802EA040BCC6804FA0CF4F8
S3150800D06044EA0B048460446824EA030B4C68C4F35E
S3150800D0700013AB4043EA0B03436050E00022A24092
S3150800D08042EA0C029A6033686FEA08044A6812F4A6
S3150800D090803F0CBF234048EA0303336073684A683D
S3150800D0A012F4003F0CBF234048EA03037360B268DA
S3150800D0B04B6813F4801F0CBF224048EA0202B26094
S3150800D0C0F3684A6812F4001F0CBF234048EA0303BA
S3150800D0D0F3600135102D6AD00123AB400A6803EAD4
S3150800D0E002084345F5D14A6822F01002022A9CD06C
S3150800D0F004684FEA450C032202FA0CF2D24304EA0A
S3150800D100020B4C6804F0030404FA0CF444EA0B041A
S3150800D11004604C6824F01004013C012C9AD9C368B9
S3150800D1201A408B6803FA0CF31343C3604B6813F079
S3150800D130805FCED0002301937B6C43F480437B64ED
S3150800D1407B6C03F480430193019B25F0030303F1F1
S3150800D150804303F59C339A6805F00304A4004FF056
S3150800D1600F0C0CFA04FC22EA0C0C704586D04845D4
S3150800D17013D0504513D0114A904212D002F580625E
S3150800D180904210D002F5806290420ED002F580627D
S3150800D19090420CBF0622072271E701226FE702229E
S3150800D1A06DE703226BE7042269E7052267E703B008
S3150800D1B0BDE8F08F00380240003C0140000C0240F8
S3150800D1C00000024000040240000802402DE9F04F2A
S3150800D1D000234FF00108DFF818A1DFF81891DFF8EF
S3150800D1E018B108E04FF0000E0EFA04F4A44560D01A
S3150800D1F00133102B77D008FA03F202EA0105AA4296
S3150800D200F6D106685F000324BC40E4432640066066
S3150800D2104FEAD30E00EB8E0EDEF820C003F00706A9
S3150800D220B6000F2707FA06F62CEA0606CEF820609F
S3150800D230866826408660466826EA02024260C26818
S3150800D2401440C46023F0030202F1804202F59C32C6
S3150800D250966803F00304A400A74006EA070C5045A5
S3150800D260C0D0584517D0214EB04216D006F5806674
S3150800D270B04215D006F58066B04214D006F5806631
S3150800D280B04213D006F58066B0420CBF4FF0060ECA
S3150800D2904FF0070EA8E7C646A6E74FF0020EA3E72B
S3150800D2A04FF0030EA0E74FF0040E9DE74FF0050E72
S3150800D2B09AE7946824EA07079760D9F80020ED43AF
S3150800D2C02A40C9F80020D9F804202A40C9F80420C1
S3150800D2D0D9F808202A40C9F80820D9F80C201540A2
S3150800D2E0C9F80C5084E7BDE8F08F00BF000802407B
S3150800D2F000000240003C0140000402400369194254
S3150800D30014BF01200020704712B9090481617047D3
S3150800D310816170477047000008B5054B5B69034299
S3150800D32000D108BD024B5861FFF7F4FFF9E700BFCB
S3150800D330003C014003685A6912F4806F0DD06FF4FF
S3150800D34080625A610423036400230363202280F861
S3150800D3503D2080F83C3001207047002070472DE9B9
S3150800D360F041064690461D46C1F307478CB2012F89
S3150800D37033680CBF5B699B6934EA03030CBF01235E
S3150800D3800023434513D1B5F1FF3FF0D02DB1FFF788
S3150800D39023F9069BC01A8542E9D20023336320226B
S3150800D3A086F83D2086F83C300320BDE8F081002051
S3150800D3B0BDE8F0812DE9F041044617469846C1F3C9
S3150800D3C007468DB2012E23680CBF5B699B6935EA57
S3150800D3D0030314BF0123002363B323685A6912F4B5
S3150800D3E0806F13D1B7F1FF3FECD02FB1FFF7F4F8F8
S3150800D3F0A0EB08008742E5D200232363202284F8A5
S3150800D4003D2084F83C300320BDE8F0811A6842F4D8
S3150800D41000721A6023686FF480625A6104232364D9
S3150800D42000232363202284F83D2084F83C30012021
S3150800D430BDE8F0810020BDE8F08170B504460D46D0
S3150800D440164623685B6913F0800F19D12046FFF74B
S3150800D45071FFB8B9B5F1FF3FF3D025B1FFF7BCF8B6
S3150800D460801B8542EDD2236C43F0200323640023FE
S3150800D4702363202284F83D2084F83C30032070BDC5
S3150800D480002070BD012070BD2DE9F04184B005462D
S3150800D490884616461F460B9C0268136843F4807339
S3150800D4A0136000940A9B00224FF00111FFF757FF03
S3150800D4B020B10323184604B0BDE8F0812A6808F0B5
S3150800D4C0FE03136123460A9A22492846FFF772FF8C
S3150800D4D028B12B6C042B0CBF01230323EAE7002396
S3150800D4E003932B685A6903929B690393039B22460D
S3150800D4F00A992846FFF7A1FF034658B12B6C042B5F
S3150800D50001D00323D6E72A68136843F4007313602F
S3150800D5100123CFE7012F0ED02B68320A1A61224663
S3150800D5200A992846FFF789FF034678B12B6C042B26
S3150800D53005D00323BEE72A68F6B21661BAE72A6859
S3150800D540136843F4007313600123B3E72A68F6B23D
S3150800D5501661AFE7020001002DE9F04184B00546E7
S3150800D5600E46174698460B9C0268136843F4806378
S3150800D57013600268136843F48073136000940A9B6F
S3150800D58000224FF00111FFF7EAFE20B103231846E7
S3150800D59004B0BDE8F0812B68F6B206F0FE021A6107
S3150800D5A023460A9A3C492846FFF704FF28B12B6C04
S3150800D5B0042B0CBF01230323E9E7002303932B68FD
S3150800D5C05A6903929B690393039B22460A99284644
S3150800D5D0FFF733FF58B12B6C042B01D00323D6E792
S3150800D5E02A68136843F4007313600123CFE7B8F180
S3150800D5F0010F0DD02B683A0A1A6122460A99284665
S3150800D600FFF71BFFC8B12B6C042B0FD00323BEE713
S3150800D6102B68FFB21F6122460A992846FFF70DFFBD
S3150800D620B0B12B6C042B0CD00323B0E72A6813681F
S3150800D63043F4007313600123A9E72B68FFB21F6147
S3150800D640E9E72A68136843F40073136001239EE729
S3150800D6502A68136843F48073136000940A9B0022B7
S3150800D6604FF001112846FFF77AFE08B103238EE72B
S3150800D6702B6846F001061E6123460A9A0649284683
S3150800D680FFF798FE0346002881D02B6C042B0CBFAD
S3150800D690012303237BE700BF0200010070B504469F
S3150800D6A00D46164623685B6913F0040F19D1204608
S3150800D6B0FFF740FEB8B9B5F1FF3FF3D025B1FEF745
S3150800D6C08BFF801B8542EDD2236C43F02003236435
S3150800D6D000232363202284F83D2084F83C3003206D
S3150800D6E070BD002070BD012070BD70B505460C46A2
S3150800D6F016462B685A6912F0400F22D15A6912F061
S3150800D700100F11D124B1FEF767FF801B8442F0D2B7
S3150800D7102B6C43F020032B64202385F83D3000232F
S3150800D72085F83C30032070BD6FF010025A61002363
S3150800D7302B642B63202285F83D2085F83C30012098
S3150800D74070BD002070BD0000002872D038B50446B0
S3150800D75090F83D30002B41D0242384F83D302268D0
S3150800D760136823F00103136000F0B0FB324BA3FBF0
S3150800D77000239B0C22685360216865682F4A9542EE
S3150800D78031D801330B62226863682C498B4234D83E
S3150800D7905B00B0FBF3F0C0F30B03032B98BF042028
S3150800D7A0D0612268E369216A0B4313602268236902
S3150800D7B0E1680B43936022686369A1690B43D360F0
S3150800D7C02268136843F001031360002020642023B5
S3150800D7D084F83D30206384F83E0038BD80F83C303C
S3150800D7E018F034F9B8E74FF4967202FB03F3144ABB
S3150800D7F0A2FB03239B090133C4E7A16849B903EBDC
S3150800D8004303B0FBF3F0C0F30B0373B140F40040DD
S3150800D810C6E703EB830303EB8303B0FBF3F0C0F324
S3150800D8200B0323B140F44040BAE70120B8E70120D2
S3150800D830B6E70120704700BF83DE1B43A0860100C0
S3150800D840D34D62102DE9F04383B004460F46904647
S3150800D8509946BDF82C50FEF7BFFE94F83D30DBB272
S3150800D860202B18BF022303D0184603B0BDE8F08367
S3150800D870064600901923012243492046FFF76FFD0B
S3150800D88008B10223F0E794F83C30012B01D10223BA
S3150800D890EAE7012384F83C302268136823F400631E
S3150800D8A01360212384F83D30402384F83E3000235A
S3150800D8B02364A3F58033E36201960C9B00934B46E1
S3150800D8C0424639462046FFF7DFFD70B9002D2ED1B6
S3150800D8D032460C992046FFF7E1FE0346002844D05D
S3150800D8E0236C042B3AD00323BEE7236C042B4FF09A
S3150800D8F0000384F83C300CBF01230323B4E7236CF0
S3150800D900042B01D00323AFE72268136843F400739E
S3150800D91013600123A8E7002BDAD00A9B5B78136112
S3150800D920023DADB20A9B02330A93002DD0D032468F
S3150800D9300C992046FFF781FD0028E0D123680A9A52
S3150800D94012781A616B1E9BB22268516911F0040F96
S3150800D950E1D10A9A01320A921D46E6E7226813685F
S3150800D96043F40073136001237EE721680A6842F4D2
S3150800D97000720A60202284F83D20002284F83E20A6
S3150800D98084F83C2070E700BF020010002DE9F04340
S3150800D99087B004460D4690469946BDF83C60FEF7AA
S3150800D9A01BFE94F83D30DBB2202B18BF022503D0AE
S3150800D9B0284607B0BDE8F0830746009019230122E0
S3150800D9C082492046FFF7CBFC08B10225F0E794F818
S3150800D9D03C30012B01D10225EAE7012384F83C30CB
S3150800D9E02268136823F400631360222384F83D3009
S3150800D9F0402384F83E3000232364A3F58033E36292
S3150800DA000197109B00934B46424629462046FFF74E
S3150800DA10A3FD054648B1236C042B4FF0000384F898
S3150800DA203C300CBF01250325C2E766B900230293E3
S3150800DA3023685A6902929A690292029A1A6842F40B
S3150800DA4000721A6054E0012E0ED0022E29D000234F
S3150800DA50059323685A6905929B690593059BDFF828
S3150800DA6070914FF0000869E02268136823F4806318
S3150800DA7013600023039323685A6903929A690392F1
S3150800DA80039A1A6842F400721A603A4610992046B8
S3150800DA90FFF72BFE002834D123681B690E9A1370F2
S3150800DAA026E02268136823F48063136022681368EB
S3150800DAB043F4006313600023049323685A690492AD
S3150800DAC09B690493049B0097109B002240492046BB
S3150800DAD0FFF745FC002872D12268136843F40073E7
S3150800DAE0136023681B690E9A137023681B695370A9
S3150800DAF0202384F83D30002384F83E3084F83C30F7
S3150800DB0056E7236C202B0CBF0325012550E73A4620
S3150800DB1010992046FFF7E9FD002841D123681B69C3
S3150800DB200E9A137023685A6912F0040F3ED10E9BA1
S3150800DB3001330E93013EB6B2002ED9D0032EE6D895
S3150800DB40012EA2D0022EBED00097109B424649460F
S3150800DB502046FFF704FC002833D12268136823F413
S3150800DB608063136023681B690E9A13700097109BD5
S3150800DB70424649462046FFF7F2FB20BB2268136857
S3150800DB8043F40073136023681B690E9A5370236865
S3150800DB901B699370033EB6B2134603330E93CBE765
S3150800DBA0236C202B0CBF0325012501E71B690E9A60
S3150800DBB05370023EB6B2134602330E93BCE70325F2
S3150800DBC0F6E60325F4E60325F2E600BF0200100098
S3150800DBD00400010030B583B000230193234B1A6C6F
S3150800DBE042F080521A641B6C03F080530193019B28
S3150800DBF04FF4803393FAA3F3B3FA83F303F1845310
S3150800DC0003F560339B0001221A60FEF7E5FC054622
S3150800DC10174C636813F4803F08D1FEF7DDFC401B00
S3150800DC20B0F57A7FF5D9032003B030BD4FF4003341
S3150800DC3093FAA3F3B3FA83F303F1845303F560333A
S3150800DC409B0001221A60FEF7C7FC0546084C63686C
S3150800DC5013F4003F07D1FEF7BFFC401BB0F57A7FEF
S3150800DC60F5D90320E0E70020DEE700BF00380240D0
S3150800DC700070004070B588B00C46164608B30023FD
S3150800DC800293204D2A6B42F004022A632A6B02F0A3
S3150800DC9004020292029A4FF400720392022204923C
S3150800DCA0032206920593079303A91748FFF7B0F9CD
S3150800DCB0AB6844EAC60423F078431C43AC6008B05A
S3150800DCC070BD002301930F4D2A6B42F001022A63AF
S3150800DCD02A6B02F001020192019A4FF480720392B4
S3150800DCE002220492032206920593079303A9074882
S3150800DCF0FFF78EF9AA6822F0EC6232431443AC604F
S3150800DD00DDE700BF0038024000080240000002407C
S3150800DD10674B1B6803F00F038B4209D2CBB2644AE8
S3150800DD201370136803F00F03994201D0012070475E
S3150800DD302DE9F041036813F0020F06D05D4A936897
S3150800DD4023F0F0038468234393600D460446036872
S3150800DD5013F0010F6AD04268012A27D0931E012BBF
S3150800DD602CD9544B1B6813F0020F00F09E805149C2
S3150800DD708B6823F0030313438B60FEF72DFC0646DE
S3150800DD806368012B22D0022B30D0032B3ED0494F9B
S3150800DD9041F28838BB6813F00C0F47D0FEF71CFC1D
S3150800DDA0801B4045F6D90320BDE8F081414B1B682E
S3150800DDB013F4003FDBD10120BDE8F0813D4B1B6821
S3150800DDC013F0007FD3D10120BDE8F081394F41F22D
S3150800DDD08838BB6803F00C03042B27D0FEF7FCFB3E
S3150800DDE0801B4045F5D90320BDE8F081314F41F24B
S3150800DDF08838BB6803F00C03082B17D0FEF7ECFB3A
S3150800DE00801B4045F5D90320BDE8F081294F41F232
S3150800DE108838BB6803F00C030C2B07D0FEF7DCFB35
S3150800DE20801B4045F5D90320BDE8F081204B1B68CF
S3150800DE3003F00F039D420AD2EAB21D4B1A701B6803
S3150800DE4003F00F039D4202D00120BDE8F08123684C
S3150800DE5013F0040F06D0174A936823F4E053E168D9
S3150800DE600B439360236813F0080F07D0114A936891
S3150800DE70216923F4604343EAC103936000F030FD4F
S3150800DE800C4B9B68F02292FAA2F2B2FA82F203F0E5
S3150800DE90F003D340084AD35CD840084B18600020EA
S3150800DEA0FEF762FB0020BDE8F0810120BDE8F081A5
S3150800DEB0003C024000380240408902080000002069
S3150800DEC0014B1868704700BF00000020084B9B688C
S3150800DED04FF4E05292FAA2F2B2FA82F203F4E05355
S3150800DEE0D340044AD35C044A1068D840704700BF40
S3150800DEF0003802404089020800000020084B9B6851
S3150800DF004FF4604292FAA2F2B2FA82F203F4604344
S3150800DF10D340044AD35C044A1068D840704700BF0F
S3150800DF200038024040890208000000202DE9F0432D
S3150800DF3083B00446036813F0010F00F0AB80964ADD
S3150800DF40D2F88C3023F0C063816B0B43C2F88C3057
S3150800DF50856BB5FA85F56D09236813F0020F0CD0A9
S3150800DF608D4AD2F88C3023F0C053E16B0B43C2F8CC
S3150800DF708C30E36B002B08BF0125236813F0040FD0
S3150800DF8000F08A80844AD2F88C3023F44013216B3F
S3150800DF900B43C2F88C30266BB6F5801F08BF0125E7
S3150800DFA0B6FA86F67609236813F0080F0FD07A4A70
S3150800DFB0D2F88C3023F44003616B0B43C2F88C30E3
S3150800DFC0636BB3F5800F69D0002B08BF0126236861
S3150800DFD013F0200F64D1236813F0100F03D094F8C0
S3150800DFE058206E4B1A60236813F0800F08D06A4ACF
S3150800DFF0D2F8943023F44003E16C0B43C2F8943012
S3150800E000236813F0400F08D0634AD2F8943023F0FF
S3150800E0108063A16C0B43C2F89430236813F4807FA5
S3150800E0200DD05D4AD2F8943023F00063616D0B433E
S3150800E030C2F89430636DB3F1006F08BF01262368F8
S3150800E04013F4007F08D0544AD2F8943023F0805352
S3150800E050616C0B43C2F89430236813F4806F0CD0BC
S3150800E0604D4AD2F8943023F00053216D0B43C2F881
S3150800E0709430236DB3F1005F7BD0012D79D02368EE
S3150800E080B3F5006F75D0012E00F0C781002003B0EC
S3150800E090BDE8F08300255FE7002684E7012596E7BB
S3150800E0A0002301933C4B1A6C42F080521A641B6C95
S3150800E0B003F080530193019B394A136843F4807334
S3150800E0C01360FEF789FA8046354F3B6813F4807F64
S3150800E0D007D1FEF781FAA0EB08000228F5D903203C
S3150800E0E0D5E72D4B1B6F13F4407312D0226C02F444
S3150800E0F0407293420DD0284B1A6F22F44072294978
S3150800E10001200860002008601A671B6F13F0010FD2
S3150800E11012D1236C03F44072B2F5407F1ED01E4A1A
S3150800E120936823F4F81393601B4A116F236CC3F3A7
S3150800E1300B030B4313674EE7FEF74EFA8146164F5D
S3150800E14041F288383B6F13F0020FE2D1FEF744FA2A
S3150800E150A0EB09004045F5D9032098E70E498A68DF
S3150800E16022F4F81223F0704323F4407313438B60B0
S3150800E170DAE700220C4B1A60FEF72EFA0746064D20
S3150800E1802B6813F0006F11D0FEF726FAC01B022881
S3150800E190F6D903207BE700BF00380240E01147426A
S3150800E1A000700040400E474268004742236813F05B
S3150800E1B0010F01D0A26B2AB113F0020F43D0E36B13
S3150800E1C0002B40D1CB49D1F884304FF4403090FA37
S3150800E1D0A0FEBEFA8EFED1F884504FF0706C9CFA01
S3150800E1E0ACF8B8FA88F847F6C07292FAA2F2B2FA10
S3150800E1F082F790FAA0F0B0FA80F09CFAACFCBCFA70
S3150800E2008CFC4FF0E04999FAA9F9B9FA89F9A2689C
S3150800E210BA40676907FA09F73A4367683A4305F067
S3150800E220706525FA08F808FA0CFC42EA0C0203F4B1
S3150800E230403323FA0EF3013323F00043013B8340B6
S3150800E2401343C1F88430236813F0040F03D0226BFC
S3150800E250B2F5801F53D013F0080F03D0636BB3F5E4
S3150800E260800F4CD0236813F4806F04D0236DB3F16C
S3150800E270005F00F08F80236813F4006F2CD047F6F8
S3150800E280C07090FAA0F0B0FA80F04FF4403393FAD9
S3150800E290A3F3B3FA83F54FF0706191FAA1F1B1FADD
S3150800E2A081F14FF0E04292FAA2F2B2FA82F2E36802
S3150800E2B05B08013BAB40A56805FA00F003436068BC
S3150800E2C00343206900FA01F10B43616901FA02F27E
S3150800E2D01343884AC2F884300122874B1A60FEF736
S3150800E2E07BF90746834D2B6813F0006F7FF4CBAE9E
S3150800E2F0FEF772F9C01B0228F5D90320C7E67D4947
S3150800E300D1F884304FF4403090FAA0FEBEFA8EFE63
S3150800E310D1F884504FF0E04C9CFAACF8B8FA88F87B
S3150800E32047F6C07292FAA2F2B2FA82F790FAA0F011
S3150800E330B0FA80F04FF0706999FAA9F9B9FA89F933
S3150800E3409CFAACFCBCFA8CFCA268BA40276907FAAE
S3150800E35009F73A4367683A4305F0E04525FA08F8AD
S3150800E36008FA0CFC42EA0C0203F4403323FA0EF3D3
S3150800E370013323F00043013B83401343C1F8843043
S3150800E380D1F88C20A36A013B22F01F021343C1F87F
S3150800E3908C3067E7DFF85CE1DEF884204FF4403321
S3150800E3A093FAA3FCBCFA8CFCDEF884104FF0E0402C
S3150800E3B090FAA0F8B8FA88F847F6C07999FAA9F950
S3150800E3C0B9FA89F993FAA3F3B3FA83F74FF07065AC
S3150800E3D095FAA5F5B5FA85F590FAA0F0B0FA80F0A9
S3150800E3E0E3685B08013BBB40A76807FA09F73B43AC
S3150800E3F067683B4301F0E04121FA08F808FA00F0A3
S3150800E400034302F4403222FA0CF20132520002FAB5
S3150800E41005F52B43CEF884302DE70022374B1A60DA
S3150800E420FEF7DAF80646334D2B6813F0005F06D080
S3150800E430FEF7D2F8801B0228F6D9032027E62368C0
S3150800E44013F0040F01D0226B22B113F0080F37D056
S3150800E450636BABBB2749D1F888304FF4403090FA4C
S3150800E460A0F7B7FA87F747F6C07292FAA2F2B2FA9D
S3150800E47082F690FAA0F0B0FA80F04FF0706595FA3F
S3150800E480A5F5B5FA85F5E269B240666A06FA05F5B4
S3150800E4902A43A5692A4303F44033FB40013323F09A
S3150800E4A00043013B83401343C1F88830D1F88C30D0
S3150800E4B0E26A013A23F4F85343EA0223C1F88C309E
S3150800E4C0236813F4807F03D0636DB3F1006F17D010
S3150800E4D001220A4B1A60FEF77FF80546054C2368A9
S3150800E4E013F0005F37D1FEF777F8401B0228F6D9FC
S3150800E4F00320CCE5003802406800474270004742D6
S3150800E5001648D0F888204FF0706191FAA1F7B7FA4B
S3150800E51087F747F6C07595FAA5F5B5FA85F54FF468
S3150800E520403393FAA3F3B3FA83F691FAA1F1B1FA59
S3150800E53081F1236A5B08013BB340E66906FA05F5F3
S3150800E5402B43A469234302F07062FA408A401343BE
S3150800E550C0F88830BCE7002099E500BF00380240C3
S3150800E560F0B583B00446036813F0010F34D0AE4B00
S3150800E5709B6803F00C03042B25D0AB4B9B6803F078
S3150800E5800C03082B1AD0A84B9B6803F00C030C2B22
S3150800E5904CD02279A54B1A706368002B4CD0FEF735
S3150800E5A01BF80646A04D2B6813F4003F14D1FEF75E
S3150800E5B013F8801B6428F6D9032088E19A4B5B6818
S3150800E5C013F4800FDFD0984B1B6813F4003F03D079
S3150800E5D06368002B00F07881236813F0020F5CD083
S3150800E5E0914B9B6813F00C0F3AD08F4B9B6803F046
S3150800E5F00C03082B2FD08C4B9B6803F00C030C2BB9
S3150800E60038D0E368002B6ED00122894B1A60FDF7DB
S3150800E610E3FF0646844D2B6813F0020F55D1FDF72C
S3150800E620DBFF801B0228F6D9032050E17E4B5B688E
S3150800E63013F4800FADD0C6E7FDF7CEFF06467A4D38
S3150800E6402B6813F4003FC7D0FDF7C6FF801B64286C
S3150800E650F6D903203BE1744B5B6813F4800FCAD1EB
S3150800E660714B1B6813F0020F0AD0E368012B07D021
S3150800E67001202CE16C4B5B6813F4800FC1D1EFE7E6
S3150800E68069480168F82393FAA3F3B3FA83F2236976
S3150800E690934021F0F80213430360236813F0080F30
S3150800E6A045D063698BB30122624B1A60FDF794FF6C
S3150800E6B006465D4D6B6F13F0020F38D1FDF78CFFE0
S3150800E6C0801B0228F6D9032001E157480168F82380
S3150800E6D093FAA3F3B3FA83F22369934021F0F8027D
S3150800E6E013430360D9E70022514B1A60FDF774FF04
S3150800E6F006464D4D2B6813F0020FCED0FDF76CFF82
S3150800E700801B0228F6D90320E1E00022494B1A6053
S3150800E710FDF762FF0646444D6B6F13F0020F06D0F5
S3150800E720FDF75AFF801B0228F6D90320CFE023689D
S3150800E73013F0040F1FD1A369002B00F0C7803A4AD3
S3150800E740926802F00C02082A00F0C380022B59D006
S3150800E7500022394B1A60FDF73FFF0546324C236805
S3150800E76013F0007F00F0AE80FDF736FF401B02284D
S3150800E770F5D90320ABE0002301932B4B1A6C42F02A
S3150800E78080521A641B6C03F080530193019B2B4A39
S3150800E790136843F480731360FDF71EFF0646274D82
S3150800E7A02B6813F4807F06D1FDF716FF801B02281D
S3150800E7B0F6D903208BE0227A214B1A70A36883B11D
S3150800E7C0FDF70AFF0746184D41F288362B6F13F0FE
S3150800E7D0020FB0D1FDF700FFC01BB042F6D90320E7
S3150800E7E075E0FDF7F9FE07460F4D41F288362B6FA7
S3150800E7F013F0020F9FD0FDF7EFFEC01BB042F6D90B
S3150800E800032064E000220C4B1A60FDF7E5FE06467D
S3150800E810054D2B6813F0007F14D0FDF7DDFE801B35
S3150800E8200228F6D9032052E0003802400238024096
S3150800E83000004742800E4742600047420070004091
S3150800E8407038024047F6C07696FAA6F6B6FA86F605
S3150800E8504FF4403292FAA2F2B2FA82F54FF07060A3
S3150800E86090FAA0F0B0FA80F04FF0E04191FAA1F1E9
S3150800E870B1FA81F1E369226A1343626AB24013432B
S3150800E880A26A5208013AAA401343E26A8240134335
S3150800E890226B02FA01F10B430F4A536001220F4B18
S3150800E8A01A60FDF799FE05460B4C236813F0007FA6
S3150800E8B006D1FDF791FE401B0228F6D9032006E093
S3150800E8C0002004E0002002E0012000E0002003B060
S3150800E8D0F0BD0120FBE700BF003802406000474258
S3150800E8E0274B9B6803F00C03082B03D00C2B25D071
S3150800E8F024487047224B5A6802F03F025B68204B57
S3150800E9005B6847F6C07191FAA1F0B0FA80F00B4047
S3150800E910C3401C48B0FBF2F000FB03F0184B5B68E1
S3150800E9204FF4403292FAA2F2B2FA82F203F440337A
S3150800E930D34001335B00B0FBF3F07047104B5A68C5
S3150800E94002F03F025B680E4B5B6847F6C07191FAAE
S3150800E950A1F0B0FA80F00B40C3400A48B0FBF2F0D1
S3150800E96000FB03F0064B5B684FF0E04292FAA2F216
S3150800E970B2FA82F203F0E043D340B0FBF3F07047FB
S3150800E980003802400024F400F8B507460E4615463E
S3150800E9901C463A68936836EA03030CBF0123002332
S3150800E9A09D4238D0B4F1FF3FF4D02CB1FDF714FEE8
S3150800E9B0069BC01A8442ECD83A68536823F0E003F1
S3150800E9C053607B68B3F5827F0BD0BB6AB3F5005FF3
S3150800E9D014D0012387F85130002387F850300320DC
S3150800E9E0F8BDBB68B3F5004F02D0B3F5806FECD124
S3150800E9F03A68136823F040031360E6E73A68136839
S3150800EA0023F400531B041B0C13603A68136843F481
S3150800EA1000531360DDE70020F8BD10B582B0044648
S3150800EA2000920B4600228021FFF7AEFF034620B175
S3150800EA30636D43F0200363650323184602B010BDD7
S3150800EA4000283BD010B504460023836290F8513065
S3150800EA50002B2ED0022384F851302268136823F045
S3150800EA604003136022686368A1680B43E1680B439F
S3150800EA7021690B4361690B43E1690B43216A0B4327
S3150800EA80A16A0B43A16901F400710B431360226864
S3150800EA90638B03F00403616A0B4353602268D369EE
S3150800EAA023F40063D36100206065012384F85130A4
S3150800EAB010BD80F8503016F0F5FFCBE701207047FF
S3150800EAC02DE9F04184B01D4690F85030012B03D152
S3150800EAD0022004B0BDE8F08104460E4690460123A4
S3150800EAE080F85030FDF778FD074694F85130DBB2D0
S3150800EAF0012B07D00220012384F85130002384F823
S3150800EB005030E6E7002E00F09E80B8F1000F00F0C6
S3150800EB109C80032384F85130002363652663A4F898
S3150800EB203480A4F83680A363A387E38763642364E9
S3150800EB30A368B3F5004F1BD023681A6812F0400F7C
S3150800EB4003D11A6842F040021A60E368B3F5006F11
S3150800EB5014D063681BB1E38E9BB2012B41D12368A5
S3150800EB6016F8012B1A73E38E013B9BB2E38638E055
S3150800EB702268136843F480431360DDE763681BB1BA
S3150800EB80E38E9BB2012B12D1236836F8022BDA608A
S3150800EB90E38E013B9BB2E38609E0002D57D0B5F121
S3150800EBA0FF3F04D0FDF718FDC01B854251D9E38EFF
S3150800EBB09BB233B323689A6812F0020FEDD036F889
S3150800EBC0022BDA60E38E013B9BB2E386EFE7002D6A
S3150800EBD041D0B5F1FF3F04D0FDF7FEFCC01B8542CE
S3150800EBE03BD9E38E9BB263B123689A6812F0020F91
S3150800EBF0EDD016F8012B1A73E38E013B9BB2E38620
S3150800EC00EFE700972B46012202212046FFF7BCFEBC
S3150800EC1008B103206FE73A4629462046FFF7FDFE6E
S3150800EC2018B120236365012065E7A36833B9039308
S3150800EC302368DA6803929B680393039B606D003030
S3150800EC4018BF012057E7012055E7012053E70320A5
S3150800EC5051E703204FE703204DE703204BE72DE953
S3150800EC60F04F85B098460E9D90F85030012B04D190
S3150800EC700223184605B0BDE8F08F04460F4616462F
S3150800EC80012380F85030FDF7A7FC814694F85130EF
S3150800EC90DBB2012B13D06268B2F5827F07D002235C
S3150800ECA0012284F85120002284F85020E1E7A26866
S3150800ECB0002A40F0E480042B01D00223F0E7002F5D
S3150800ECC000F0DF80002E00F0DE80B8F1000F00F0C3
S3150800ECD0DC8094F85130DBB2012B04BF052384F89D
S3150800ECE0513000236365A663A4F83E80A4F83C80EF
S3150800ECF02763A4F83680A4F8348023646364236801
S3150800ED001A6812F0400F03D11A6842F040021A60DE
S3150800ED10E368B3F5006F13D063681BB1E38E9BB24B
S3150800ED20012B07D1236817F8012B1A73E38E013BD1
S3150800ED309BB2E3864FF001084FF0000BC24661E034
S3150800ED4063681BB1E38E9BB2012B07D1236837F8A2
S3150800ED50022BDA60E38E013B9BB2E3864FF0010893
S3150800ED604FF0000BC24618E0E38F9BB263B12368ED
S3150800ED709A6812F0010F07D0DB6826F8023BE38F8A
S3150800ED80013B9BB2E387D046B5F1FF3F05D0FDF7BF
S3150800ED9023FCA0EB0900854279D9E38E9BB21BB907
S3150800EDA0E38F9BB2002B48D0B8F1000FDCD0E38E7E
S3150800EDB09BB2002BD8D023689A6812F0020FD3D0E2
S3150800EDC037F8022BDA60E38E013B9BB2E386D8461E
S3150800EDD0CAE7E38F9BB263B123689A6812F0010F02
S3150800EDE007D0DB683370E38F013B9BB2E3870136BC
S3150800EDF0D046B5F1FF3F05D0FDF7EEFBA0EB0900C5
S3150800EE00854246D9E38E9BB213B9E38F9BB2A3B171
S3150800EE10B8F1000FDDD0E38E9BB2002BD9D0236862
S3150800EE209A6812F0020FD4D03A781A73E38E013B2F
S3150800EE309BB2E3860137D846CBE7CDF800902B4640
S3150800EE40012202212046FFF79FFD08B1032327E789
S3150800EE504A4629462046FFF7E0FD034618B1202317
S3150800EE60636501231CE7A268002A7FF419AF0392A1
S3150800EE702268D168039192680392039A10E70223E5
S3150800EE800EE701230CE701230AE7012308E703231A
S3150800EE9006E7032304E72DE9F04182B004460D4650
S3150800EEA090461E464368B3F5827F07D094F85030E3
S3150800EEB0012B0FD1022002B0BDE8F0818368002B38
S3150800EEC0F4D1042380F85130009613460A46FFF71A
S3150800EED0C6FEF0E7012384F85030FDF77DFB0746B0
S3150800EEE094F85130DBB2012B07D00220012384F8B5
S3150800EEF05130002384F85030DDE7002D71D0B8F189
S3150800EF00000F70D0042384F8513000236365A5638D
S3150800EF10A4F83C80A4F83E802363A386E386236492
S3150800EF206364A368B3F5004F0BD023681A6812F020
S3150800EF30400F03D11A6842F040021A60E36883B1B1
S3150800EF4029E02268136823F480431360EDE7002E56
S3150800EF504BD0B6F1FF3F04D0FDF73EFBC01B8642FF
S3150800EF6045D9E38F9BB233B323689A6812F0010F31
S3150800EF70EDD01B7B05F8013BE38F013B9BB2E38792
S3150800EF80EFE7002E35D0B6F1FF3F04D0FDF724FB9E
S3150800EF90C01B86422FD9E38F9BB263B123689A6858
S3150800EFA012F0010FEDD0DB6825F8023BE38F013B39
S3150800EFB09BB2E387EFE76368B3F5827F04D0606DA1
S3150800EFC0003018BF012091E7A368B3F5004F02D0BF
S3150800EFD0B3F5806FF3D12268136823F040031360FA
S3150800EFE0EDE7012082E7012080E703207EE7032082
S3150800EFF07CE703207AE7032078E77047022380F846
S3150800F00039300268136843F001031360012380F85E
S3150800F010393000207047704770477047704770470F
S3150800F02010B5044603681A6912F0020F11D0DA689F
S3150800F03012F0020F0DD06FF002021A610123037657
S3150800F04003689B6913F0030F70D0FFF7E6FF0023F0
S3150800F050237623681A6912F0040F12D0DA6812F0C0
S3150800F060040F0ED06FF004021A6102232376236878
S3150800F0709B6913F4407F5FD02046FFF7CEFF00233D
S3150800F080237623681A6912F0080F12D0DA6812F08C
S3150800F090080F0ED06FF008021A610423237623683E
S3150800F0A0DB6913F0030F4ED02046FFF7B6FF0023A7
S3150800F0B0237623681A6912F0100F12D0DA6812F054
S3150800F0C0100F0ED06FF010021A61082323762368FA
S3150800F0D0DB6913F4407F3DD02046FFF79EFF0023EF
S3150800F0E0237623681A6912F0010F03D0DA6812F042
S3150800F0F0010F36D123681A6912F0800F03D0DA6837
S3150800F10012F0800F34D123681A6912F0400F03D029
S3150800F110DA6812F0400F32D123681A6912F0200F0C
S3150800F12003D0DA6812F0200F30D110BDFFF774FF54
S3150800F1302046FFF773FF8AE72046FFF76DFF204654
S3150800F140FFF76CFF9BE72046FFF766FF2046FFF7B1
S3150800F15065FFACE72046FFF75FFF2046FFF75EFF37
S3150800F160BDE76FF001021A612046FFF754FFC1E7B9
S3150800F1706FF080021A61204600F094F8C3E76FF03A
S3150800F18040021A612046FFF74AFFC5E76FF02002E2
S3150800F1901A61204600F085F8C7E700000368314A7F
S3150800F1A090422FD0B0F1804F2CD0A2F57C429042ED
S3150800F1B028D002F58062904224D002F580629042FF
S3150800F1C020D002F5784290421CD0274A90422FD090
S3150800F1D002F5806290422BD002F58062904227D0D9
S3150800F1E0A2F59832904223D002F5806290421FD051
S3150800F1F002F5806290421BD003608B68C3620B687D
S3150800F200836221E023F070034A681343154A90424B
S3150800F2100ED0B0F1804F0BD0A2F57C42904207D0B9
S3150800F22002F58062904203D002F58062904213D1C3
S3150800F23023F44073CA68134303608B68C3620B6880
S3150800F2408362084B984202D0084B984201D10B6959
S3150800F250036301234361704702F578429042E7D081
S3150800F260B3E700BF00000140004001400004014030
S3150800F270A8B110B5044690F839305BB1022384F87A
S3150800F2803930211D2068FFF789FF012384F83930BA
S3150800F290002010BD80F83830FFF7AFFEEEE70120FA
S3150800F2A07047704770470268D36823F49073D36039
S3150800F2B00268536923F001035361202380F83A302A
S3150800F2C0704700002DE9F04704460268136923F4E5
S3150800F2D04053C1680B4313610168CA6822F4164299
S3150800F2E022F00C0283680069034360690343E069FE
S3150800F2F003431343CB602268536923F44073A1691F
S3150800F3000B435361E369B3F5004F5FD02568B64BED
S3150800F3109D4200F0128103F580639D4200F00D8145
S3150800F320FEF7D4FD00EB800000EB800063689B00CD
S3150800F330B0FBF3F3DFF8B482A8FB03235B091E01D5
S3150800F340FEF7C4FD00EB800000EB800063689B00BD
S3150800F350B0FBF3F7FEF7BAFD00EB800000EB800088
S3150800F36063689B00B0FBF3F3A8FB03235B094FF02C
S3150800F370640A0AFB13731B013233A8FB03235B09D8
S3150800F38003F0F007FEF7A2FD00EB800000EB80001B
S3150800F39063689B00B0FBF3F9FEF798FD00EB80006D
S3150800F3A000EB800063689B00B0FBF3F3A8FB032324
S3150800F3B05B090AFB13931B013233A8FB0323C3F330
S3150800F3C043133B433344AB60BDE8F087256803F13C
S3150800F3D0804303F510439D4259D003F580639D424F
S3150800F3E055D0FEF773FD00EB800000EB80006368E4
S3150800F3F05B00B0FBF3F3DFF8F481A8FB03235B099A
S3150800F4001F01FEF763FD00EB800000EB80006368D8
S3150800F4105B00B0FBF3F6FEF759FD00EB800000EB4E
S3150800F420800063685B00B0FBF3F3A8FB03235B096A
S3150800F4304FF0640A0AFB1363DB003233A8FB03238D
S3150800F4401B0903F4F876FEF741FD00EB800000EB9C
S3150800F450800063685B00B0FBF3F9FEF737FD00EB4D
S3150800F460800000EB800063685B00B0FBF3F3A8FB49
S3150800F47003235B090AFB1393DB003233A8FB032340
S3150800F480C3F342133B443344AB60BDE8F087FEF751
S3150800F49035FD00EB800000EB800063685B00B0FB85
S3150800F4A0F3F3DFF84881A8FB03235B091F01FEF786
S3150800F4B025FD00EB800000EB800063685B00B0FB75
S3150800F4C0F3F6FEF71BFD00EB800000EB8000636897
S3150800F4D05B00B0FBF3F3A8FB03235B094FF0640A58
S3150800F4E00AFB1363DB003233A8FB03231B0903F46F
S3150800F4F0F876FEF703FD00EB800000EB80006368FA
S3150800F5005B00B0FBF3F9FEF7F9FC00EB800000EBBB
S3150800F510800063685B00B0FBF3F3A8FB03235B0979
S3150800F5200AFB1393DB003233A8FB0323C3F342130E
S3150800F5303B443344AB60BDE8F087FEF7DFFC00EBE5
S3150800F540800000EB800063689B00B0FBF3F3DFF8F4
S3150800F5509C80A8FB03235B091E01FEF7CFFC00EB8A
S3150800F560800000EB800063689B00B0FBF3F7FEF7B2
S3150800F570C5FC00EB800000EB800063689B00B0FBD5
S3150800F580F3F3A8FB03235B094FF0640A0AFB137322
S3150800F5901B013233A8FB03235B0903F0F007FEF7D0
S3150800F5A0ADFC00EB800000EB800063689B00B0FBBD
S3150800F5B0F3F9FEF7A3FC00EB800000EB800063681C
S3150800F5C09B00B0FBF3F3A8FB03235B090AFB139329
S3150800F5D01B013233A8FB0323C3F343133B433344D2
S3150800F5E0AB60BDE8F08700BF001001401F85EB51F6
S3150800F5F02DE9F04107460E4615469846069C3A6898
S3150800F600136836EA03030CBF01230023AB421ED15D
S3150800F610B4F1FF3FF4D02CB1FCF7DEFFA0EB0800F5
S3150800F6208442ECD23A68D36823F4D073D3603A683C
S3150800F630536923F001035361202387F8393087F88B
S3150800F6403A30002387F838300320BDE8F0810020DF
S3150800F650BDE8F08158B310B5044690F839300BB3BD
S3150800F660242384F839302268D36823F40053D360FE
S3150800F6702046FFF727FE2268136923F49043136197
S3150800F6802268536923F02A0353612268D36843F436
S3150800F6900053D3600020E063202384F8393084F8CF
S3150800F6A03A3010BD80F8383016F080FAD8E70120D5
S3150800F6B070472DE9F04782B01F4690F83930DBB223
S3150800F6C0202B04D00223184602B0BDE8F087044672
S3150800F6D00E461546002952D0002A52D090F83830E6
S3150800F6E0012B01D10223EEE7012380F838300023ED
S3150800F6F0C363212380F83930FCF76EFF8046A58462
S3150800F7004FF0000A4FF0800912E000974346524630
S3150800F71049462046FFF76CFF002834D12268338813
S3150800F720C3F3080353602369ABB90236E58CA5B168
S3150800F730013DE584A368B3F5805FE6D000974346AC
S3150800F740524649462046FFF753FFF0B923683278F8
S3150800F7505A600136EAE70136E8E700974346002291
S3150800F76040212046FFF744FF034608B10323AAE7D2
S3150800F770202284F83920002284F83820A3E70123C0
S3150800F780A1E701239FE703239DE703239BE72DE9D1
S3150800F790F04782B01F4690F83A30DBB2202B03D0F0
S3150800F7A0022002B0BDE8F08704460E461546002939
S3150800F7B055D0002A55D090F83830012B01D10220B7
S3150800F7C0EFE7012380F838300023C363222380F84B
S3150800F7D03A30FCF701FF8246A5854FF000094FF045
S3150800F7E020081FE0009753464A4641462046FFF741
S3150800F7F0FFFE002837D1236933B923685B68C3F352
S3150800F800080326F8023B0BE023685B68DBB226F8A0
S3150800F810013B05E023685B6803F07F03337001361C
S3150800F820E58DADB1013DE585A368B3F5805FD9D017
S3150800F830009753464A4641462046FFF7D9FEA0B9E7
S3150800F8402369002BE6D123685B6833700136E7E746
S3150800F850202384F83A30002084F83800A1E70120F4
S3150800F8609FE701209DE703209BE7032099E7000017
S3150800F87038B590F83940E4B2202C01D0022038BDC2
S3150800F880002931D0002A31D090F83830012B01D127
S3150800F890022038BD13460446012280F8382001624A
S3150800F8A08384C3840025C563212280F83920026B2E
S3150800F8B00F48D063226B0F481064226B0E48D06441
S3150800F8C0226B156522680432206BFDF751FA23680E
S3150800F8D06FF040021A6084F838502268536943F082
S3150800F8E080035361284638BD012038BD012038BD44
S3150800F8F095F90008CDF90008B5FA000838B590F86A
S3150800F9003A40E4B2202C01D0022038BD002937D075
S3150800F910002A37D090F83830012B01D1022038BDA3
S3150800F92013460A460546012180F838108262838507
S3150800F9300024C463222180F83A10416B1248C86338
S3150800F940696B12480864696B1148C864696B0C6571
S3150800F95029680431686BFDF70BFA2A68D36843F403
S3150800F9608073D3602A68536943F0010353612A6898
S3150800F970536943F04003536185F83840204638BD43
S3150800F980012038BD012038BDD7F90008A9FA0008BA
S3150800F990B5FA000808B5836B0268126812F4807F0E
S3150800F9A00FD10022DA8419684A6922F080024A6176
S3150800F9B01968CA6842F04002CA60202283F83920D2
S3150800F9C008BD18460FF05EFB08BD704708B5806B8A
S3150800F9D0FFF7FBFF08BD08B5836B0268126812F4CF
S3150800F9E0807F13D10022DA851968CA6822F48072EA
S3150800F9F0CA6019684A6922F001024A6119684A69A7
S3150800FA0022F040024A61202283F83A20184614F070
S3150800FA10A9F808BD08B590F83A30DBB2222B01D018
S3150800FA20022008BD8368B3F5805F0ED0036903BB67
S3150800FA30836A5A1C8262026852681A70C38D013B37
S3150800FA409BB2C385F3B1002008BD826A036943B936
S3150800FA5003685B68C3F308031380836A023383620F
S3150800FA60ECE703685B68DBB21380836A0133836261
S3150800FA70E4E7826A531C836203685B6803F07F03CA
S3150800FA801370DBE70268D36823F49073D3600268C7
S3150800FA90536923F001035361202380F83A3014F0A8
S3150800FAA061F8002008BD704708B5806BFFF7FBFFBB
S3150800FAB008BD704710B5846B2268516994F83930CF
S3150800FAC0DBB2212B0ED023685A6994F83A30DBB2A0
S3150800FAD0222B14D0E36B43F01003E3632046FFF7B1
S3150800FAE0E8FF10BD11F0800FEDD00023E384D36842
S3150800FAF023F0C003D360202384F83930E3E712F0FB
S3150800FB00400FE7D00023E3852046FFF7CCFBE1E76B
S3150800FB1010B5044602681368D068516913F00F0FD0
S3150800FB2017D113F0200F02D010F0200F0DD113F0CB
S3150800FB30800F02D010F0800F79D113F0400F03D058
S3150800FB4010F0400F40F0A28010BD2046FFF762FF7C
S3150800FB5010BD11F0010102D110F4907FE7D013F027
S3150800FB60010F06D010F4807F03D0E26B42F0010249
S3150800FB70E26313F0040F0DD0002900F09280E26BC7
S3150800FB8042F00202E26313F0020F08D113F0080FE5
S3150800FB900CD10FE013F0020F00F0868051B1E26B32
S3150800FBA042F00402E26313F0080F03D0E26B42F05E
S3150800FBB00802E263E26B002AC6D013F0200F02D0D7
S3150800FBC010F0200F21D123685A69E36B13F0080F50
S3150800FBD002D112F0400F24D02046FFF764FB2368B9
S3150800FBE05A6912F0400F18D05A6922F040025A6139
S3150800FBF0636B73B12F4A1A65606BFDF703F900282A
S3150800FC00A2D0606B036D984710BD2046FFF702FF30
S3150800FC10D9E72046FFF74DFF10BD2046FFF749FFFD
S3150800FC2010BD2046FFF745FF0023E36310BD94F897
S3150800FC303930DBB2212B87D1A368B3F5805F16D0A4
S3150800FC40236A591C21621B785360E38C013B9BB2E3
S3150800FC50E384002B7FF478AF2268D36823F080030F
S3150800FC60D3602268D36843F04003D36010BD236A8B
S3150800FC701B88C3F30803536023691BB9236A02333D
S3150800FC802362E2E7236A01332362DEE7D36823F0BF
S3150800FC904003D360202384F8393020460FF0F2F968
S3150800FCA010BD13F0020F85D113F0080F82D000297A
S3150800FCB080D07BE7B9FC000808B5806B0023C385B4
S3150800FCC0C384FFF7F6FE08BD0E49D1F8883043F421
S3150800FCD07003C1F888300C4B1A6842F001021A60AA
S3150800FCE0002098601A6822F0847222F480321A6022
S3150800FCF0064A5A601A6822F480221A60D860044BB1
S3150800FD008B60704700ED00E0003802401030002498
S3150800FD100080000810B582B002AB03F8011D026826
S3150800FD20546801221946A04702B010BD4FF0FF30B3
S3150800FD3070474FF0FF307047704710B514464FF0C4
S3150800FD40FF3392B20069FFF7B4FC204610BD00B538
S3150800FD5083B04FF0FF3301220DF107010069FFF769
S3150800FD6016FD9DF8070003B05DF804FBFEE70120C9
S3150800FD70704700001622024B1A604FF0FF3070479A
S3150800FD8098D3002010B51446012807D002280DD0B4
S3150800FD9009220A4B1A604FF0FF3010BD4FF0FF33AF
S3150800FDA092B20748FFF785FC204610BD4FF0FF3397
S3150800FDB092B20348FFF77DFC204610BD98D3002079
S3150800FDC0D4CF002008B503460A4A1068EFF3088224
S3150800FDD00344934202D8074A136008BD192206490C
S3150800FDE00220FFF7CFFF0C22044B1A604FF0FF30BA
S3150800FDF008BD00BF04000020A402030898D3002011
S3150800FE0010B50446FEF75CF8054BA3FB0030000D61
S3150800FE1004FB00F00A380138B0F1FF3FFBD110BDF2
S3150800FE2083DE1B4308B5FCF7DDFB08BD08B50120DA
S3150800FE30FFF7E6FF08BD08B50A20FFF7E1FF08BD92
S3150800FE4010B582B018468DF807200139062919D849
S3150800FE50DFE801F0041B2A3B4C5656002D4C0022C5
S3150800FE6010212046FDF750FA0120FCF7BBFB0122C2
S3150800FE7010212046FDF748FA01224FF40041264892
S3150800FE80FDF742FA012002B010BD9DF807302BB9E4
S3150800FE90002220211F48FDF737FAF3E70122202127
S3150800FEA01C48FDF731FAEDE79DF8073033B9012212
S3150800FEB04FF400411848FDF727FAE3E700224FF40C
S3150800FEC000411548FDF720FADCE79DF807303BB9F5
S3150800FED0002210210F48FDF717FAFFF7ACFFD1E70C
S3150800FEE0012210210B48FDF70FFAF6E74FF47A7353
S3150800FEF001220DF1070109480068FEF7E1FDC1E797
S3150800FF004FF47A739DF80720014604480068FEF707
S3150800FF10D7FDB7E70004024000000240480A002067
S3150800FF2008B5084B186001224FF400410648FDF752
S3150800FF30EBF90A20FCF756FB044A0549054800F088
S3150800FF40D3FC08BD480A00200000024041FE000814
S3150800FF500C00002050D300202DE9F04F89B0074649
S3150800FF600D46039116469B46BDF84840DDF84CA061
S3150800FF70009400F05CF8002856D0002C54D00BF101
S3150800FF800703C3F3CC0304933444A3B20593ABF13C
S3150800FF9008039BB2DA080132069223F007032A46C1
S3150800FFA00F321344079318E05B46554632E0013595
S3150800FFB0ADB24FEA5808AC4208D018F0010FF6D097
S3150800FFC032462946384600F0DCFCF0E7049B9A44A2
S3150800FFD00136B6B2059B9E4226D0039BDC1DA4B211
S3150800FFE0BBF1070FE0D9069B0AEB030955464FF00C
S3150800FFF0020815F8013B0093434632462146384627
S3150801000000F0C6FC0834A4B24D45F2D10BF0070343
S31508010010BDF81C40002BD9D095F80080E51FADB27C
S315080100201C44073CA4B2C8E709B0BDE8F08F70B418
S31508010030BDF80C40013C1444A4B2C58FB0F8426027
S31508010040964215D3AC4204D2A24294BF00220122A1
S31508010050FAB1013B0B449BB2828FB0F8400088424B
S315080100600DD3934217D2994294BF002001200EE086
S31508010070AC420BD3A24294BF00220122E8E7934285
S315080100800BD3994294BF0020012000E0002070BCE8
S3150801009070470020FBE70120F9E70020F7E710B5D4
S315080100A08C6800230121A04710BD10B58C68002378
S315080100B00321A04710BD10B58C6800231A460421F8
S315080100C0A04710BD10B58C68002301220421A04762
S315080100D010BD10B58C6800230221A04710BD10B5CC
S315080100E08C6800230521A04710BD2DE9F84F074666
S315080100F08B46551E0026B0464FF0FF0A4FF0010900
S3150801010041E0FF2C11D0FE2C4BD0EF2C4CD8DF2C24
S3150801011014D8CF2C1AD8BF2C20D814F0800F45D16B
S315080101202046FFF77FFE46462DE052465946384699
S31508010130FFF7D5FF0646A0B3464624E004F00F02B2
S3150801014059463846FFF7C5FF46461CE004F00F023C
S3150801015059463846FFF7A9FF464614E05946384638
S31508010160FFF7A9FF2401023404F0FE042046FFF735
S3150801017059FE59463846FFF7A5FF2046FFF752FEB6
S31508010180464600E04E4615F8014F002EB9D1FF2C20
S31508010190F8D0224659463846FFF7A1FF0028F2D182
S315080101A006463046BDE8F88F4646ECE74646EAE796
S315080101B02DE9F04103F1FF3E013A53FA82FC00248E
S315080101C00F4B104A1EF8015F661C03EB040805F085
S315080101D00F0717443F7D88F808700234E4B253FAD2
S315080101E086F602EB15152D7D3572E645EAD18C6842
S315080101F0054B80220621A0470120BDE8F08100BFFA
S315080102004C0A002070890208540A00200120704710
S31508010210F8B506460D464B681F7A1C8807FB042469
S3150801022004F0FF040E4AFFF760FF224629463046CE
S31508010230FFF755FF621CD2B229463046FFF74FFF3A
S31508010240002229463046FFF744FF5C2229463046FC
S31508010250FFF745FF012229463046FFF73AFFF8BD69
S31508010260948902082DE9F04F83B006460D4690465B
S315080102709B46A2F10A030B2B0FD8DFE803F0060E03
S315080102800E0E0E4162670E0E0E170222FFF707FFCA
S31508010290314A29463046FFF728FF5B46424629463A
S315080102A0304600F06DFD03B0BDE8F08FD1F804903B
S315080102B0D9F80C70B9F80AA04FEA9A0AB9F80030C9
S315080102C0002BEAD000245FFA8AF3019322462946D5
S315080102D03046FFF79DFF3B46019A29463046FFF710
S315080102E067FFFFF7A3FD002229463046FFF7DDFE2B
S315080102F057440134E4B2B9F80030A342E6D8CCE752
S315080103000122FFF7D2FE002229463046FFF7E1FE19
S31508010310C12229463046FFF7E2FE01222946304628
S31508010320FFF7D7FE9BF80020520829463046FFF70B
S31508010330D6FEFFF77BFD002229463046FFF7B5FEBC
S31508010340ABE7064AFFF7D1FE0120ACE7044AFFF7FF
S31508010350CCFE0120A7E700BFA4890208248A020867
S31508010360308A02082DE9F04F83B006460D469046BD
S315080103709B46A2F10A030B2B0FD8DFE803F0060E02
S315080103800E0E0E3F5E630E0E0E170222FFF787FE54
S315080103902F4A29463046FFF7A8FE5B4642462946BC
S315080103A0304600F025FC03B0BDE8F08FD1F8049083
S315080103B0D9F80C70B9F80AA04FEA9A0AB9F80030C8
S315080103C0002BEAD000245FFA8AF3019322462946D4
S315080103D03046FFF71DFF3B46019A29463046FFF78F
S315080103E0E7FE002229463046FFF75FFE57440134EF
S315080103F0E4B2B9F80030A342E8D8CEE70122FFF704
S3150801040054FE002229463046FFF763FEC1222946DB
S315080104103046FFF764FE012229463046FFF759FEAA
S315080104209BF80020520829463046FFF758FE00225D
S3150801043029463046FFF739FEAFE7064AFFF755FE6C
S315080104400120B0E7044AFFF750FE0120ABE700BFE1
S31508010450A4890208248A0208308A02084218435CE1
S31508010460507800EB032080B270470078704708B5D2
S31508010470FFF7FBFF18B1022801D0032008BD0620AB
S3150801048008BD0020704790F92900013080B27047F5
S3150801049008B50621FFF7E2FF08BD08B50821FFF7F1
S315080104A0DDFF08BD807A7047C07A70472DE9F84F9D
S315080104B080460E46D0F808B05846FFF7D6FF824662
S315080104C05846FFF7D4FF8146BAF1010F14BFFF273B
S315080104D00F275846FFF7E6FF04465846FFF7E4FF9D
S315080104E005465846FFF7D9FF602E03D910B158447F
S315080104F061240AE05846FFF7CBFF402E03D910B115
S315080105005844412401E00BF11100B5420ED3AC4227
S315080105101ED9002088F81C0088F81F0088F82000DA
S3150801052088F81D0088F81E00BDE8F88F002088F8B5
S315080105301C0088F81F0088F8200088F81D0088F834
S315080105401E00BDE8F88F0130AC42E2D00134E4B2B6
S315080105500378FF2BF7D0B44204D083783B404B4451
S315080105601844F1E7BAF1000F18D0BAF1020F15D005
S3150801057003F00F02023A88F81E201B0988F81D307D
S31508010580437803F00F0288F820201B0988F81F30EA
S3150801059083781B0988F81C30BDE8F88F88F81F3066
S315080105A0437888F82030C37888F81C30037988F8AE
S315080105B01D30437988F81E30BDE8F88F2DE9F04FD4
S315080105C085B007468A4616461946FFF76FFF002883
S315080105D053D00546B868FFF74AFF804697F81F903B
S315080105E097F8204097F91D309A441FFA8AF319465D
S315080105F00393A2B297F91E301344F61AB6B20092C3
S315080106004B4632463846FFF712FDA0B109F10709F4
S31508010610C9F3C40302935CB304F1FF3A5FFA8AFA99
S315080106200AF1010AB2441FFA8AFA4544013BDBB2D0
S3150801063003F1010B13E097F91C001BE015F8013BC8
S315080106400093434632462146384600F0A1F908345C
S31508010650A4B2A945F2D10136B6B2B24508D0029B79
S31508010660002BF8D005EB0B09039C4FF00008E5E7D2
S3150801067097F91C0005B0BDE8F08F0020FAE72DE9CF
S31508010680F04180460C4617461E46436A984707447A
S31508010690337893B1BFB200253A4621464046FFF763
S315080106A08DFF80B20444A4B20544ADB216F8013FE9
S315080106B0002BF1D12846BDE8F0810025FAE78368C9
S315080106C0CBB190F82820BAB95A7980F829201B7B32
S315080106D080F82A3090F9293090F92A209B1A9BB282
S315080106E090F82B20402A04D0DBB202FB03F3C3F3B4
S315080106F08F1380F82C307047012A06D05A7B80F870
S3150801070029209B7B80F82A30E4E7DA7B80F82920C8
S315080107101B7C80F82A30DDE708B5002280F82820FE
S31508010720FFF7CDFF08BD08B5012380F82830FFF78C
S31508010730C6FF08BD014B4362704700BF8304010829
S31508010740014B4362704700BF8704010870B50D4627
S31508010750097871B1064600243046FFF7A7FE96F9D7
S315080107601C301C44A4B215F8011F0029F4D12046F7
S3150801077070BD0024FBE7000083688B4207D010B5E3
S3150801078004468160FFF79BFF014B636210BD70470A
S315080107908304010810B50C68A04710BD38B5044696
S315080107A00D46836B0220984700230A2229462046D4
S315080107B0FFF7F0FF0546A36B03209847A36B0020BC
S315080107C09847284638BD38B504460D46836B02203E
S315080107D09847A36B012098470023142229462046EF
S315080107E0FFF7D8FF04F13C03172229462046FFF7F5
S315080107F0D1FFA36B0020984738BD70B504460D4656
S31508010800836B02209847A36B012098470023152282
S3150801081029462046FFF7BEFF064620B9A36B0020EE
S315080108209847304670BD04F13C03172229462046F5
S31508010830FFF7B0FFF2E700B583B002AB03F8012D6D
S315080108400F22FFF7A7FF03B05DF804FB10B5C285B9
S31508010850038600F12E033222FFF79CFF10BD00B577
S3150801086083B00DF106034622FFF794FFBDF8060093
S3150801087003B05DF804FB00B583B00DF1060347220A
S31508010880FFF788FFBDF8060003B05DF804FB08B55D
S3150801089000234822FFF77EFF08BD10B504464168CC
S315080108A0FFF7DDFF208061682046FFF7E4FF6080DF
S315080108B061682046FFF7EBFFE07404F13C03172259
S315080108C061682046FFF766FF10BD10B5044641680A
S315080108D0FFF764FF034608B9184610BD2046FFF71F
S315080108E0DCFF0123F8E700002DE9F04104460F4635
S315080108F0904600258560C560457401260674222345
S315080109008374856180F83460FFF714FF84F82860E2
S3150801091084F8295084F82A50402384F82B3084F827
S315080109202C50054BA3636760C7F808802046FFF77C
S31508010930CCFFBDE8F08100BF6D11010808B541681B
S31508010940FFF741FF08BD10B50446836903B198470F
S3150801095061682046FFF751FF10BD08B50A46416890
S31508010960FFF769FF08BD08B5002310224168FFF7A4
S3150801097011FF08BD08B5002311224168FFF70AFFD8
S3150801098008BD08B513460A464168FFF75FFF08BD6B
S3150801099038B54568C185028680F833309DF8103030
S315080109A080F8323000F12E033B222946FFF7F2FE8A
S315080109B038BD80F834107047C37C282B04D0022B2D
S315080109C00CBF032001207047FF207047C37C302BE2
S315080109D006D010B50446FFF7EFFF84F8340010BDC2
S315080109E0FF2380F8343080F8353070470022828042
S315080109F00388013BC38002727047028883881344C7
S31508010A009BB2838041888B420DD2037A01330372EC
S31508010A10C3881A4492B291429CBF01F1FF3292B245
S31508010A20C2800120704700207047C36842891A4472
S31508010A30002103F8011B9A42FBD1704710B4C38801
S31508010A408B4234BF00230123914294BF0021012127
S31508010A50848843EA010094428CBF002000F001001B
S31508010A600B4018435DF8044B704700230B808388BD
S31508010A704B804389013B8B80C388CB80704708B57F
S31508010A804B884A79012A03D0032A08D01A4602E07C
S31508010A9003F1080292B21946FFF7D0FF08BDA3F188
S31508010AA008011A468BB2F6E770B49DF80C60C46863
S31508010AB04589AD088088121AD2B212FB05F2880858
S31508010AC010FA82F2490001F0060136B9032088407E
S31508010AD0C0B2A55C25EA0000A05403F0030303FA9B
S31508010AE001F1A35C1943A15470BC7047C3684289DC
S31508010AF003EB4202002103F8011B9A42FBD170471E
S31508010B0030B583B04C888388A34206D8C388A342EC
S31508010B1003D30D884389AB4201D803B030BD8B7925
S31508010B20009222462946FFF7BFFFF6E7F8B50746C2
S31508010B300D460C7900260CE0324629463846FFF761
S31508010B40DFFF09E02B8801332B80640014F0FF04D2
S31508010B501CD014F0800FEFD16B79032BF5D801A2C5
S31508010B6052F823F0450B0108750B01087D0B0108A6
S31508010B70850B01086B8801336B80E6E72B88013BFF
S31508010B802B80E2E76B88013B6B80DEE7F8BD00BF8F
S31508010B90F8B507460D460C79012606E02B88013380
S31508010BA02B80A40014F0FF0420D0A309AB713246B0
S31508010BB029463846FFF7A4FF6B79032BF1D801A222
S31508010BC052F823F09D0B0108D50B0108DD0B01082E
S31508010BD0E50B01086B8801336B80E2E72B88013B43
S31508010BE02B80DEE76B88013B6B80DAE7F8BD00BF37
S31508010BF038B51D464C68143A342A1CD8DFE802F089
S31508010C003E461B501B1B1B1B1B1B1B1B1B1B1B1BA2
S31508010C101B1B1B1B1B1B1B1B37311B1B1B1B2A1BD4
S31508010C201B1B1B1B1B1B1B1D1B1B1B1B1B1B1B1B03
S31508010C301B1B565A5E00012341E029462046FFF751
S31508010C401EFF08B901233AE029462046FFF76EFF41
S31508010C50012334E0002229462046FFF751FF0123EC
S31508010C602DE029462046FFF793FF012327E00122BD
S31508010C7029462046FFF744FF012320E02046FFF7D7
S31508010C80B5FE2046FFF732FF012318E02046FFF79D
S31508010C90B4FE034698B12046FFF728FF01230EE06C
S31508010CA029462046FFF7E1FE012308E063892B80E8
S31508010CB0012304E063882B80012300E00223184600
S31508010CC038BD30B4C4684589AD088088121AD2B2D5
S31508010CD012FB05F2880810FA82F2490001F00601B2
S31508010CE003208840C0B203F003038B40A15C21EACC
S31508010CF000011943A15430BC70474A88838893423E
S31508010D000DD8C38893420AD310B50C884389A342E8
S31508010D1000D810BD8B792146FFF7D3FFF9E7704755
S31508010D2070B506460D460C790BE029463046FFF7A5
S31508010D30E4FF09E02B8801332B80640014F0FF04DB
S31508010D401CD014F0800FF0D16B79032BF5D801A2D2
S31508010D5052F823F0350D0108650D01086D0D0108DE
S31508010D60750D01086B8801336B80E6E72B88013B1B
S31508010D702B80E2E76B88013B6B80DEE770BD00BF25
S31508010D8038B51D464C68143A342A1CD8DFE802F0F7
S31508010D9030381B421B1B1B1B1B1B1B1B1B1B1B1B3B
S31508010DA01B1B1B1B1B1B1B1B1B1B1B1B1B1B2A1B75
S31508010DB01B1B1B1B1B1B1B1D1B1B1B1B1B1B1B1B72
S31508010DC01B1B484C5000012333E029462046FFF7F8
S31508010DD056FE08B901232CE029462046FFF7A0FF55
S31508010DE0012326E029462046FFF787FF012320E055
S31508010DF02046FFF71AFE2046FFF7F8FD012318E003
S31508010E002046FFF7FAFD034698B12046FFF70DFE87
S31508010E1001230EE029462046FFF727FE012308E0B5
S31508010E2063892B80012304E063882B80012300E07A
S31508010E300223184638BD2DE9F04782B082460C4692
S31508010E4017469846072B17D9A3F1080525F0070574
S31508010E5001F108031D44ADB2FF264FF000090096C3
S31508010E604B463A4621465046FFF792FD0834A4B24E
S31508010E70AC42F4D108F00708B8F1000F02D102B06C
S31508010E80BDE8F08788F00703013303F00703FF2263
S31508010E9002FA03F3DBB2009300233A462146504691
S31508010EA0FFF776FDEBE72DE9F04782B082460F465C
S31508010EB014469846072B17D9A3F1080525F0070507
S31508010EC002F108031D44ADB2FF264FF00109009651
S31508010ED04B46224639465046FFF75AFD0834A4B216
S31508010EE0AC42F4D108F00708B8F1000F02D102B0FC
S31508010EF0BDE8F08788F00703013303F00703FF22F3
S31508010F0002FA03F3DBB2009301232246394650461F
S31508010F10FFF73EFDEBE72DE9F04182B006460F46A5
S31508010F2015469846BDF820400094FFF780F810B999
S31508010F3002B0BDE8F08143462A4639463046FFF7F6
S31508010F407AFF23462A4639463046FFF7ACFF08F1B1
S31508010F50FF31394423462A4689B23046FFF7A3FFB3
S31508010F60013C2C444346A2B239463046FFF763FF9B
S31508010F70DEE72DE9F04180460F4615461E46BDF8C7
S31508010F80184033462A4639464046FFF754FF01358D
S31508010F90ADB2013CA4B2002CF3D1BDE8F0812DE934
S31508010FA0F04182B005460E4617469846BDF82040E0
S31508010FB00094FFF73CF810B902B0BDE8F08100943F
S31508010FC043463A4631462846FFF7D3FFF4E7002061
S31508010FD070472DE9F843054617461C464E68A2F1A7
S31508010FE01703302B1AD8DFE803F020191919191934
S31508010FF0191919191919191919191919191919610A
S315080110007E191919196119191919191919197E192F
S31508011010191919191919191919535A0023463A464A
S315080110203146FFF7B7FBBDE8F88323461722314659
S31508011030FFF7B0FB31462846FFF711FCB4F80490D8
S315080110406FEA090981441FFA89F931462846FFF7EB
S3150801105006FC2788FF430744BFB231462846FFF7F7
S315080110600AFCB4F806806FEA080880441FFA88F873
S3150801107031462846FFF7FFFB6388DB431844A4F88B
S315080110800090A4F80280A780E0800120BDE8F883DB
S315080110903146FFF7E4FB20800120BDE8F88331469D
S315080110A0FFF7E9FB20800120BDE8F8833146FFF709
S315080110B0E2FBB4F802806FEA080880441FFA88F850
S315080110C031462846FFF7CBFB2388DB4318442080AB
S315080110D0A4F8028023463A4631462846FFF75AFBCA
S315080110E00120BDE8F8833146FFF7C5FBB4F8028055
S315080110F06FEA080880441FFA88F831462846FFF740
S31508011100AEFB2388DB4318442080A4F80280637968
S31508011110023303F00303637123463A4631462846F0
S31508011120FFF738FB0120BDE8F883000008B54268DF
S31508011130044B9A4200D008BD5B684360FFF7ADFBDC
S31508011140F9E700BF8800002008B54368054A9342BD
S315080111501CBF53604260044A024B1A60FFF79DFBAD
S3150801116008BD00BF88000020D30F01087047FF287B
S3150801117008DDB0F5007F07DBB0F5407FB4BFA520D9
S31508011180A7207047A1207047A320704770B584B087
S31508011190841840F2FE339C4202DD002004B070BD83
S315080111A015460E460446FFF7E2FF0A230293019508
S315080111B000960123E2B2C1B20248FCF7E7FB01201F
S315080111C0ECE700BFCCCE002070B586B0841840F29B
S315080111D0FE339C4202DD002006B070BD15460E4660
S315080111E00446FFF7C4FF0A230293019505AB009352
S315080111F00123E2B2C1B20648FCF7C8FB9DF81420E8
S315080112009DF8153043EA022333800120E4E700BF45
S31508011210CCCE002070B584B0841840F2FE339C42CF
S3150801122002DD002004B070BD15460E460446FFF7E0
S315080112309EFF0A230293019500960123E2B2C1B2E9
S315080112400248FCF7A3FB0120ECE700BFCCCE002047
S31508011250FF2808DDB0F5007F07DBB0F5407FB4BF96
S31508011260A420A6207047A0207047A220704700003E
S3150801127070B584B0841840F2FE339C4202DD00202A
S3150801128004B070BD15460E460446FFF7E1FF0A2372
S315080112900293019500960123E2B2C1B20348FCF715
S315080112A0D1FA0420FBF79EF90120E9E7CCCE00200C
S315080112B070B584B0841840F2FE339C4202DD0020EA
S315080112C004B070BD15460E460446FFF7C1FF0A2352
S315080112D00293019500960123E2B2C1B20348FCF7D5
S315080112E0B1FA0420FBF77EF90120E9E7CCCE00200C
S315080112F030B587B00023ADF814300B888DF815305A
S31508011300811840F2FE33994202DD002007B030BD54
S3150801131015460446FFF79CFF0A230293019505AB80
S3150801132000930123E2B2C1B20348FCF78BFA042009
S31508011330FBF758F90120E9E7CCCE0020017000221D
S3150801134042708270C2704260C26002610F49416197
S31508011350A1F1B561A1F58B318161C2610262426277
S3150801136002854285C26240F6B83101860849416361
S3150801137041F288310187428702218187C287082184
S3150801138080F8401080F84120704700BF008BD48256
S31508011390801A060070B582B0047861F07F018DF875
S315080113A000108DF801208DF802309DF818308DF85F
S315080113B003309DF81C308DF80430032C01DD02B092
S315080113C070BD0B4E0B4D002236F814102846FBF75C
S315080113D09BFF4FF47A73052269460748FDF770FBB0
S315080113E0012236F814102846FBF78EFFE7E700BFFF
S315080113F094000020000C02406C11002000B583B057
S31508011400CBB20193C1F307230093C1F307430A0E35
S315080114102D21FFF7BFFF03B05DF804FB00B583B0CC
S31508011420084A8A42A8BF0A46D3B20193C2F30723E0
S315080114300093C2F30743120E2721FFF7ABFF03B050
S315080114405DF804FB00FE7F0000B583B04FF6FF721E
S315080114508A42A8BF0A46D3B20193C2F3072300936F
S31508011460C2F30743120E2821FFF794FF03B05DF874
S3150801147004FB30B583B005460C464FF6FF728A4227
S31508011480A8BF0A46D3B20193C2F307230093C2F356
S315080114900743120E2621FFF77DFF21462846FFF74F
S315080114A0D3FF03B030BD2DE9F04383B006460D46A0
S315080114B00423019300240094234622462021FFF7A2
S315080114C069FF2F0EC5F30748C5F30729EDB2019544
S315080114D0CDF8009043463A4621213046FFF75AFF98
S315080114E00195CDF8009043463A462D213046FFF73F
S315080114F051FF019400942346224620213046FFF7E6
S3150801150049FF03B0BDE8F08300B583B001920091AD
S3150801151000221021FFF73EFF03B05DF804FB00002F
S31508011520042B00DD70472DE9F0411C4616460D4691
S31508011530DFF834800A4F002238F813103846FBF7D3
S31508011540E3FEC823B2B229460648FDF7B9FA0122D5
S3150801155038F814103846FBF7D7FEBDE8F08100BF0E
S31508011560000C02406C11002094000020F0B587B0F1
S315080115700546274B93E8030004908DF81410C823F9
S31508011580052204A92348FDF79BFA29780122224B53
S3150801159033F811102148FBF7B7FE214F2B78214E5E
S315080115A0012237F813103046FBF7AEFE0A20FBF787
S315080115B019F8A1238DF8083000248DF809408DF813
S315080115C00A408DF80B408DF80C402B78052202A9AC
S315080115D02846FFF7A5FF0A20FBF704F8AD238DF887
S315080115E000308DF801408DF802408DF803408DF8E2
S315080115F004402B78052269462846FFF791FF2B7888
S31508011600224637F813103046FBF77EFE07B0F0BDC9
S3150801161020FF02086C11002094000020000C0240F3
S315080116203C0800200008024030B58FB00446057812
S31508011630334B03F1080292E803000C908DF834103D
S3150801164003F1100292E803000A908DF82C1003F1B9
S31508011650180292E8030008908DF8241003F120027D
S3150801166092E8030006908DF81C1003F1280292E80F
S31508011670030004908DF8141093228DF80820002297
S315080116808DF809208DF80A208DF80B208DF80C208D
S31508011690303393E8030000908DF804102B46052299
S315080116A00CA92046FFF73CFF2B4605220CA920462C
S315080116B0FFF736FF2B4605220AA92046FFF730FF1A
S315080116C02B46052208A92046FFF72AFF2B460522A5
S315080116D006A92046FFF724FF2B46052204A9204622
S315080116E0FFF71EFF2B46052202A92046FFF718FF22
S315080116F02B46052269462046FFF712FF0FB030BD7B
S3150801170020FF020830B58BB004460578264B03F155
S31508011710080292E8030008908DF8241003F11002DC
S3150801172092E8030006908DF81C1003F1380292E83E
S31508011730030004908DF81410203393E803000290F7
S315080117408DF80C1080238DF8003000238DF80130B8
S315080117508DF802308DF803308DF804302B460522BA
S3150801176008A92046FFF7DCFE2B46052208A92046D4
S31508011770FFF7D6FE2B46052206A92046FFF7D0FE1F
S315080117802B46052204A92046FFF7CAFE2B46052249
S3150801179002A92046FFF7C4FE2B46052269462046C4
S315080117A0FFF7BEFE0BB030BD20FF020830B593B07F
S315080117B0044605783D4B03F1500292E80300109068
S315080117C08DF84410A5228DF8382000228DF839208D
S315080117D08DF83A208DF83B208DF83C2003F158010D
S315080117E003C90C908DF8341003F1600103C90A90FE
S315080117F08DF82C1003F1680103C908908DF824109F
S3150801180003F1700103C906908DF81C1003F17801E4
S3150801181003C904908DF81410A0218DF808108DF8CD
S3150801182009208DF80A208DF80B208DF80C208033BD
S3150801183093E8030000908DF804102B46052210A9A1
S315080118402046FFF76DFE2B4605220EA92046FFF717
S3150801185067FE2B4605220CA92046FFF761FE2B469B
S3150801186005220AA92046FFF75BFE2B46052208A991
S315080118702046FFF755FE2B46052206A92046FFF707
S315080118804FFE2B46052204A92046FFF749FE2B46A3
S31508011890052202A92046FFF743FE2B460522694683
S315080118A02046FFF73DFE13B030BD00BF20FF0208FA
S315080118B02DE9F041044690461F469DF818509DF8BB
S315080118C01C6001291CD002291DD02046FFF76EFF96
S315080118D0C4F8348041462046FFF7A0FD27863946DD
S315080118E02046FFF7C6FD84F8405084F841609DF80C
S315080118F02030324629462046FFF706FEBDE8F0812C
S31508011900FFF700FFE1E7FFF78FFEDEE700000000C3
S3150801191070B582B0002501951F4B1A6C42F0010281
S315080119201A641B6C03F0010301931C4C4FF08043AE
S3150801193023600126DE606560A56010EE100AF6F7E1
S31508011940E1FD02460B4612A1D1E90001F6F758FF5F
S315080119500022134BF6F776FCF7F720F907EE900A03
S31508011960FCEEE77AC4ED037A256165612046FDF749
S315080119707FFC2046FDF742FB2A4631461C20FBF731
S31508011980BFF81C20FBF7ECF802B070BDAFF300807E
S31508011990000000002A75954100380240D80F002042
S315080119A00000F03F70B596B005460C464F26324604
S315080119B0002102A814F0C3FD52238DF80830112323
S315080119C08DF8093080238DF80A30FF238DF80C3005
S315080119D063788DF80F3023788DF81030A3788DF859
S315080119E01130E3788DF8123023798DF81330637945
S315080119F08DF81430A3798DF815300023E371A98980
S31508011A00A868EB7D0193AB7D0093334602AAF8F7EC
S31508011A1001F916B070BDA0F12C00C3E708B52C304A
S31508011A20F9F72CF908BD10B47F2380F8303080F817
S31508011A30313080F8323080F83330416B6FF317015B
S31508011A404163C26E6FF31702C266002380F837300E
S31508011A5080F8383090F8524044F0800480F85240BB
S31508011A6090F8564044F0800480F8564090F85B4060
S31508011A7044F0800480F85B4090F85F4044F08004AD
S31508011A8080F85F4090F8644044F0800480F8644030
S31508011A9090F8684044F0800480F86840082464F3AC
S31508011AA0030180F83410114664F3030180F86C10C1
S31508011AB0120E63F3030280F86F2080F87A3080F8FB
S31508011AC0733080F8723080F8763080F8753080F897
S31508011AD0743080F8783080F8773080F879305DF89E
S31508011AE0044B704710B584B004467F2380F8303024
S31508011AF080F8313080F8323080F83330416B6FF33B
S31508011B0017014163C26E6FF31702C266002380F89C
S31508011B10373080F8383090F8520040F0800084F869
S31508011B20520094F8560040F0800084F8560094F864
S31508011B305B0040F0800084F85B0094F85F0040F099
S31508011B40800084F85F0094F8640040F0800084F80F
S31508011B50640094F8680040F0800084F86800082062
S31508011B6060F3030184F83410114660F3030184F825
S31508011B706C10120E63F3030284F86F2084F87A302E
S31508011B8084F8733084F8723084F8763084F87530C6
S31508011B9084F8743084F8783084F8773084F87930AA
S31508011BA043238DF80C3002238DF80D30A189E27D8F
S31508011BB00192A27D009203AAA068F8F72BF8636840
S31508011BC013B1984704B010BD002384F8743084F823
S31508011BD07530142384F87630012384F87930F1E7D7
S31508011BE010B586B0414B93F93C302BB1012B2DD062
S31508011BF0022B53D006B010BD3D4A536C23F0100397
S31508011C0053643C4C4FF4C0612046FBF7DFFA2520AC
S31508011C10FAF7B2FF4FF4C0630193374B02930123DE
S31508011C20039301A92046FBF7F3F9002206211720A1
S31508011C30FAF766FF1720FAF793FF002207212820F3
S31508011C40FAF75EFF2820FAF78BFFD3E74FF4C06156
S31508011C502848FBF7BBFA1720FAF78EFF2820FAF770
S31508011C608BFF2248254B03644FF4614343640023E9
S31508011C708364C36403650C2242658365C36540308A
S31508011C80FDF7E8FC48B91948036C5B68012200F1C5
S31508011C9080014030FDF732FEACE7FEE74FF4C06144
S31508011CA01448FBF793FA1720FAF766FF2820FAF784
S31508011CB063FF0E48114B03644FF4E1334364002379
S31508011CC08364C36403650C2242658365C36540303A
S31508011CD0FDF7C0FC48B90548036C5B68012200F1B1
S31508011CE080014030FDF70AFE84E7FEE7D80F0020A1
S31508011CF00038024000000240000031100010014087
S31508011D0030B5ADB000210191364B1A6C42F08052C4
S31508011D101A641B6C03F0805301930291324B1A68C3
S31508011D2042F440421A601B6803F4404302930723B6
S31508011D301F93012320932193229310222392022396
S31508011D4025934FF48001269127924FF4B472289275
S31508011D50299305222A922B931FA8FCF701FC002838
S31508011D603ED1FBF737FF00283BD107231A930225FB
S31508011D701B9580231C934FF480531D9300241E94B6
S31508011D8005211AA8FBF7C4FF4FF440730393149473
S31508011D904FF000631893102309934FF4C0730A9305
S31508011DA008230B930C9501230E9303A8FCF7BEF8A1
S31508011DB0224621462046FBF75DFFFCF781F80B4BCF
S31508011DC0A3FB00308009FAF7E5FE0420FAF706FFBF
S31508011DD0224621464FF0FF30FAF792FE2DB030BD6C
S31508011DE0FEE7FEE70038024000700040D34D62105E
S31508011DF0F8B51D4CB4F8B41004F184074900384607
S31508011E00FFF737FBB4F8F81004F1C8064900304665
S31508011E10FFF72FFBB4F83C01F6F762FB0022134BE0
S31508011E20F6F7C4FBF6F79AFE04F5867501462846C9
S31508011E30FFF71FFBB4F8801104F5A8744900204682
S31508011E40FFF717FB00213846FFF7E8FA002130466D
S31508011E50FFF7E4FA00212846FFF7E0FA00212046B9
S31508011E60FFF7DCFAF8BD00BFD80F00200000F83FE5
S31508011E702DE9F04788B0002306938DF81C302122FE
S31508011E808DF8182004938DF814306F238DF81030CF
S31508011E90344C0126344D4FF00008DFF8D09009F58F
S31508011EA0CA770CE0314A82F88610C2F8883008B041
S31508011EB0BDE8F08789F8CA10C9F8CC300136A246C0
S31508011EC0424621882846FBF71FFA4FF47A73052202
S31508011ED006A93846FCF7F4FD012221882846FBF7B6
S31508011EE013FA424634F8021B2846FBF70DFA4FF45B
S31508011EF07A730093052302AA04A93846FCF7AFFEB4
S31508011F000122BAF800102846FBF7FEF99DF80810D9
S31508011F109DF809209DF80A301B0443EA02639DF8DF
S31508011F200C2013439DF80B2043EA0223721E032A51
S31508011F3014D801A050F822F0531F0108491F0108BF
S31508011F40B51E0108A51E010889F80E11C9F8103138
S31508011F50B4E789F85211C9F85431AFE7032EADDD5C
S31508011F60A5E700BF94000020000C0240D80F00200E
S31508011F702DE9F04F89B0002306938DF81C302222F3
S31508011F808DF8182004938DF814306F238DF81030CE
S31508011F903D4C04F1080A25463C4E4FF00009DFF88E
S31508011FA0F4802F464A4635F8021B3046FBF7ACF952
S31508011FB04FF47A73052206A94046FCF781FD0122F2
S31508011FC039883046FBF7A0F95545EAD101252F4F47
S31508011FD04FF0000ADFF8B88008F5CA790CE02C4AF8
S31508011FE082F88610C2F8943009B0BDE8F08F88F8F7
S31508011FF0CA10C8F8D83001356E1EA346524634F8C1
S31508012000021B3846FBF780F94FF47A7300930523D0
S3150801201002AA04A94846FCF722FE0122BBF80010D1
S315080120203846FBF771F99DF808109DF809209DF8C7
S315080120300A301B0443EA02639DF80C2013439DF8FA
S315080120400B2043EA0223B3F5000FC8BF03F17F4310
S31508012050032E15D801A252F826F000BF77200108F1
S315080120606D200108EF1F0108DF1F010888F80E110E
S31508012070C8F81C31BFE788F85211C8F86031BAE7C9
S31508012080032DB8DDB0E700BF94000020000C024024
S31508012090D80F00206C11002070B5FFF769FF4FF4C7
S315080120A000717948FBF72AF9002866D1774B9D68B4
S315080120B06D424FF400517448FBF720F900286BD1A3
S315080120C0724B9D684FF480416F48FBF717F900285A
S315080120D071D16E4B9C684FF400616B48FBF70EF9A2
S315080120E0002877D1694B9C686442694B93F9EC31B6
S315080120F0012B00F0AE80664B93F9ED31012B08BF39
S315080121000024644E4FF47A713046FFF7B2F985EA36
S31508012110E571A1EBE5713046FFF780F9002D00F076
S31508012120A780002D0ADD5A4BD3F89810D3F89C30B6
S315080121309942D8BF19465748FFF760F9002D59DB70
S31508012140554D4FF47A712846FFF793F984EAE471FD
S31508012150A1EBE4712846FFF761F9002C58D0002C51
S315080121605FDD4B4BD3F8DC10D3F8E0309942D8BF8A
S3150801217019464948FFF742F970BD4FF48071424844
S31508012180FBF7BCF8002891D080213F48FBF7B6F849
S31508012190002500288DD189E74FF480513A48FBF78D
S315080121A0ADF800288CD04FF400613748FBF7A6F844
S315080121B0002887D184E74FF400513348FBF79EF88E
S315080121C0002886D080213048FBF798F8002400289B
S315080121D081D17EE74FF480612B48FBF78FF8002801
S315080121E080D04FF400712848FBF788F800287FF45F
S315080121F07CAF77E7264BD3F89820D3F89C108A4210
S31508012200CEBF03F1840011462248FFF7F7F897E796
S315080122104FF4FA612846FFF72CF900212846FFF703
S31508012220FDF81B4BD3F8DC10D3F8E0309942C8BF50
S3150801223019461948FFF7E2F870BD164C4FF47A7142
S315080122402046FFF716F900212046FFF7E7F8002494
S315080122500EE00F4B93F9ED31012BEED00D4D4FF4F6
S315080122607A712846FFF705F900212846FFF7D6F8BF
S31508012270084D4FF4FA612846FFF7FBF80021284676
S31508012280FFF7CCF85CE700BF00100240940000207D
S31508012290D80F00205C100020A010002070B5FFF7B1
S315080122A067FE4FF400718648FBF728F8002874D1B9
S315080122B0844BD3F840516D424FF400518048FBF7E7
S315080122C01DF8002878D17F4BD3F840514FF480414F
S315080122D07B48FBF713F800287FD17A4BD3F8844162
S315080122E04FF400617648FBF709F8002840F086802C
S315080122F0744BD3F884416442724B93F9EE31012B46
S3150801230000F0C0806F4B93F9EF31012B08BF002411
S315080123106C4B03F58676B3F83C113046FFF7A9F8FE
S3150801232085EAE571A1EBE5713046FFF777F8002DEF
S3150801233000F0B980002D0ADD624BD3F82011D3F8DD
S3150801234024319942D8BF19465F48FFF757F8002D3F
S3150801235065DB5C4B03F5A875B3F880112846FFF7D2
S3150801236088F884EAE471A1EBE4712846FFF756F888
S3150801237041F288312846FFF767F8002C5DD0002C1A
S3150801238066DD504BD3F86411D3F868319942D8BF4A
S3150801239019464E48FFF732F870BD4FF48071484828
S315080123A0FAF7ACFF002883D080214548FAF7A6FF43
S315080123B00025002880D17BE74FF480514048FAF781
S315080123C09DFF00283FF47FAF4FF400613C48FAF7C0
S315080123D095FF00287FF47AAF75E74FF40051384826
S315080123E0FAF78CFF00283FF478AF80213448FAF7D2
S315080123F085FF002400287FF473AF6EE74FF48061F0
S315080124002F48FAF77BFF00283FF472AF4FF40071AB
S315080124102B48FAF773FF00287FF46EAF68E7294B5C
S31508012420D3F82021D3F824118A42CEBF03F586704A
S3150801243011462548FEF7E2FF8BE7A5F5A873B3F821
S3150801244080112846FFF715F800212846FEF7E6FF12
S315080124501C4BD3F86411D3F868319942C8BF1946A1
S315080124601A48FEF7CBFF70BD164B03F58674B3F811
S315080124703C112046FEF7FDFF00212046FEF7CEFF60
S31508012480002410E00F4B93F9EF31012BECD00D4BE3
S3150801249003F58675B3F83C112846FEF7EAFF0021D5
S315080124A02846FEF7BBFF074B03F58675B3F83C11C3
S315080124B02846FEF7DEFF00212846FEF7AFFF48E76C
S315080124C000100240D80F0020E41000202811002037
S315080124D008B54FF480416C48FAF710FFC0B96B4A4A
S315080124E0B2F86C3201339BB2A2F86C320121684A08
S315080124F0117340F2E14293423CDD13F0070F39D1E3
S315080125001022624B83F86E223222614B1A7309E05C
S3150801251000216048F8F77CFB0028E0D100225B4BDC
S31508012520A3F86C224FF480615748FAF7E7FE0028B2
S315080125304BD1564AB2F8703201339BB2A2F87032C7
S315080125400121534A117340F2E242934265DD524A30
S31508012550A2FB0312D20802EB8202A3EB420292B259
S31508012560002A5AD11222494B83F86E223222484B4D
S315080125701A7334E040F2ED22934210DD474AA2FB7A
S315080125800312D208C2EB02129A1A92B23AB910226F
S315080125903E4B83F86E2214223D4B1A73C2E7F92B80
S315080125A0C0DD3F4AA2FB0312D20802EB820202EB0C
S315080125B082029B1A9BB2002BB4D11022334B83F8AB
S315080125C06E220522324B1A73ACE702213148F8F71D
S315080125D01FFB0028ADD100222C4BA3F870224FF423
S315080125E000412948FAF78AFE002841D1274AB2F85C
S315080125F0723201339BB2A2F87232FA2B42DD294AB2
S3150801260082FB03121211FA2101FB1233012B39D174
S315080126100F221E4B83F86E2208BD40F2EE2293422A
S3150801262010DD1E4AA2FB0312D208C2EB02129A1A45
S3150801263092B23AB91222154B83F86E221422144B20
S315080126401A73CCE7FA2BCADD154AA2FB0312D20884
S3150801265002EB820202EB82029B1A9BB2002BBED1CD
S3150801266012220A4B83F86E220522094B1A73B6E722
S315080126700E210848F8F7CCFA0028B7D10022034BF7
S31508012680A3F8722208BD00BF00100240D80F00202F
S3150801269094000020F4110020CDCCCCCC8988888800
S315080126A01F85EB51D34D621010B510211348F8F769
S315080126B0AFFAF0B1124AB2F8743201339BB2A2F8FA
S315080126C07432FA2B19DD0F4A82FB03121211FA2111
S315080126D001FB1233012B10D1094B93F8053263B173
S315080126E0074C04F5F870F7F764FF0023A4F8743271
S315080126F010BD0022024BA3F8742210BDF41100206C
S31508012700D80F0020D34D621070B52DED048BF0EE75
S31508012710408A4E48D0ED507AF8EE677A87EE809A6D
S31508012720002100F50770F8F7A6FA494B93F912301C
S31508012730022B04D0032B05D023B1803803E0C0F166
S31508012740800000E00020414B93F9EE31012B25D0A2
S3150801275000F10D031A2B68D9002820DA07EE900A32
S31508012760B8EEE78AF1EE497A17EE900AF5F7CAFE4E
S315080127700022384BF5F71AFF04460D4668EE087A2B
S3150801278017EE900AF5F7BEFE02460B462046294685
S31508012790F5F70CFFF6F7BAF904461DE0002007EE37
S315080127A0900AF8EEE77A67EEA77A17EE900AF5F738
S315080127B0A9FE04460D4619EE100AF5F7A3FE0022F6
S315080127C0244BF5F7F3FE02460B4620462946F5F754
S315080127D0EDFEF6F79BF904461C4E06F5867584EA66
S315080127E0E471A1EBE4712846FEF718FEB6F83C3110
S315080127F007EE903AF8EEE77A87EEA87AFCEEC77A02
S3150801280017EE901A2846FEF734FE002C0FDDD6F88F
S315080128102011D6F824319942CEBF284619460E48CA
S31508012820FEF7ECFDBDEC048B70BD0020B7E7002C6C
S31508012830F8DA064BD3F82011D3F824319942C8BFE8
S3150801284019460548FEF7DAFDECE700BFD80F002068
S31508012850940000200000103FE41000200000000052
S3150801286070B52DED048BF0EE608A534DD5ED617A86
S31508012870F8EE677A87EE809A05F5077509212846E5
S31508012880F8F7F0F9044608212846F8F7EBF9201A73
S315080128904A4B93F91330022B2FD0032B00D003B9DF
S315080128A00020454B93F9EF31012B28D000F10D0398
S315080128B01A2B6CD9002823DA07EE900AB8EEE78AB4
S315080128C0F1EE497A17EE900AF5F71CFE38A3D3E91B
S315080128D00023F5F795FF04460D4668EE087A17EECC
S315080128E0900AF5F70FFE02460B4620462946F5F7EC
S315080128F05DFEF6F70BF9044620E04042D1E70020D9
S3150801290007EE900AF8EEE77A67EEA77A17EE900ACD
S31508012910F5F7F8FD04460D4619EE100AF5F7F2FD2E
S3150801292023A3D3E90023F5F76BFF02460B4620469E
S315080129302946F5F73BFEF6F7E9F804461E4E06F575
S31508012940A87584EAE471A1EBE4712846FEF766FDF1
S31508012950B6F8803107EE903AF8EEE77A87EEA87A6C
S31508012960FCEEC77A17EE901A2846FEF782FD002C70
S315080129700FDBD6F86411D6F868319942CEBF2846DE
S3150801298019460F48FEF73AFDBDEC048B70BD0020D1
S31508012990B6E7094BD3F86411D3F868319942C8BF31
S315080129A019460748FEF72AFDEEE700BFAFF3008098
S315080129B00000000020C0EF40D80F0020940000203E
S315080129C028110020F8B52DED048BB0EE409AF0EEF3
S315080129D0608AD248D0ED2E7AF8EE677AC7EE809AE9
S315080129E0022100F50770F8F746F9CD4B93F9103037
S315080129F0022B64D0032B65D0002B63D0803800F1FD
S31508012A000D031A2B98BF002080EAE074A4EBE0744A
S31508012A10E4B2C24B93F9EC31012B55D0002855DBB2
S31508012A2007EE900AF8EEE77A67EEA77A17EE900AAC
S31508012A30F5F768FD06460F4619EE900AF5F762FDA9
S31508012A400022B84BF5F7B2FD02460B463046394629
S31508012A50F5F7ACFDF6F75AF8054685EAE571A1EBF7
S31508012A60E571B148FEF7DAFC002D62DDAB48D0F816
S31508012A709860D0F89C50B0F8B43007EE903AF8EE6A
S31508012A80E77A87EE897AFCEEC77A17EE901A8430D0
S31508012A90FEF7EFFCAE4239DDA04D314605F1840063
S31508012AA0FEF7ACFCD5F888309E4244D185F86242DF
S31508012AB0002285F86322012285F869223BE0C0F1EC
S31508012AC080009CE700209FE70020A9E707EE900A0F
S31508012AD0B8EEE78AF1EE697A17EE900AF5F712FD74
S31508012AE00022904BF5F762FD06460F4668EE087A16
S31508012AF017EE900AF5F706FD02460B4630463946AB
S31508012B00F5F754FDF6F702F80546A6E7834E29467A
S31508012B1006F18400FEF772FCD6F888309D420AD188
S31508012B2086F86242002286F86322012286F8692223
S31508012B3001E0002D16DB7948D0ED3F7AF8EE677A89
S31508012B4087EEA89A032100F50770F8F794F8744BF5
S31508012B5093F91130022B41D0032B42D0002B40D0E0
S31508012B6082383FE06D48D0F89850D0F89C60B0F8AC
S31508012B70B43007EE903AF8EEE77A87EE897AFCEEFA
S31508012B80C77A17EE901A8430FEF773FCB54212DD48
S31508012B90624D314605F18400FEF730FCD5F88830E0
S31508012BA09E42C8D185F86242002285F86322012235
S31508012BB085F86922BFE7594E294606F18400FEF7D2
S31508012BC01DFCD6F888309D42B5D186F862420022AE
S31508012BD086F86322012286F86922ACE7C0F18200F1
S31508012BE000E000204D4B93F9ED31012B2AD000F17D
S31508012BF00D031A2B71D980EAE075A5EBE075EDB2E4
S31508012C00002821DA07EE900AB8EEE78AF1EE497A4A
S31508012C1017EE900AF5F776FC0022424BF5F7C6FC4B
S31508012C2006460F4668EE087A17EE900AF5F76AFC2B
S31508012C3002460B4630463946F5F7B8FCF5F766FF06
S31508012C4006461EE00025284607EE900AF8EEE77AC2
S31508012C5067EEA77A17EE900AF5F754FC06460F4673
S31508012C6019EE100AF5F74EFC00222E4BF5F79EFCDD
S31508012C7002460B4630463946F5F798FCF5F746FF06
S31508012C80064686EAE671A1EBE6712848FEF7C6FB19
S31508012C90002E4DDB2148D0F8DC70D0F8E060B0F8A2
S31508012CA0F83007EE903AF8EEE77A87EEA87AFCEE66
S31508012CB0C77A17EE901AC830FEF7DBFBB74219DD63
S31508012CC0164E394606F1C800FEF798FBD6F8CC3001
S31508012CD09F4205D0BDEC048BF8BD00252846B3E715
S31508012CE02C4486F86242002286F86322012286F87D
S31508012CF06922EFE7094F314607F1C800FEF77EFB67
S31508012D00D7F8CC309E42E5D12C4487F8624200229E
S31508012D1087F86322012287F86922DBE7D80F0020AA
S31508012D20940000200000103F5C100020A010002035
S31508012D301E48D0F8DC60D0F8E070B0F8F83007EE3D
S31508012D40903AF8EEE77A87EEA87AFCEEC77A17EE9C
S31508012D50901AC830FEF78DFBBE4213DD134E394675
S31508012D6006F1C800FEF74AFBD6F8CC309F42B1D12E
S31508012D702C4486F86242002286F86322012286F8EC
S31508012D806922A7E7094F314607F1C800FEF736FB66
S31508012D90D7F8CC309E429DD12C4487F86242002256
S31508012DA087F86322012287F8692293E7D80F002062
S31508012DB008B50022484B83F86E224FF480414748F4
S31508012DC0FAF79CFA88B90B22434B83F87622424AD2
S31508012DD092F8763292F877229A421CBF3E4A82F8D6
S31508012DE06E323D4A82F8773208BD00213C48F7F732
S31508012DF021FF0028E7D14FF480613848FAF77EFAB7
S31508012E0020B90D22344B83F87622E0E702213448B3
S31508012E10F7F710FF0028F4D14FF400412F48FAF7CD
S31508012E206DFA20B90A222C4B83F87622CFE70E21B8
S31508012E302B48F7F7FFFE0028F4D14FF480512748B5
S31508012E40FAF75CFA20B90C22234B83F87622BEE7FF
S31508012E5003212348F7F7EEFE0028F4D14FF48071D9
S31508012E601E48FAF74BFA20B90E221B4B83F8762235
S31508012E70ADE701211A48F7F7DDFE0028F4D10F2145
S31508012E801748F7F7D7FE20B10822134B83F87622A5
S31508012E909DE705211248F7F7CDFE20B109220E4B11
S31508012EA083F8762293E708210D48F7F7C3FE20B188
S31508012EB03622094B83F8762289E709210848F7F76C
S31508012EC0B9FE20B13722044B83F876227FE7002228
S31508012ED0014B83F876227AE7D80F002000100240CA
S31508012EE0F4110020000000002DE9F843744ED6F8CD
S31508012EF07842D6F88032E41A002CB8BF6442C6F884
S31508012F008842D6F87C52D6F88432ED1A002DB8BF1D
S31508012F106D42C6F88C526B4B187DF5F7E1FA002223
S31508012F20694BF5F76DFCF5F739FEF7EE007A07EE12
S31508012F30100A37EEC77A07EE904AF8EE677A67EE17
S31508012F40877AFCEEE77A17EE900AC6EDA47A07EEC1
S31508012F50905AF8EE677A67EE877AFCEEE77A17EE0B
S31508012F60904AC6EDA57A96F898321BB196F9993228
S31508012F70042B78D0524AD2F8A432D2F89C125B1AA2
S31508012F80002BB8BF5B42D2F8A852D2F8A022AD1ADC
S31508012F90002DB8BF6D42B3FBF0F007EE900AF8EECC
S31508012FA0677A17EE900AF5F7ADFA00224FF08043DB
S31508012FB0F5F74AF9F5F7AAFD0646414BC3F8AC02FF
S31508012FC02846F5F77DFA3CA3D3E90023F5F760FD1A
S31508012FD0002859D001223A4BC3F8B022384CD4F80C
S31508012FE0B05205FB06F3C4F8B432D4F8A402D4F8F7
S31508012FF09C32C01AF5F774FA804689463046F5F7C9
S315080130006FFA0022314BF5F71DF902460B46404689
S315080130104946F5F7F5FBF5F7C1FD07EE900AFDEE12
S31508013020E77AC4EDAE7AD4F8A802D4F8A032C01A69
S31508013030F5F756FA06460F462846F5F751FA0022DD
S31508013040224BF5F7FFF802460B4630463946F5F7A7
S31508013050D7FBF5F7A3FD07EE900AFDEEE77AC4ED77
S31508013060AF7ABDE8F883D6F88830D6F89C125B1A91
S31508013070002BB8BF5B42D6F8CC50D6F8A022AD1AC1
S31508013080002DB8BF6D4286E7B5FBF4F007EE900A4E
S31508013090F8EE677A17EE900AF5F734FA00224FF040
S315080130A08043F5F7D1F8F5F731FD054BC3F8B002C2
S315080130B094E700BFAFF300800000000000F4C040B1
S315080130C0D80F002094000020000059400000F03F6E
S315080130D02DE9F0473A4AD2F8AC3290FBF3F803FBF4
S315080130E0180092F9C02252B9013BA3EB4003B8F18B
S315080130F0000F08F00102B8BF524202FB0300304B31
S31508013100D3F8B872D3F8A42207FB1027D3F8BC2248
S31508013110D3F8A83202FB18382A4B93F91530032B3A
S315080131204BD8DFE803F0022A36404FF47A72244B73
S31508013130A3F8C222FA254FF0960A234E4CF25031D3
S315080131401F4C04F184094846FEF768F9514648467A
S31508013150FEF78FF9C83431462046FEF75FF929464E
S315080131602046FEF786F939464846FEF747F94146AD
S315080131702046FEF743F9BDE8F0874FF4FA72104B83
S31508013180A3F8C22240F6B8354FF4FA6A0F4E0E4933
S31508013190D6E7FA220A4BA3F8C22241F28835AA4693
S315080131A00B4E0C49CCE76422054BA3F8C22242F226
S315080131B02835AA46084E3146C2E74FF0010ABFE74D
S315080131C0D80F002094000020A0860100400D0300BE
S315080131D0801A0600E0930400D0DD0600F0B58FB032
S315080131E03C493D48FDF7C8FA3C4B93F882308BB908
S315080131F03A4B93F8813033B1394B0822F8213648D6
S31508013200FDF73DFA11E0374B0822F8213248FDF760
S3150801321036FA0AE0314B93F88130002B37D0324B1E
S315080132200822F8212C48FDF72AFA2B4C2F4920466B
S31508013230FDF7A2FA2046FDF76FFA2046FDF780FA58
S3150801324094F8295094F82A30ED1AEDB2268803210C
S315080132502046FDF7AEFB264B002211462046FDF718
S315080132600EFA1E4B93F8C4323E2B17D01B4AD2F8DE
S31508013270B432D2F8C8221F4901A813F069FA01AB82
S315080132806A000F211448FDF7FAF90FB0F0BD1A4B81
S315080132900822F8211048FDF7F2F9C6E72746174B29
S315080132A02A460F212046FDF7EAF9154B01AC0FCB4B
S315080132B007C4237001A93846FDF748FA301A00EB0E
S315080132C0D07001AB3322C0F34F013846FDF7D7F969
S315080132D0CCE700BF2C9A020850D30020D80F002053
S315080132E000030308F802030804030308A0A302085D
S315080132F00803030838030308FC0203081803030834
S315080133002803030800B583B0064B019332230093C3
S315080133103A230A4601460448FCF71EFE03B05DF847
S3150801332004FB00BFAC00002050D300202DE9F04F6C
S3150801333083B0244C24492046FDF71EFA2046FDF7A2
S31508013340EBF92046FDF7FCF9B4F800A01F4F94F8F5
S31508013350298094F82A30A8EB03085FFA88F8002533
S315080133602E46DFF86CB03C4639681648FDF7EEF98B
S31508013370AAEB000000EBD070C0F34F0902211148F7
S31508013380FDF717FB9BF9CC32B3420ED004372368FD
S315080133902A4649460B48FDF772F901364544ADB24E
S315080133A0042EE0D103B0BDE8F08FCDF80080534676
S315080133B02A4600210348FDF7F2FD00210148FDF7E1
S315080133C0F8FAE3E750D300203C8A02083C020020C1
S315080133D0D80F00202DE9F04782B0254C2549204613
S315080133E0FDF7CAF92046FDF797F92046FDF7A8F932
S315080133F094F8296094F82A30F61AF6B2B4F80080DF
S3150801340002212046FDF7D5FA1B4BD3F8B831002225
S3150801341011462046FDF733F9B6B234460025144F56
S31508013420DFF858A0DFF8589002213846FDF7C1FAAF
S315080134309AF9CD32AB420ED059F8253022464121B0
S315080134403846FDF71CF901353444A4B2032DEBD1F6
S3150801345002B0BDE8F0870096434622460021384669
S31508013460FDF79DFD00213846FDF7A3FAE4E700BF05
S3150801347050D300203C8A020894000020D80F00206F
S315080134805002002010B58EB00D4C2046FDF74BF9C1
S315080134902046FDF79BFA2046FDF752F909492046D1
S315080134A0FDF76AF9084BD3F8C81101A813F082F998
S315080134B001AB002211462046FDF7E1F80EB010BD1A
S315080134C050D30020D4F7020894000020F0B58FB03D
S315080134D04B4C4C492046FDF74FF92046FDF71CF9A0
S315080134E02046FDF72DF903212046FDF762FA464BE2
S315080134F093F9CE32002B71D0434B93F9CE32012B7F
S3150801350075D03F4C01AB002211462046FDF7B7F8AE
S315080135103E492046FDF730F92046FDF7FDF82046DD
S31508013520FDF70EF925883A4E374F97F8CF3206EB55
S315080135308303D3F8CC112046FDF708F997F8CF3263
S3150801354006EB8303281A00EBD070D3F8CC310F228F
S31508013550C0F34F012046FDF792F82E492046FDF7A4
S315080135600BF92046FDF7D8F801212046FDF721FA87
S3150801357097F8CF3206EB8303D3F80C122046FDF7F2
S31508013580E5F897F8CF3206EB8303281A00EBD070DB
S31508013590D3F80C322B22C0F34F012046FDF76FF802
S315080135A097F8CF3206EB8303D3F84C122046FDF782
S315080135B0CDF897F8CF3206EB8306281A00EBD070C0
S315080135C0D6F84C323522C0F34F012046FDF757F89D
S315080135D003212046FDF7EDF90FB0F0BD0A4B93F82C
S315080135E0CF2201320C4901A813F0B2F884E7064B41
S315080135F093F8CF22043A094901A813F0A9F880E7FC
S3150801360050D30020A0A30208D80F0020D0C3020877
S3150801361094000020D4F7020844030308640303084E
S315080136202DE9F04F91B00646584C59492046FDF709
S31508013630A3F82046FDF770F82046FDF781F894F8BF
S31508013640297094F82A30FF1AFFB203212046FDF7A4
S31508013650B0F9504B002211462046FDF710F84E4DA1
S3150801366005EB8603D3F88C32002264212046FDF748
S3150801367006F84A4901EB0611D1F8D432D1F8D0221D
S31508013680D1F8D8120091464903A813F061F8BFB2E0
S3150801369003AB3A464B212046FCF7F1FF05EB4606FC
S315080136A0B6F99C32DFF8FC9089FB0321DA17C2EBE5
S315080136B0A10202EB8201A3EB4103DFF8EC801BB206
S315080136C012B2414603A813F043F803AB7A004B2123
S315080136D02046FCF7D4FFB6F9A43289FB0329DA1789
S315080136E0C2EBA90202EB8201A3EB41031BB212B2A0
S315080136F0414603A813F02CF803AB07EB47024B210D
S315080137002046FCF7BCFF05F52B753C460026DFF87D
S315080137107C90DFF888B014E01F4BD3F8BC32224600
S3150801372000214846FCF7ABFF0435DAF8003022469B
S3150801373041464846FCF7A3FF01363C44A4B2042E91
S3150801374020D0AA4629684846FDF700F8C0F1460088
S315080137505FFA80F803214846FDF72BF99BF91033E8
S31508013760B342E1D19BF89832002BD5D00097462376
S31508013770224600214846FDF712FC00214846FDF77E
S3150801378018F9D1E711B0BDE8F08F00BF50D300207A
S31508013790A0A302088003030894000020D80F002084
S315080137A09003030867666666C80303082DE9F04FA8
S315080137B091B05F4D5F492846FCF7DEFF2846FCF7C6
S315080137C0ABFF2846FCF7BCFF95F8296095F82A3027
S315080137D0F61AF6B203212846FDF7EBF8564CD4F84B
S315080137E0F032D4F8EC22554903A812F0B1FF03AB25
S315080137F0002211462846FCF742FFD4F8FC32504A0B
S31508013800B2F812234F4903A812F0A2FFB6B203ABCE
S31508013810324678212846FCF732FF94F9083304EB3F
S315080138204303B3F80023484903A812F091FF03ABF9
S31508013830720078212846FCF722FFD4F8FC22434976
S3150801384003A812F085FF03AB06EB4602782128464A
S31508013850FCF715FF01212846FDF7ABF8D4F8FC2241
S3150801386094F9083304EB4303B3F8007302EB8201BE
S31508013870490091FBF7F1364880FB0130CB17C3EBC2
S31508013880A00303EB8303A1EB430392FBF7F2314950
S3150801389003A812F05DFF03ABB20019212846FCF715
S315080138A0EEFE03212846FDF784F804F543743546F0
S315080138B00027DFF87C90DFF888B014E01E4BD3F8B8
S315080138C0BC322A4600214846FCF7D9FE0434DAF808
S315080138D000302A4641464846FCF7D1FE01373544B1
S315080138E0ADB2032F20D0A24621684846FCF72EFF29
S315080138F0C0F169005FFA80F803214846FDF759F8D7
S315080139009BF91433BB42E1D19BF89832002BD5D0F1
S31508013910009669232A4600214846FDF740FB002107
S315080139204846FDF746F8D1E711B0BDE8F08F00BF6C
S3150801393050D30020A0A30208940000209C0303088A
S31508013940D80F0020A4030308B403030834070308A7
S3150801395067666666BC0303082DE9F04F91B0584EB9
S3150801396058493046FCF708FF3046FCF7D5FE304685
S31508013970FCF7E6FE96F8295096F82A30ED1AEDB2CC
S3150801398003213046FDF715F84F4CD4F8F432D4F834
S31508013990EC224E4903A812F0DBFE03AB00221146C6
S315080139A03046FCF76CFED4F8FC32494AB2F81223C9
S315080139B0484903A812F0CCFEADB203AB2A467D21D5
S315080139C03046FCF75CFE94F9383304EB4303B3F84D
S315080139D01823414903A812F0BBFE03AB6A007D21F7
S315080139E03046FCF74CFE01213046FCF7E2FFD4F8DD
S315080139F0FC2294F9383304EB4303B3F8187302EB4A
S31508013A008201490091FBF7F1344880FB0130CB175D
S31508013A10C3EBA00303EB8303A1EB430392FBF7F28A
S31508013A202F4903A812F094FE03AB05EB45021E21AC
S31508013A303046FCF724FE03213046FCF7BAFF04F5AD
S31508013A404F742E460027DFF87890DFF884B0A24637
S31508013A5021684846FCF77AFEC0F16E005FFA80F8E5
S31508013A6003214846FCF7A5FF9BF91533BB420FD046
S31508013A700434DAF80030324641464846FCF7FFFD81
S31508013A8001372E44B6B2022FE1D111B0BDE8F08F4D
S31508013A909BF8983243B90C4BD3F8BC323246002115
S31508013AA04846FCF7ECFDE3E700956E233246002114
S31508013AB04846FDF774FA00214846FCF77AFFD7E72E
S31508013AC050D30020A0A30208940000209C030308F9
S31508013AD0D80F0020A4030308B403030867666666C3
S31508013AE0D40303082DE9F04F91B0964CB4F9443349
S31508013AF0D4F8FC1201FB03F6934D94492846FCF7CA
S31508013B003BFE01212846FCF754FF914AA2FB0632E7
S31508013B10D20B48F6A04303FB12638E49A1FB0303AC
S31508013B20A1FB060189094FF4167000FB11618A4849
S31508013B30A0FB0101C90800919B09884903A812F055
S31508013B4007FE03AB36220A212846FCF798FDD4F86E
S31508013B50FC22834903A812F0FBFD03AB3622872119
S31508013B602846FCF78CFDD4F8FC62D4F848137D4A44
S31508013B7082FB01304FEAE17CCCEBA00000EB400070
S31508013B80A1EBC00000EB8000400082FB0073C01768
S31508013B9082FB0672F717DFF8E4E18EFB0198884489
S31508013BA0CCEB281CCCEB0C1CA1EB4C0101EB8101E5
S31508013BB049008EFB018C8C44C917C1EB2C1101916C
S31508013BC08EFB061E7644C7EB26160096C0EBA303AA
S31508013BD0C7EBA202644903A812F0BAFD03AB3E2261
S31508013BE00A212846FCF74BFD604F39462846FCF763
S31508013BF0C3FD2846FCF790FD2846FCF7A1FD95F87C
S31508013C00296095F82A30F61AF6B203212846FCF7F8
S31508013C10D0FED4F8F832D4F8EC22554903A812F0AC
S31508013C2097FD03AB002211462846FCF728FDB4F997
S31508013C304433DFF84C8188FB0321DA17C2EBA10272
S31508013C4002EB8201A3EB41031BB212B2494903A855
S31508013C5012F07EFDB6B203AB32467D212846FCF74B
S31508013C600EFDB4F94C33B4F9440388FB0321DA1782
S31508013C70C2EBA10202EB8201A3EB410388FB001808
S31508013C80C117C1EBA80101EB810EA0EB4E0000B2F2
S31508013C90019009B200911BB212B2374903A812F07A
S31508013CA057FD03AB72007D212846FCF7E8FC39462F
S31508013CB02846FCF761FD03212846FCF77AFE04F540
S31508013CC0547435460027DFF88090DFF8B8B014E061
S31508013CD01C4BD3F8BC322A4600214846FCF7CFFCD8
S31508013CE00434DAF800302A4641464846FCF7C7FC50
S31508013CF001373544ADB2032F20D0A2462168484684
S31508013D00FCF724FDC0F178001FFA80F80321484624
S31508013D10FCF74FFE9BF91633BB42E1D19BF898326B
S31508013D20002BD5D0009678232A4600214846FDF770
S31508013D3036F900214846FCF73CFED1E711B0BDE84B
S31508013D40F08F00BF9400002050D30020D4F702085A
S31508013D50D55204E9B5814E1BCDCCCCCCEC03030876
S31508013D6004040308ABAAAA2A10040308A0A302089C
S31508013D709C030308C8030308340403088988888850
S31508013D8067666666D80F00202DE9F04190B05B4959
S31508013D905B48FCF7F1FC5B4B93F882308BB9594BC6
S31508013DA093F8813033B1584B0822F8215448FCF76F
S31508013DB066FC11E0554B0822F8215148FCF75FFCD7
S31508013DC00AE0504B93F88130002B69D0504B0822FA
S31508013DD0F8214B48FCF753FC494D4E492846FCF758
S31508013DE0CBFC2846FCF798FC2846FCF7A9FC95F875
S31508013DF0294095F82A30E41AE4B22E880321284688
S31508013E00FCF7D7FD444B002211462846FCF737FC40
S31508013E103C4B93F8C432332B49D0342B4ED0394E10
S31508013E20D6F81833D6F8C8223C4903A812F090FCF4
S31508013E30A4B2334D03AB62000F212846FCF71FFCE1
S31508013E40D6F81803D6F8C812401A354BB3F94413F5
S31508013E5001FB00F0334AA2FB0032D20B48F6A0431D
S31508013E6003FB12033049A1FB0363A1FB0061890926
S31508013E704FF4167606FB11012C48A0FB0101C9086F
S31508013E8000919B092A4903A812F062FC03AB04EBD3
S31508013E9044020F212846FCF7F2FB10B0BDE8F08179
S31508013EA0244B0822F8211648FCF7E9FB94E7224B34
S31508013EB022460F212846FCF7E2FBB0E7DFF84080EF
S31508013EC01E4B22460F214046FCF7D9FB03AD1C4F7A
S31508013ED00FCF0FC597E8030085E8030003A94046FD
S31508013EE0FCF734FC301A00EBD07003AB3322C0F375
S31508013EF04F014046FCF7C3FB91E700BF2C9A020825
S31508013F0050D30020D80F002000030308F802030845
S31508013F1004030308A0A30208480403083803030896
S31508013F2094000020D55204E9B5814E1BCDCCCCCCEA
S31508013F308C040308FC020308180303086404030835
S31508013F4074040308000000002DE9F04F2DED028BE3
S31508013F5091B0CB4CCB492046FCF70EFC2046FCF72A
S31508013F60DBFB2046FCF7ECFB94F8295094F82A3041
S31508013F70ED1AEDB203212046FCF71BFDC24ED6F819
S31508013F80C032002211462046FCF779FB0321204660
S31508013F90FCF70FFD96F9643306EB8306D6F85C1336
S31508013FA003A812F0D5FBADB203AB2A466E21204613
S31508013FB0FCF765FBB54B93F898322BB1B34A92F9E6
S31508013FC01C23012A00F0FE82B14BB24AB24903A86A
S31508013FD012F0BEFB03AB6A006E21A948FCF74FFB42
S31508013FE0AA4B93F89832012B00F00E81A74B93F850
S31508013FF09832022B00F09781A44B93F898322BB193
S31508014000A24B93F91C33022B00F01C83A04BA14A47
S31508014010A14903A812F09CFB03AB05EB45026E21EF
S315080140209748FCF72CFB994B93F89832012B00F033
S315080140308181964B93F89832022B00F0E081012199
S315080140408F48FCF7B6FC914B93F8983243B18F4BE6
S3150801405093F91C33012B00F0D981022B00F0F18171
S315080140608A4BD3F8A400D3F8A030C01A0028B8BFE9
S31508014070404207EE900AF8EEE77A17EE900AF4F74F
S3150801408041FA7BA3D3E90023F4F7BAFBF4F786FDDB
S3150801409000EE100ABDEEC08AF8EEC87A30EE670A5D
S315080140A0DFED7E7A20EE270A11F0F4FEFDEEC07AE6
S315080140B017EE903A092B18EE102ACCBF78497949A0
S315080140C003A812F045FBAC00023403AB22460021DB
S315080140D06B48FCF7D4FA6D4B93F8983243B16B4BA6
S315080140E093F91C33012B00F0C781022B00F0DF8105
S315080140F0664BD3F8E800D3F8E430C01A0028B8BFF5
S31508014100404207EE900AF8EEE77A17EE900AF4F7BE
S31508014110F9F959A3D3E90023F4F772FBF4F73EFD45
S3150801412000EE100ABDEEC08AF8EEC87A30EE670ACC
S31508014130DFED5A7A20EE270A11F0ACFEFDEEC07AC1
S3150801414017EE903A092B18EE102ACCBF5649574953
S3150801415003A812F0FDFA03AB22464B214848FCF7A7
S315080141608EFA4A4B93F9CE32012B9FED517ADFED48
S31508014170517A18BFB0EE677A444B93F8983243B137
S31508014180424B93F91C33012B00F0AC81022B00F052
S31508014190B9813E4AD2F82C31D2F828219B1A002B34
S315080141A0B8BF5B4207EE903AF8EEE77A87EE870AE0
S315080141B0BDEEC08AF8EEC87A30EE670ADFED377AC7
S315080141C020EE270A11F066FEFDEEC07A17EE903A48
S315080141D0092B18EE102ACCBF3749384903A812F023
S315080141E0B7FA274E03AB224696213046FCF747FA23
S315080141F003213046FCF7DDFB314F2C460026DFF85C
S315080142008090DFF888B0A3E1204B93F91C33012B8A
S315080142107FF4F6AE1D4B93F80532002B52D01C4B9A
S315080142201C4A1D4903A812F093FA154C03A9204606
S31508014230FCF78CFA074603212046FCF7BAFB6E0009
S31508014240FBB20095013332466D212046FCF7A7FEE5
S3150801425000212046FCF7ADFB03AB32466E21204612
S31508014260FCF70DFA03212046FCF7A3FBBEE600BFC7
S315080142706891ED7CD796A9403CF889037CF4C04047
S3150801428050D30020A0A3020894000020D80F0020D4
S31508014290A8040308B0040308BC0403080000C842C4
S315080142A0D4040308E0040308EC040308F80403082B
S315080142B0DBAC2D4774D13546040503081005030800
S315080142C0FC030020B84FB94C39462046FCF73EFAA4
S315080142D06E005FFA80F8009508F1010332466D21F8
S315080142E02046FCF75CFE00212046FCF762FB03AB87
S315080142F097E8070003C31A7003AB32466E212046BE
S31508014300FCF7BDF903212046FCF753FBA84AA94946
S3150801431003A812F01DFA03AB324608F16E012046D6
S31508014320FCF7ADF962E6A44B93F91C33012B7FF434
S3150801433067AE50E1A04B93F91C33022B7FF47FAE95
S315080143409D4B93F8053243B3994B974A9B4903A86A
S3150801435012F0FEF9954C03A92046FCF7F7F9074632
S3150801436003212046FCF725FB05EB4506FBB2009524
S31508014370013332466D212046FCF711FE0021204605
S31508014380FCF717FB03AB32466E212046FCF777F99B
S3150801439003212046FCF70DFB4BE6834F834C394638
S315080143A02046FCF7D3F905EB45065FFA80F8009538
S315080143B008F1010332466D212046FCF7F0FD002184
S315080143C02046FCF7F6FA03AB97E8070003C31A7011
S315080143D003AB32466E212046FCF751F903212046EC
S315080143E0FCF7E7FA724A734903A812F0B1F903AB6D
S315080143F0324608F16E012046FCF741F919E66E4B83
S3150801440093F91C33022B7FF41AAE27E16A4BD3F8D2
S315080144108800D3F8A430C01A0028B8BF404207EE76
S31508014420900AF8EEE77A17EE900AF4F76BF85AA3B2
S31508014430D3E90023F4F7E4F9F4F7B0FB00EE100A28
S3150801444028E65D4BD3F88800D3F8A030C01A0028B7
S31508014450B8BF404207EE900AF8EEE77A17EE900ADF
S31508014460F4F750F84CA3D3E90023F4F7C9F9F4F7A4
S3150801447095FB00EE100A0DE64F4BD3F8CC00D3F8A6
S31508014480E830C01A0028B8BF404207EE900AF8EE95
S31508014490E77A17EE900AF4F735F841A3D3E9002332
S315080144A0F4F7AEF9F4F77AFB00EE100A3AE6424B56
S315080144B0D3F8CC00D3F8E430C01A0028B8BF40427C
S315080144C007EE900AF8EEE77A17EE900AF4F71AF86B
S315080144D033A3D3E90023F4F793F9F4F75FFB00EE6E
S315080144E0100A1FE6344AD2F81031D2F82C219B1A49
S315080144F0002BB8BF5B4207EE903AF8EEE77A87EEF3
S31508014500870A55E62C4AD2F81031D2F828219B1A87
S31508014510002BB8BF5B4207EE903AF8EEE77A87EED2
S31508014520870A45E6264BD3F8BC322246002148467F
S31508014530FCF7A5F80437DAF8003022464146484622
S31508014540FCF79DF801362C44A4B2032E00F0BE8078
S31508014550BA4639684846FCF7F9F8C0F164005FFACB
S3150801456080F803214846FCF724FA9BF91C33B34229
S31508014570E0D19BF89832002BD4D0009564232246CB
S3150801458000214846FCF70BFD00214846FCF711FAC5
S31508014590D0E700BFAFF300806891ED7CD796A940BC
S315080145A03CF889037CF4C040B004030850D30020CA
S315080145B0A8040308C4040308D80F0020BC04030890
S315080145C094000020012B3FF425AE434B93F8983213
S315080145D0022B7FF411AD414A414903A812F0B8F8FC
S315080145E06E00404C03AB32466E212046FCF747F875
S315080145F003A92046FCF7AAF80746DFF8EC804146EE
S315080146002046FCF7A3F8FFB2C3B200950133324640
S3150801461007F16D012046FCF7C2FC00212046FCF794
S31508014620C8F998E803000390ADF8101003AB3246B9
S3150801463007F16E012046FCF722F803212046FCF714
S31508014640B8F9D9E4244B93F89832012B3FF478AEA4
S31508014650214B93F89832022B7FF4F1AC1F4A20497B
S3150801466003A812F075F805EB45061E4C03AB324656
S315080146706E212046FCF703F803A92046FCF766F8E5
S315080146800746DFF8648041462046FCF75FF8FFB22B
S31508014690C3B200950133324607F16D012046FCF796
S315080146A07EFC00212046FCF784F998E80300039074
S315080146B0ADF8101003AB324607F16E012046FBF741
S315080146C0DEFF03212046FCF774F9B8E411B0BDEC0E
S315080146D0028BBDE8F08F00BFD80F0020B004030895
S315080146E0CC04030850D30020A80403082DE9F04F91
S315080146F091B0D14B93F9643343B1CF4B93F96433FA
S31508014700012B00F01A8111B0BDE8F08FCA4CB4F93B
S315080147104433D4F8481301FB03F6C84DC849284663
S31508014720FCF72AF801212846FCF743F9C54AA2FBFA
S315080147300632D20B48F6A04303FB1263C249A1FB1A
S315080147400303A1FB060189094FF4167000FB1161E9
S31508014750BE48A0FB0101C90800919B09BC4903A8F1
S3150801476011F0F6FF03AB36220A212846FBF787FF2D
S31508014770D4F84813B74B83FB01024FEAE17ECEEB2F
S31508014780A20202EB4200A1EBC00000EB8000400050
S3150801479083FB0063C017B04F87FB01C60E44CEEBFF
S315080147A02616C6EB061EA1EB4E0101EB8101490057
S315080147B087FB01E70F44C917C1EB27110191009641
S315080147C0C0EBA303A54903A811F0C2FF03AB3E2220
S315080147D00A212846FBF753FFA14F39462846FBF71E
S315080147E0CBFF2846FBF798FF2846FBF7A9FF95F864
S315080147F0296095F82A30F61AF6B203212846FCF7FD
S31508014800D8F8D4F8C432002211462846FBF737FFF8
S31508014810B4F94433DFF8588288FB0321DA17C2EB6F
S31508014820A10202EB8201A3EB41031BB212B28D492D
S3150801483003A811F08DFFB6B203AB32467D21284697
S31508014840FBF71DFFB4F94C33B4F9440388FB032184
S31508014850DA17C2EBA10202EB8201A3EB410388FB43
S315080148600018C117C1EBA80101EB810EA0EB4E00A0
S3150801487000B2019009B200911BB212B27A4903A89B
S3150801488011F066FF03AB72007D212846FBF7F7FEA0
S31508014890D4F84823754903A811F05AFF03AB06EB70
S315080148A046027D212846FBF7EAFE39462846FBF7EC
S315080148B063FF03212846FCF77CF804F55D74354649
S315080148C00027DFF87891DFF8ACB115E05A4BD3F839
S315080148D0BC322A4600214846FBF7D1FE0434DAF8F1
S315080148E000302A4641464846FBF7C9FE013735449A
S315080148F0ADB2032F3FF401AFA24621684846FBF744
S3150801490025FFC0F178001FFA80F803214846FCF715
S3150801491050F89BF91D33BB42E0D19BF89832002B26
S31508014920D4D0009678232A4600214846FCF737FB5F
S3150801493000214846FCF73DF8D0E7404C4849204657
S31508014940FBF71AFF2046FBF7E7FE2046FBF7F8FEC2
S3150801495094F8295094F82A30ED1AEDB2032120462D
S31508014960FCF727F8344ED6F8C43200221146204601
S31508014970FBF785FED6F88003B0F5167F38DA3C4B8F
S3150801498083FB0023C217C2EBA30202EB8203A0EB4F
S315080149904303344903A811F0DBFEADB2274C03AB40
S315080149A02A467D212046FBF76AFE2D492046FBF75C
S315080149B0E3FE03212046FBF7FCFF1F4BD3F88413C4
S315080149C02046FBF7C3FEC0F1780086B203212046D4
S315080149D0FBF7EFFF274B93F92233002B4ED0164BEB
S315080149E0D3F884332A4631461448FBF748FE8AE64B
S315080149F0204BB3F91E130144B3F920030844114AA5
S31508014A00A2FB0032D20B48F6A04303FB12030E4960
S31508014A10A1FB0343A1FB004189094FF4167404FB6A
S31508014A2011010A48A0FB0101C90800919B09124915
S31508014A3003A811F08DFEB0E79400002050D30020A2
S31508014A40D4F70208D55204E9B5814E1BCDCCCCCC9E
S31508014A50EC030308ABAAAA2A8988888810040308E4
S31508014A60A0A30208C80303083404030804040308BE
S31508014A7067666666D80F00201C0503080C4B93F879
S31508014A80983243B90B4BD3F8BC322A4600210A485F
S31508014A90FBF7F5FDA3E7009578232A460021204672
S31508014AA0FCF77DFA00212046FBF783FF97E700BF55
S31508014AB0D80F00209400002050D300202DE9F04F94
S31508014AC091B09E4D9E492846FBF756FE2846FBF7B0
S31508014AD023FE2846FBF734FE95F8294095F82A3037
S31508014AE0E41AE4B2974B93F9643343B1954B93F9BE
S31508014AF06433012B00F08F8011B0BDE8F08F0321DC
S31508014B002846FBF756FF8F4ED6F8C83200221146C3
S31508014B102846FBF7B4FD8C4FD6F88823394603A8F7
S31508014B2011F016FE1FFA84F903AB4A466921284695
S31508014B30FBF7A5FDDFF82882B8F92423394603A82F
S31508014B4011F006FE03AB4FEA490269212846FBF735
S31508014B5096FDB8F92623394603A811F0F9FD03ABEA
S31508014B6009EB490269212846FBF789FD96F98C2349
S31508014B70022A12D01346023A744903A811F0E8FD35
S31508014B8003AB4FEA890269216C48FBF778FD704F40
S31508014B904D460026DFF8C8B11BE06E4B93E80300CB
S31508014BA003908DF81010EBE7664BD3F8BC322A4612
S31508014BB000216248FBF763FD0437DAF800302A461C
S31508014BC041465E48FBF75BFD01364D44ADB2042E06
S31508014BD08CD0BA4639685948FBF7B8FDC0F164006C
S31508014BE01FFA80F803215548FBF7E3FE9BF92833A2
S31508014BF0B342E1D19BF89832002BD5D0CDF800907D
S31508014C0064232A4600214D48FCF7C9F900214B487F
S31508014C10FBF7CFFED0E7494E03213046FBF7C9FE25
S31508014C20484DD5F8C832002211463046FBF727FD14
S31508014C30D5F8A033484981FB0321DA17C2EBA10253
S31508014C4002EB8200642101FB03F1D5F8807391FB25
S31508014C50F7F10091A3EB4003404903A811F078FD51
S31508014C60A4B203AB224669213046FBF708FD3C4B4B
S31508014C7093F9293305EB8303D3F8A41303A811F099
S31508014C8067FD03AB620069213046FBF7F8FC95F92D
S31508014C908C23022A14D01346023A2C4903A811F090
S31508014CA057FD03AB04EB440269212448FBF7E7FCF3
S31508014CB02C4F25460026DFF88490DFF8A4B01CE0C7
S31508014CC0244B93E8030003908DF81010E9E71D4B78
S31508014CD0D3F8BC322A4600214846FBF7D0FC0437F4
S31508014CE0DAF800302A4641464846FBF7C8FC013641
S31508014CF02544ADB2032E3FF4FFAEBA46396848469D
S31508014D00FBF724FDC0F164001FFA80F80321484629
S31508014D10FBF74FFE9BF92A33B342E0D19BF8983251
S31508014D20002BD4D0009464232A4600214846FCF778
S31508014D3036F900214846FBF73CFED0E750D3002060
S31508014D40A0A3020894000020040403083005030800
S31508014D5024040020280503086766666640050308DB
S31508014D60D80F0020400400202DE9F0418EB0424CB6
S31508014D7042492046FBF700FD2046FBF7CDFC2046BD
S31508014D80FBF7DEFC94F8295094F82A60AD1BEEB2C5
S31508014D90B4F8008003212046FBF70BFE384BD3F805
S31508014DA0CC32002211462046FBF769FC354FD7F86D
S31508014DB0E820D7F8E430D21A334981FB0231D317F8
S31508014DC0D7F8A450D7F8A020AD1A304A82FB0502BD
S31508014DD02A44ED17C3EB2133C5EBE2222C4901A87E
S31508014DE011F0B6FCB6B201AB32460F212046FBF7ED
S31508014DF046FCD7F82C21D7F82831D21A254901A81B
S31508014E0011F0A6FC01AB72000F212046FBF737FC17
S31508014E10D7F87021D7F86C31D21A1F4901A811F0B9
S31508014E2097FC01AB06EB46020F212046FBF727FC50
S31508014E3097F89832C3B101AC184D0FCD0FC42B6842
S31508014E4023600D4C01A92046FBF780FCA8EB000066
S31508014E5000EBD07001AB3322C0F34F012046FBF7BC
S31508014E600EFC0EB0BDE8F0810D4B322211462046EC
S31508014E70FBF705FCF5E700BF50D30020A0A3020805
S31508014E8094000020D80F00206B2ECA782B8316A019
S31508014E905405030868050308780503089C050308F3
S31508014EA0880503082DE9F0439FB0AB49AB48FBF7EA
S31508014EB063FCAB4B93F882308BB9A94B93F88130DD
S31508014EC033B1A84B0822F821A448FBF7D8FB10E018
S31508014ED0A54B0822F821A148FBF7D1FB09E0A04B15
S31508014EE093F881307BB3A14B0822F8219B48FBF745
S31508014EF0C6FB9A4C9E492046FBF73EFC2046FBF72B
S31508014F000BFC2046FBF71CFC94F8292094F82A3060
S31508014F10D21AD5B2268803212046FBF74AFD954BBE
S31508014F2093F8B833022B15D0924B93F8B833012B6B
S31508014F3015D0904B93F96433B3B1012B00F06C8112
S31508014F401FB0BDE8F0838C4B0822F8218348FBF794
S31508014F5096FBCEE702212046FBF72BFDE4E701216C
S31508014F607E48FBF726FDE4E7824BD3F8D0320022D0
S31508014F7011467A48FBF783FB794B93F8C432192B10
S31508014F8041D01A2B00F02481754ED6F81833D6F87D
S31508014F90C8227A4911A811F0DBFBADB26F4C11ABEF
S31508014FA06A000F212046FBF76AFBD6F81803D6F8E4
S31508014FB0C812401A6F4BB3F9441301FB00F0704A4B
S31508014FC0A2FB0032D20B48F6A04303FB12036D493C
S31508014FD0A1FB0363A1FB006189094FF4167606FB61
S31508014FE011016948A0FB0101C90800919B0967499C
S31508014FF011A811F0ADFB11AB05EB45020F212046B7
S31508015000FBF73DFB9CE75B4B93F98C33022B14D0E2
S31508015010022B25DD524B93F82C33643B0A2B1FD800
S31508015020DFE813F053005A0062006A0072007A0042
S3150801503082008A009200C800CF00494B93F82B33AF
S31508015040013B082B0CD8DFE803F0051D242B320B96
S315080150500B0B3900474BD3F8BC1304A811F0AAFB74
S31508015060444AD2F8DC33D2F8D82304A90091484936
S3150801507011A811F06DFB11AB2A460F213748FBF732
S31508015080FEFA81E73B4BD3F8C01304A811F092FB53
S31508015090E6E7384BD3F8C41304A811F08BFBDFE716
S315080150A0344BD3F8C81304A811F084FBD8E7314B65
S315080150B0D3F8CC1304A811F07DFBD1E72D4BD3F817
S315080150C0D01304A811F076FBCAE72A4BD3F8BC1310
S315080150D004A811F06FFBC3E7264BD3F8D4232D4957
S315080150E004A811F035FBBBE7224BD3F8D4232A4990
S315080150F004A811F02DFBB3E71E4BD3F8D423274997
S3150801510004A811F025FBABE71A4BD3F8D42324499D
S3150801511004A811F01DFBA3E7164BD3F8D4232149A4
S3150801512004A811F015FB9BE7124BD3F8D4231E49AB
S3150801513004A811F00DFB93E70E4BD3F8D4231B49B2
S3150801514004A811F005FB8BE70A4BD3F8D4231849B9
S3150801515004A811F0FDFA83E72C9A020850D300201F
S31508015160D80F002000030308F80203080403030804
S31508015170A0A3020894000020FC02030838030308D0
S31508015180D55204E9B5814E1BCDCCCCCC8C04030891
S31508015190D0050308B0050308B4050308B8050308D4
S315080151A0BC050308C0050308C4050308C8050308A8
S315080151B0CC050308534BD3F8CC1304A811F0FAFA1B
S315080151C04EE7504BD3F8D01304A811F0F3FA47E78A
S315080151D04C4FD7F8E033D7F8D8234B4911A811F02B
S315080151E0B7FA4A4C11AB2A460F212046FBF747FA74
S315080151F0D7F8EC1311A811F0ABFA11A92046FBF761
S31508015200A5FA301A00EBD07011AB3322C0F34F0167
S315080152102046FBF734FAB7E63A4BD3F8DC320022DC
S3150801522011463A48FBF72BFA394B93F8C432192B36
S315080152305AD01A2B5FD0364CD4F81873D4F8C862F2
S31508015240304BD3F8F003F3F75DF90022314BF3F74E
S31508015250ADF980468946B81BF3F742F902460B4673
S3150801526040464946F3F7A2F9F3F778FC2A4AA2FB26
S315080152700032D30B48F6A04101FB13032749A1FBD2
S31508015280030188094FF4167E0EFB1030244BA3FB4D
S3150801529000E3DB0803EB830EA0EB4E0003900293B9
S315080152A089090191D20B00923B4632461D4911A844
S315080152B011F04EFAADB211AB6A000F211348FBF794
S315080152C0DEF994F92933012B7FF43AAEB4F82E238B
S315080152D0154911A811F03CFA11AB05EB45020F214E
S315080152E00A48FBF7CCF92BE6104B2A460F2107484B
S315080152F0FBF7C5F99FE70E4B2A460F210348FBF733
S31508015300BEF998E7940000209C03030850D30020B7
S31508015310D80F002000002440D55204E9B5814E1B60
S31508015320CDCCCCCCD8050308F80503081803030827
S31508015330640403082DE9F04F83B0314C3149204606
S31508015340FBF71AFA2046FBF7E7F92046FBF7F8F9C7
S3150801535094F8299094F82A30A9EB03095FFA89F998
S3150801536003212046FBF725FB274DD5F8D832002225
S3150801537011462046FBF783F905F57D751FFA89F96C
S315080153804C460026DFF87880DFF880B014E01E4B23
S31508015390D3F8BC32224600214046FBF770F90435A2
S315080153A0DAF80030224639464046FBF768F90136F5
S315080153B04C44A4B2032E20D0AA4629684046FBF7DE
S315080153C0C5F9C0F1640087B203214046FBF7F1FA3B
S315080153D09BF93033B342E2D19BF89832002BD6D0F1
S315080153E0CDF800906423224600214046FBF7D7FDFD
S315080153F000214046FBF7DDFAD1E703B0BDE8F08F9F
S3150801540050D30020A0A3020894000020D80F002042
S315080154102DE9F04F2DED048B91B0894B93F9993213
S31508015420012B40F31381042B40F34E82082B40F3E2
S31508015430E08211B0BDEC048BBDE8F08F804BD3F848
S315080154407802D3F88830C01A0028B8BF404207EE60
S31508015450900AF8EEE77A17EE900AF3F753F874A371
S31508015460D3E90023F3F7CCF9F3F798FB08EE900A92
S3150801547054E1734BD3F87C02D3F8CC30C01A002818
S31508015480B8BF404207EE900AF8EEE77A17EE900A9F
S31508015490F3F738F868A3D3E90023F3F7B1F9F3F77B
S315080154A07DFB08EE100A7FE19BF8983243B9654BFC
S315080154B0D3F8BC322A4600214846FBF7E0F8D1E189
S315080154C00094AA232A4600214846FBF768FD0021D5
S315080154D04846FBF76EFAC5E15A4BD3F8BC322A4661
S315080154E000214846FBF7CBF80436DAF800302A469D
S315080154F041464846FBF7C3F801372544ADB2052FA7
S3150801550097D0B24631684846FBF720F9C0F18200C8
S315080155101FFA80F803214846FBF74BFA9BF99932A3
S31508015520BB42E1D19BF89832002BD5D00094822357
S315080155302A4600214846FBF732FD00214846FBF77B
S3150801554038FAD1E73F4BD3F8BC32324600214846F8
S31508015550FBF795F80434DAF80030324641464846F6
S31508015560FBF78DF801372E44B6B2082F20D0A24694
S3150801557021684846FBF7EAF8C0F182001FFA80F86D
S3150801558003214846FBF715FA9BF99932BB42E1D14B
S315080155909BF89832002BD5D00095822332460021FC
S315080155A04846FBF7FCFC00214846FBF702FAD1E71F
S315080155B0234B93F99932082B0DD0234C032120460E
S315080155C0FBF7F7F91F4BD3F82434AA006E212046BE
S315080155D0FBF755F82DE71A4B93F89832ABB1AE00A5
S315080155E0194C0095FF23324600212046FBF7D7FCCC
S315080155F000212046FBF7DDF9124BD3F82434324655
S315080156006E212046FBF73BF813E7AD000D4E0E4C15
S31508015610D6F8BC322A4600212046FBF730F8D6F8E0
S3150801562024342A466E212046FBF729F801E700BFF4
S315080156306891ED7CD796A9403CF889037CF4C04073
S31508015640D80F00209400002050D30020904D914996
S315080156502846FBF791F82846FBF75EF82846FBF73C
S315080156606FF895F8294095F82A30E41AE4B203212F
S315080156702846FBF79EF9884AD2F86C34D2F8682492
S31508015680864903A811F064F803AB0022114628469F
S31508015690FAF7F5FF824BD3F878321BB9804BD3F86A
S315080156A07C322BB17F4B2246B4217948FAF7E7FFC2
S315080156B07B4BD3F880321BB9794BD3F884322BB1A3
S315080156C0784B6200B4217248FAF7D9FF0121704874
S315080156D0FBF76FF9724B93F898322BB1704B93F92C
S315080156E09932012B3FF4AAAE6D4BD3F87802D3F861
S315080156F08032C01A0028B8BF404207EE900AF8EE79
S31508015700E77A17EE900AF2F7FDFE5DA3D3E90023C7
S31508015710F3F776F8F3F742FA08EE900ABDEEE88A4F
S31508015720F8EEC87A78EEE77A9FED5F0A27EE800AE7
S3150801573010F0B0FBFDEEC07A17EE903A092B18EE81
S31508015740102ACCBF59495A4903A811F001F8A4B245
S3150801575004EB440503AB2A4600214D48FAF78FFFAF
S315080157604F4B93F898322BB14D4B93F99932012B44
S315080157703FF47FAE4A4BD3F87C02D3F88432C01A81
S315080157800028B8BF404207EE900AF8EEE77A17EE0E
S31508015790900AF2F7B7FE3CA3D3E90023F3F730F8F2
S315080157A0F3F7FCF908EE100ABDEEC89AF8EEC97AC5
S315080157B078EE677A9FED3C0A27EE800A10F06AFBBD
S315080157C0FDEEC07A17EE903A092B19EE102ACCBFD6
S315080157D03849394903A810F0BBFF03AB2A467D2196
S315080157E02B48FAF74CFF88EE880ABDEEC08AF8EE18
S315080157F0C87A30EE670ADFED2C7A20EE270A10F018
S3150801580049FBFDEEC07A17EE903A092B18EE102ADD
S31508015810CCBF2A492A4903A810F09AFF1C4D03ABAD
S31508015820A20032212846FAF72AFF03212846FBF768
S31508015830C0F8244F25460026DFF85490DFF860B0FB
S31508015840BA4639684846FAF781FFC0F1AA001FFA35
S3150801585080F803214846FBF7ACF89BF99932B34225
S315080158603FF422AE0437DAF800302A464146484664
S31508015870FAF705FF01362544ADB2022EE0D1D8E587
S315080158806891ED7CD796A9403CF889037CF4C04021
S3150801589050D30020A0A3020894000020980603080C
S315080158A0D80F00200C0603080000C842100603089A
S315080158B020060308300603084006030854060308B1
S315080158C068060308980400207F4D80492846FAF7A0
S315080158D053FF2846FAF720FF2846FAF731FF95F8CD
S315080158E0294095F82A30E41AE4B203212846FBF741
S315080158F060F8774ED6F87034D6F86824754903A847
S3150801590010F026FF03AB002211462846FAF7B7FE28
S31508015910714B327D714903A810F01AFFA4B203AB8B
S31508015920224687212846FAF7AAFE6D4BD3F89C3200
S315080159301BB96B4BD3F8A0322BB16A4B6200872196
S315080159406148FAF79CFE664BD3F8A4321BB9644B3F
S31508015950D3F8A83233B1634B04EB440287215A4882
S31508015960FAF78DFEFDF7C0FA574D5F492846FAF753
S3150801597003FF01212846FBF71CF82846FAF7CCFE57
S315080159802846FAF7DDFE564FD7F8AC32D7F8B022DB
S31508015990564903A810F0DCFE03ABA20032212846C3
S315080159A0FAF76DFE4A4ED7F8B432D6F85424504960
S315080159B003A810F0CDFE03AB04EB8402322128467E
S315080159C0FAF75DFE41492846FAF7D6FE2846FAF760
S315080159D0A3FE2846FAF7B4FE03212846FAF7E9FF9B
S315080159E006F20C4625460227DFF8DC90DFF8F0B010
S315080159F087E5354E35493046FAF7BEFE3046FAF7A1
S31508015A008BFE3046FAF79CFE96F8295096F82A300E
S31508015A10ED1AEDB203213046FAF7CBFF2C4CD4F838
S31508015A207434D4F86824334903A810F091FE03AB03
S31508015A30002211463046FAF722FEB4F94C332E49B4
S31508015A4081FB0321DA17C2EBA10202EB8201A3EB68
S31508015A5041031BB212B2294903A810F079FEADB26F
S31508015A6003AB2A4687213046FAF709FE1C4B93F900
S31508015A70C03204EB8303D3F8781403A810F068FE48
S31508015A8003AB6A0087213046FAF7F9FD94F9153018
S31508015A9004EB8303D3F8801403A810F059FE03AB73
S31508015AA005EB450287213046FAF7E9FD0321304621
S31508015AB0FAF77FFF04F583642E460527DFF8089079
S31508015AC0DFF81CB053E500BF50D30020A0A302089D
S31508015AD094000020A0060308A8060308680903081D
S31508015AE0D80F00200C060308D4F702087C06030821
S31508015AF090060308AC06030867666666C8030308CA
S31508015B002DE9F04F91B0694C69492046FAF734FE00
S31508015B102046FAF701FE2046FAF712FE94F82950B4
S31508015B2094F82A30ED1AEDB203212046FAF741FF1F
S31508015B30604ED6F8E432002211462046FAF79FFD58
S31508015B4096F99034002B47D1D6F8941403A810F08F
S31508015B5031FEADB203AB2A4641215448FAF78FFD0F
S31508015B60544B93F99134002B42D1524BD3F89414E8
S31508015B7003A810F01FFE03AB6A0041214B48FAF750
S31508015B807EFD4C4B93F99234002B3DD1494BD3F80A
S31508015B90941403A810F00EFE03AB05EB4502412150
S31508015BA04248FAF76CFD434B93F99334002B37D1EE
S31508015BB0404BD3F8941403A810F0FCFD03ABAA00DC
S31508015BC041213A48FAF75BFD3B4F2C460026DFF8A0
S31508015BD0DC90DFF8ECB044E0364A02EB8303D3F8F5
S31508015BE0943492F98C23354903A810F0B1FDB0E736
S31508015BF0304A02EB8303D3F8943492F98C232F4964
S31508015C0003A810F0A5FDB6E72A4A02EB8303D3F8E9
S31508015C10943492F98C23294903A810F099FDBBE71E
S31508015C20244A02EB8303D3F8943492F98C2323494B
S31508015C3003A810F08DFDC1E71E4BD3F8B0342246F8
S31508015C4000214846FAF71BFD0437DAF800302246E8
S31508015C5041464846FAF713FD01362C44A4B2042EF0
S31508015C6020D0BA4639684846FAF770FDC0F13C00BB
S31508015C701FFA80F803214846FAF79BFE9BF9313350
S31508015C80B342E1D19BF89832002BD5D000953C233D
S31508015C90224600214846FBF782F900214846FAF7D1
S31508015CA088FED1E711B0BDE8F08F00BF50D30020C0
S31508015CB0A0A30208940000203405002068090308FF
S31508015CC0D80F00202DE9F04F91B06E4C6E49204651
S31508015CD0FAF752FD2046FAF733FD03212046FAF773
S31508015CE068FE6A4B93F89832B3B3664C6849204606
S31508015CF0FAF742FD2046FAF70FFD2046FAF720FD8E
S31508015D0003212046FAF755FE624BD3F8E832002202
S31508015D1011462046FAF7B3FC5C4B93F89832A3B3C5
S31508015D205A4B93F89832012B42D05A4B93F98C333C
S31508015D30C3EB8377C3EB8707F6375A1E97FBF2F750
S31508015D40BFB2002B40F39B8000252C464D4EDFF851
S31508015D503C814FF0100957E04F4B2D220521204673
S31508015D60FAF78DFC4D4B2D220F212046FAF787FCB9
S31508015D704B4B392205212046FAF781FC494B39223A
S31508015D8064212046FAF77BFCAFE7474B2822182106
S31508015D902046FAF774FC454B34220F212046FAF7C0
S31508015DA06EFC434B342270212046FAF768FCB7E7AC
S31508015DB0404B282218213348FAF761FCB5E714FB52
S31508015DC007F105310E2300930A230F2289B23046C3
S31508015DD0FBF7E5F800213046FAF7EBFD6A1C364970
S31508015DE003A810F0B5FC14FB07F1063103AB4A46CC
S31508015DF089B23046FAF743FC0134E4B22546254B0D
S31508015E0093F98C339C423ADA03213046FAF7D1FDED
S31508015E1098F93233AB42E1D198F89832012BCED0BA
S31508015E20022B0DD0002BD9D114FB07F105310E2316
S31508015E3000930A230F2289B23046FBF76CF8CDE7A7
S31508015E4014FB07FA1FFA8AFA0AF105014FF00E0B3D
S31508015E50CDF800B00A230F2289B23046FBF79FF826
S31508015E600AF10401CDF800900C235A4689B230464E
S31508015E70FBF751F800213046FAF79BFDAEE711B062
S31508015E80BDE8F08F50D300202C9A0208D80F0020C5
S31508015E90A0A3020894000020B4060308B806030864
S31508015EA0EC090308BC060308C0060308E006030854
S31508015EB0E8060308F406030834070308000000008F
S31508015EC02DE9F04F9BB0D24DD24C29462046FAF720
S31508015ED053FC2046FAF727FC2046FAF777FD2046B9
S31508015EE0FAF72EFC29462046FAF746FCCA4D05F56F
S31508015EF0077600213046F4F7BEFE0246C7490DA8CB
S31508015F0010F026FC0DAB002211462046FAF7B7FB26
S31508015F1001213046F4F7AFFE0246C1490DA810F03B
S31508015F2017FC0DAB002269212046FAF7A8FB0221CE
S31508015F303046F4F7A0FE0246BA490DA810F008FC4F
S31508015F400DAB0A2200212046FAF799FB03213046B8
S31508015F50F4F791FE0246B4490DA810F0F9FB0DAB12
S31508015F600A2269212046FAF78AFB08213046F4F706
S31508015F7079FE0246AD490DA810F0EAFB0DAB1422D5
S31508015F8000212046FAF77BFB09213046F4F76AFE21
S31508015F900246A7490DA810F0DBFB0DAB14226921B7
S31508015FA02046FAF76CFBB5F9343200EE903AB5F9AA
S31508015FB0363200EE103AF8EEE00AB8EEC00A0FF0F3
S31508015FC0DBFF10EE100AF2F79DFA8DA3D3E9002341
S31508015FD0F2F73AF98CA3D3E90023F2F7E7FAF2F7D5
S31508015FE0DDFDF2F78FFA0022924BF2F72DF9F2F75F
S31508015FF08DFD024690490DA810F0AAFB0DAB1E2295
S3150801600000212046FAF73BFBB5F9343200EE903A07
S31508016010B5F9323200EE103AF8EEE00AB8EEC00AE7
S315080160200FF0AAFF10EE100AF2F76CFA74A3D3E97F
S315080160300023F2F709F974A3D3E90023F2F7B6FAB4
S31508016040F2F7ACFDF2F75EFA00227A4BF2F7FCF8AA
S31508016050F2F75CFD024679490DA810F079FB0DAB04
S315080160601E2246212046FAF70AFB754E4FF40041D7
S315080160703046F7F743F909904FF480413046F7F770
S315080160803DF90A904FF400513046F7F737F90B906E
S315080160904FF480513046F7F731F907464FF400615E
S315080160A03046F7F72BF980464FF480613046F7F70B
S315080160B025F981464FF400713046F7F71FF98246F4
S315080160C04FF480713046F7F719F983468021304637
S315080160D0F7F714F90690CDF814B0CDF810A0CDF85D
S315080160E00C90CDF8088001970B9900910A9B099AA3
S315080160F054490DA810F02CFB0DAB1E228C2120460D
S31508016100FAF7BDFAB5F8443295F8431295F84422E0
S3150801611002F00F02C3F30B1341EA02224A490DA802
S3150801612010F016FB0DAB282200212046FAF7A7FA34
S3150801613095F8432295F8443203F00F0342EA032304
S31508016140FF2B00F38F80FF2185F8641285F86532ED
S31508016150002385F86632012385F869322E4CB4F896
S31508016160483294F8471294F8482202F00F02C3F312
S315080161700B1341EA022235490DA810F0E9FA254D1B
S315080161800DAB282278212846FAF779FA94F80522E0
S315080161902F490DA810F0DCFA0DAB32220021284652
S315080161A0FAF76DFA94F83D2202F00F0229490DA873
S315080161B010F0CEFA0DAB32224B212846FAF75FFAD8
S315080161C0D4F83423244BA3FB02135B09642101FB96
S315080161D01323092B2049A1FB02124FEA521294BF3D
S315080161E01E491F490DA810F0B3FA0DAB3222AF2193
S315080161F00848FAF744FA1BB0BDE8F08FAFF3008000
S31508016200182D4454FB210940F8C1631ADCA54C40FA
S31508016210D4F7020850D30020D80F0020100703082E
S3150801622024070308380703084C070308600703080F
S31508016230700703080000E03F840703089007030876
S31508016240001002409C070308B8070308C80703089B
S31508016250D8070308E80703081F85EB51F807030861
S3150801626008080308B3F5FF7F0EDC2C4AC3F1FE03C9
S3150801627082F86432FF2382F86532002382F8663297
S31508016280012382F8693269E740F2FD2293420DDC67
S31508016290224A002182F86412FF2182F8651202332C
S315080162A082F86632012382F8693257E7B3F57F7FB0
S315080162B00EDC1A4A002182F86412C3F1FC0382F843
S315080162C06532FF2382F86632012382F8693245E78F
S315080162D040F2FB4293420DDC104A043382F86432E1
S315080162E0002382F86532FF2382F86632012382F899
S315080162F0693233E740F2FA5293423FF72FAF074A22
S31508016300FF2182F86412002182F86512C3F1FA03AB
S3150801631082F86632012382F869321FE7D80F002016
S3150801632070B590B05F4D604C29462046FAF724FABD
S315080163302046FAF7F8F92046FAF748FB2046FAF715
S31508016340FFF929462046FAF717FA584DD5F8882055
S31508016350574903A810F0FCF903AB00220621204691
S31508016360FAF78DF9534ED5F89420314603A810F063
S31508016370EFF903AB00225A212046FAF780F9D5F83E
S31508016380CC204D4903A810F0E3F903AB0A220021FA
S315080163902046FAF774F9D5F8D820314603A810F043
S315080163A0D7F903AB0A225A212046FAF768F9D5F834
S315080163B01021424903A810F0CBF903AB14220C2192
S315080163C02046FAF75CF9D5F81C21314603A810F0E6
S315080163D0BFF903AB14225A212046FAF750F9D5F82A
S315080163E05421374903A810F0B3F903AB1E220C2137
S315080163F02046FAF744F9D5F86021314603A810F08A
S31508016400A7F903AB1E225A212046FAF738F995F85F
S31508016410393395F8382395F83B13019195F83A13D2
S315080164200091284903A810F093F903AB282200210B
S315080164302046FAF724F995F80522234903A810F00E
S3150801644087F903AB322200212046FAF718F995F8A5
S315080164503D2202F00F021D4903A810F079F903AB9A
S3150801646032224B212046FAF70AF9D5F83423184B7C
S31508016470A3FB02135B09642101FB1323092B1449AE
S31508016480A1FB02124FEA521294BF1249124903A8FC
S3150801649010F05EF903AB3222AF210348FAF7EFF8A1
S315080164A010B070BDD4F7020850D30020D80F0020D1
S315080164B0140803081C080308200803082C08030805
S315080164C0340803083C080308D8070308E807030843
S315080164D01F85EB51F80703080808030800B583B0C0
S315080164E0054B01932D2300930A4601460348F9F704
S315080164F033FD03B05DF804FB5405002050D300209A
S315080165001B4B93F86E320B2B18D00D2B02D00A2B8E
S3150801651027D07047164B93F8CC3201335BB2032B65
S3150801652008DD0022124B83F8CC220122114B83F895
S31508016530CE2570470E4A82F8CC32F6E70C4B93F912
S31508016540CC321BB904220A4B83F8CC22084A92F8AA
S31508016550CC32013B82F8CC320122064B83F8CE2598
S315080165607047034A92F8CC32013382F86E32D0E78B
S31508016570D80F0020940000201D4B93F86E320A3B79
S31508016580032B34D8DFE803F02D162802184B93F8AD
S31508016590CD3201335BB2022B08DD0022144B83F89E
S315080165A0CD220122134B83F8CE257047104A82F873
S315080165B0CD32F6E70E4B93F9CD3243B907220C4B90
S315080165C083F86E2201220B4B83F8CE257047013BD7
S315080165D0074A82F8CD32F5E70722054B83F86E2282
S315080165E07047034A92F8CD32013382F86E3270470A
S315080165F0D80F002094000020F8B5B64B93F89832CE
S31508016600002B00F023810122B34B83F8CE25B14B31
S3150801661093F86E32083B0A2B10D8DFE813F00B000B
S315080166200F0043007100F6008A00DC000F00A40089
S315080166300F00C0000022A74B83F89822A64B03EB54
S315080166404003B3F99C32042B05DCA34B03EB40034F
S315080166500522A3F89C22A04B03EB4003B3F9A4320D
S31508016660002BC0F2EC809C4D05EB4005B5F99C0268
S31508016670F1F736FF0022994BF1F798FF06460F46C8
S31508016680B5F9A402F1F72CFF32463B46F2F71EFA9A
S31508016690002800F01D8130463946F2F737FAA5F889
S315080166A0A402F8BD8B4B002283F8982201218A4A5D
S315080166B082F8CF1593F910339BB9864B03EB001279
S315080166C0D3F88810C2F8D012D3F8CC10C2F8D41275
S315080166D0D3F81011C2F8D812D3F85431C2F8DC3203
S315080166E0ACE7032BAAD17B4B03EB00130022C3F8BB
S315080166F0D022C3F8D422C3F8D822C3F8DC229DE7F6
S31508016700744B93F91033012B0AD0022B96D1724B95
S3150801671003EB4003B3F8A4220132A3F8A4228DE7C0
S315080167206D4B03EB4003B3F89C220132A3F89C227C
S3150801673084E7684B93F91033012B0BD0022B7FF4B6
S315080167407DAF654B03EB4003B3F8A422013AA3F8E6
S31508016750A42273E7604B03EB4003B3F89C22013A8A
S31508016760A3F89C226AE75B4B93F91033012B0CD0F3
S31508016770022B7FF463AF584B03EB40021B7BB2F845
S31508016780A4120B44A2F8A43258E7534B03EB400278
S315080167901B7BB2F89C120B44A2F89C324EE74D4B78
S315080167A093F91033012B0CD0022B7FF447AF4A4BD8
S315080167B003EB4002197BB2F8A4325B1AA2F8A432A1
S315080167C03CE7454B03EB4002197BB2F89C325B1A56
S315080167D0A2F89C3232E73F4B93F91033012B0BD0C9
S315080167E0022B7FF42BAF3C4B03EB4003B3F8A422F7
S315080167F00532A3F8A42221E7374B03EB4003B3F88C
S315080168009C220532A3F89C2218E7324B93F91033E0
S31508016810012B0BD0022B7FF411AF2F4B03EB400357
S31508016820B3F8A422053AA3F8A42207E72A4B03EBF7
S315080168304003B3F89C22053AA3F89C22FEE6264BB0
S3150801684003EB40030022A3F8A4220CE70122224B02
S3150801685083F8CE251F4B93F86E320A3B042B37D8A3
S31508016860DFE803F0031B2A0B2F000123194A82F8DC
S315080168709832194A82F8CF35F8BD164B93F810337A
S3150801688001335BB2032B03DC124A82F81033F8BDDD
S315080168900322104B83F81023F8BD0E4B93F91033DE
S315080168A01BB901220B4B83F810230A4A92F81033BD
S315080168B0013B82F81033F8BD0722064B83F86E2296
S315080168C0F8BD044B062283F86E22002283F81023B2
S315080168D0F8BD00BFD80F0020940000200000E03F5B
S315080168E0A64B93F8C4322D2B16D0A54B93F9083332
S315080168F0032B40F333810322A14B83F80823A04BD2
S31508016900D3F8FC32B3F5346F40F330814FF4346277
S315080169109B4BC3F8FC227047984B93F89832002B8F
S3150801692000F0C580012BE0D1944B93F86E320A3BF7
S31508016930082BDAD801A252F823F000BF61690108D1
S31508016940736901087B6A0108A7690108476A010892
S31508016950EB680108DB690108EB680108116A01089F
S315080169600022864B83F898220122854B83F8CE258F
S31508016970BBE7824B93F91433012B06D0022B0BD0BC
S3150801698001227F4B83F8CE25AFE77D4A92F808337B
S31508016990013382F80833F3E7794AD2F8FC32013336
S315080169A0C2F8FC32ECE7754B93F91433012B06D088
S315080169B0022B0BD00122724B83F8CE2595E7704A3C
S315080169C092F80833013B82F80833F3E76C4AD2F8A8
S315080169D0FC32013BC2F8FC32ECE7684B93F91433FD
S315080169E0012B06D0022B0BD00122654B83F8CE254D
S315080169F07BE7634A92F80833013382F80833F3E7F1
S31508016A005F4B1A7BD3F8FC120A44C3F8FC22EBE766
S31508016A105A4B93F91433012B06D0022B0BD00122C2
S31508016A20574B83F8CE2560E7554A92F80833013B60
S31508016A3082F80833F3E7524B197BD3F8FC22521A32
S31508016A40C3F8FC22EBE74D4B93F91433012B06D01F
S31508016A50022B0BD001224A4B83F8CE2545E7484A3B
S31508016A6092F80833013382F80833F3E7444AD2F837
S31508016A70FC326433C2F8FC32ECE7404B93F9143329
S31508016A80012B06D0022B0BD001223D4B83F8CE25D4
S31508016A902BE73B4A92F80833013B82F80833F3E7C0
S31508016AA0374AD2F8FC32643BC2F8FC32ECE7334B86
S31508016AB093F86E320A3B042B3FF617AFDFE803F073
S31508016AC0032E411A46002D4B93F9143353B92B4B18
S31508016AD00022C3F83C23A3F8122383F8402301229A
S31508016AE083F86E220123254A82F89832244A82F8CD
S31508016AF0CE35FAE6214B93F8143301335BB2022BF8
S31508016B0007DC1E4A82F8143301221D4B83F8CE2571
S31508016B10EBE60222194B83F81423F5E7174B93F991
S31508016B2014331BB90122154B83F81423134A92F81F
S31508016B301433013B82F814330122114B83F8CE2515
S31508016B40D3E607220D4B83F86E22CEE60B4B0622BF
S31508016B5083F86E22002283F81523C6E6002B3FF739
S31508016B60CEAE0022064B83F80823C8E6632B03DC66
S31508016B706422034BC3F8FC22704700BFD80F0020DC
S31508016B8094000020664B93F8C4322E2B0AD0654B2D
S31508016B9093F938330F2B40F3BB800F22614B83F8EF
S31508016BA0382370475E4B93F89832002B59D0012B46
S31508016BB0EDD15B4B93F86E320A3B042BE7D8DFE83D
S31508016BC003F0030C3F1D2E000022554B83F8982233
S31508016BD00122544B83F8CE25D9E7514B93F9153346
S31508016BE0012B04D001224F4B83F8CE25CFE74D4A1E
S31508016BF092F83833013382F83833F3E7484B93F97F
S31508016C001533012B04D00122464B83F8CE25BEE766
S31508016C10444A92F83833013B82F83833F3E7404B5C
S31508016C2093F91533012B04D001223E4B83F8CE2567
S31508016C30ADE73C4A92F83833013382F83833F3E743
S31508016C40374B93F91533012B04D00122354B83F8C1
S31508016C50CE259CE7334A92F83833013B82F838331C
S31508016C60F3E72F4B93F86E320A3B042B8FD8DFE8F4
S31508016C7003F0032C3F184700294B93F9153343B901
S31508016C80274B0022A3F8122383F84023012283F815
S31508016C906E220123224A82F89832224A82F8CE3598
S31508016CA075E71F4B93F8153301335BB2012B08DDEA
S31508016CB001221B4B83F8152301221A4B83F8CE2593
S31508016CC065E7174A82F81533F6E7154B93F9153335
S31508016CD01BB90122124B83F81523114A92F8153371
S31508016CE0013B82F8153301220E4B83F8CE254EE778
S31508016CF00B4B072283F86E22002283F8142346E7FA
S31508016D00074B062283F86E22002283F816233EE7F4
S31508016D10002B03DC0022034B83F83823704700BF9E
S31508016D20D80F002094000020B34B93F96433002B4D
S31508016D3040F06B81B14B93F89832002B00F0EA8052
S31508016D40012B40F0F080AD4B93F86E320A3B082BCD
S31508016D5000F2E980DFE813F009001200BD005700D0
S31508016D609C00E7003300E70078000022A34B83F874
S31508016D7098220122A04B83F8CE25D4E09F4B93F9A4
S31508016D801D3353B99C4AB2F844330133A2F844334C
S31508016D900122994B83F8CE25C5E0012B06D1964AE7
S31508016DA0B2F84C330133A2F84C33F1E7022BEFD199
S31508016DB0914AD2F848330133C2F84833E8E78F4B92
S31508016DC093F91D335BB98C4B1A7BB3F844130A4408
S31508016DD0A3F844230122884B83F8CE25A3E0012B8F
S31508016DE007D1854B1A7BB3F84C130A44A3F84C23F5
S31508016DF0F0E7022BEED1804B1A7BD3F848130A44ED
S31508016E00C3F84823E6E77D4B93F91D3353B97A4A0C
S31508016E10B2F84433013BA2F844330122764B83F896
S31508016E20CE2580E0012B06D1734AB2F84C33013BDB
S31508016E30A2F84C33F1E7022BEFD16F4AD2F8483367
S31508016E40013BC2F84833E8E76C4B93F91D335BB94C
S31508016E50694B197BB3F84423521AA3F84423012238
S31508016E60654B83F8CE255EE0012B07D1624B197B72
S31508016E70B3F84C23521AA3F84C23F0E7022BEED1B0
S31508016E805D4B197BD3F84823521AC3F84823E6E722
S31508016E905A4B93F91D3353B9574AB2F8443314334D
S31508016EA0A2F844330122544B83F8CE253BE0012B4B
S31508016EB006D1514AB2F84C331433A2F84C33F1E7F0
S31508016EC0022BEFD14C4AD2F848331433C2F848336F
S31508016ED0E8E74A4B93F91D3353B9474AB2F84433A5
S31508016EE0143BA2F844330122434B83F8CE251AE01A
S31508016EF0012B06D1404AB2F84C33143BA2F84C3365
S31508016F00F1E7022BEFD13C4AD2F84833143BC2F8D9
S31508016F104833E8E7394B93F86E320B2B41D00D2BEA
S31508016F2025D00A2B56D0344BB3F94433052B03DC51
S31508016F300622314BA3F844232F4BD3F84833132B9E
S31508016F4050DC14222C4BC3F848232B4AB2F944339C
S31508016F50B2F94C131A1F914203DD1346264AA2F8C9
S31508016F604C33254BB3F94C33012B49DD7047234B81
S31508016F7093F81D3301335BB2022B07DC1F4A82F8F3
S31508016F801D3301221C4B83F8CE25CCE71B4B03226C
S31508016F9083F81D23002283F82823062283F86E220C
S31508016FA0EFE7164B93F91D334BB9144B012283F8BE
S31508016FB01D23022283F81C23072283F86E220F4A17
S31508016FC092F81D33013B82F81D3301220A4B83F8DF
S31508016FD0CE25A8E70123094A82F89832064A82F89B
S31508016FE0CE35A0E7B3F5346FAFDD4FF43462024B0B
S31508016FF0C3F84823A9E700BF94000020D80F002052
S315080170000222B34BA3F84C237047012BAED1D0B55E
S31508017010B04B93F89832002B00F09280012B40F088
S315080170209A80AC4B93F86E320A3B082B00F2938098
S31508017030DFE803F0050E773A689122914F000022A6
S31508017040A44B83F898220122A14B83F8CE2582E02E
S31508017050A04B93F9223353B99D4BD3F88033B3F53B
S31508017060167FACBF0A330133994AC2F8803301222D
S31508017070974B83F8CE256EE0964B93F9223373B975
S31508017080934BD3F88033B3F5167F91490A7BA6BF94
S3150801709002EB820203EB42039B18C1F880330122FB
S315080170A08B4B83F8CE2556E08A4B93F922335BB98D
S315080170B0874BD3F88033B3F5167FACBF053B03F195
S315080170C0FF33834AC2F880330122814B83F8CE25E8
S315080170D041E07F4BD3F88033B3F5167F0CDB7C494F
S315080170E00A7B6FF0090000FB0233C1F880330122E5
S315080170F0774B83F8CE252EE0754A117B5B1AC2F8C9
S315080171008033F4E7734B93F922332BB9704AD2F8DB
S3150801711080331433C2F8803301226D4B83F8CE25B0
S3150801712019E06C4B93F922332BB9694AD2F88033AB
S31508017130143BC2F880330122654B83F8CE250AE059
S31508017140644B93F86E320B2B00F085800D2B68D0BB
S315080171500A2B00F099805E4BD3F880330E2B00F38F
S315080171609B800F225A4BC3F880235A4BD3EDD17A11
S31508017170B2EE067A67EE877AB2EE0E7AF4EEC77A3F
S31508017180F1EE10FA15DDFDEEE77A514BC3EDE07A23
S315080171904F4BD3F88003F1F7A3F949A3D3E90023A9
S315080171A0F1F794FC002800F099804B4A484BC3F844
S315080171B08023484BB3F91E33002BC0F2A380B3F5E5
S315080171C0167F04DD4FF41672424BA3F81E23414B7A
S315080171D0B3F92033002BC0F29A80B3F5167F04DD8C
S315080171E04FF416723B4BA3F82023394CD4F880038D
S315080171F0F1F776F934A3D3E90023F1F7D7F906466F
S315080172000F46D4F8A003F1F76BF932463B46F1F77E
S315080172103FFC28B130463946F1F778FCC4F8A0039B
S31508017220D0BD2C4B93F8223301335BB2002B0EDD14
S31508017230284B012283F82223002283F82A230622D7
S3150801724083F86E220122224B83F8CE2583E7214A51
S3150801725082F82233F6E71F4B93F922334BB91D4BBC
S31508017260012283F82223022283F81C23072283F8AA
S315080172706E22184A92F82233013B82F82233012200
S31508017280134B83F8CE2566E70123124A82F8983212
S315080172900F4A82F8CE355EE70E4AD2EDD17AB2EEC2
S315080172A0067A67EE877A07EE103AB8EEC77AB4EE31
S315080172B0E77AF1EE10FA7FF56BAF64E7AFF300807A
S315080172C000000000005E1A41BA490C022B87863F6E
S315080172D094000020D80F0020809706000E4BD3F8A3
S315080172E08033B3F5167FFFF664AF0A2193FBF1F2FB
S315080172F001FB1232002A3FF45CAF9B1A064AC2F818
S31508017300803356E70022054BA3F81E235FE70022C8
S31508017310024BA3F8202368E794000020D80F002029
S31508017320514B93F89832002B3ED0012B45D14E4B49
S3150801733093F86E320A3B042B3FD8DFE803F0031AB1
S3150801734023112C00484B002283F898220121474A31
S3150801735082F8CE1593F830230A4483F86E227047D3
S315080173600022414B83F898220122404B83F8CE250F
S31508017370704700223C4B83F8982201223B4B83F845
S31508017380CE2570470022384B83F898220122374BC5
S3150801739083F8CE2570470022334B83F898220122C1
S315080173A0324B83F8CE2570472F4B93F86E320B2B51
S315080173B032D00D2B44D00A2B00D070472A4B01221C
S315080173C083F8982293F9303393420AD0022B03D1DA
S315080173D00122254BC3F848230122244B83F8CE25E5
S315080173E07047214BD3F8483393420BD0022B0ED06A
S315080173F01D4B93F92933012BEED101221A4BC3F800
S315080174004823E9E70222184BC3F84823F0E701228B
S31508017410154BC3F84823EBE7134B93F83033013B7D
S315080174205BB2002B07DB104A82F8303301220F4B7F
S3150801743083F8CE25704700220B4B83F83023F5E7F6
S31508017440094B93F8303301335BB2022B07DC064A4A
S3150801745082F830330122054B83F8CE25ADE70222A7
S31508017460014B83F83023F5E7D80F0020940000205C
S31508017470F0B58FB044494548F9F77EF9444B93F87E
S3150801748082308BB9424B93F8813033B1414B082294
S31508017490F8213E48F9F7F3F811E03F4B0822F821A5
S315080174A03A48F9F7ECF80AE0394B93F88130002BA2
S315080174B040D03A4B0822F8213448F9F7E0F8334C22
S315080174C037492046F9F758F92046F9F725F92046AC
S315080174D0F9F736F994F8295094F82A30ED1AEDB2ED
S315080174E0268803212046F9F764FA2E4B0022114615
S315080174F02046F9F7C4F8264B93F8C4323E2B20D020
S31508017500422B1ED0224B93F8C4323F2B34D0432B47
S3150801751032D01F4AD2F8B432D2F8C822224901A879
S315080175200FF016F901AB6A000F211848F9F7A7F809
S315080175300FB0F0BD1D4B0822F8211448F9F79FF842
S31508017540BDE7124F1A4B2A460F213846F9F797F825
S31508017550184B01AC0FCB07C4237001A93846F9F7BC
S31508017560F5F8301A00EBD07001AB3322C0F34F01A6
S315080175703846F9F784F8C5E70F4B2A460F21034821
S31508017580F9F77DF8C5E700BF2C9A020850D3002009
S31508017590D80F002000030308F802030804030308B0
S315080175A0A0A302085008030838030308FC020308CD
S315080175B01803030828030308640803082DE9F04F94
S315080175C02DED028B91B0A54B93F94C33032B40F368
S315080175D05181052B40F3EB81092B00F3D482A04E90
S315080175E0A0493046F9F7C8F83046F9F795F8304614
S315080175F0F9F7A6F896F8295096F82A30ED1AEDB259
S3150801760003213046F9F7D5F9974CD4F82836D4F83A
S315080176101C26964903A80FF09BF803AB00221146D6
S315080176203046F9F72CF88D4F97F94F3304EB83035E
S31508017630D3F82C1603A80FF08BF8ADB203AB2A4684
S3150801764087213046F9F71BF897F9C03204EB830313
S31508017650D3F8781403A80FF07BF803AB6A008721E7
S315080176603046F9F70CF894F9153004EB8303D3F88F
S31508017670801403A80FF06CF803AB05EB45028721CC
S315080176803046F8F7FCFF03213046F9F792F904F280
S31508017690FC542E460627DFF8C891DFF8C0B17CE016
S315080176A0734B2A4685216E48F8F7E9FF0CE16E4BC4
S315080176B0D3F8BC32224600214846F8F7E0FF0437E2
S315080176C0DAF80030224641464846F8F7D8FF01362F
S315080176D02C44A4B2042E00F05682BA4639684846AC
S315080176E0F9F734F8C0F182001FFA80F803214846F9
S315080176F0F9F75FF99BF94C33B342E0D19BF898321D
S31508017700002BD4D000958223224600214846F9F75A
S3150801771046FC00214846F9F74CF9D0E7524A02EBF4
S315080177208303D3F80C1603A80FF012F872E14E4A38
S3150801773002EB8303D3F80C1603A80FF009F87FE1CF
S315080177409BF8983243B9484BD3F8BC3232460021EC
S315080177504846F8F794FF09E200948223324600214D
S315080177604846F9F71CFC00214846F9F722F9FDE1DC
S315080177703D4BD3F8BC32324600214846F8F77FFF25
S315080177800434DAF80030324641464846F8F777FFBE
S3150801779001372E44B6B2092F20D0A24621684846A1
S315080177A0F8F7D4FFC0F182001FFA80F80321484692
S315080177B0F9F7FFF89BF94C33BB42E1D19BF89832B4
S315080177C0002BD5D000958223324600214846F9F789
S315080177D0E6FB00214846F9F7ECF8D1E71F4B93F988
S315080177E04C33092B0DD01E4C03212046F9F7E1F83D
S315080177F01D4BD3F80836AA006E212046F8F73FFF3D
S31508017800C1E1164B93F89832ABB1AE00144C009512
S31508017810FF23324600212046F9F7C1FB0021204605
S31508017820F9F7C7F8104BD3F8083632466E212046C9
S31508017830F8F725FFA7E1AD000B4E094CD6F8BC3287
S315080178402A4600212046F8F71AFFD6F808362A46AE
S315080178506E212046F8F713FF95E100BFD80F0020E7
S3150801786050D30020A0A3020894000020AC08030806
S315080178700C060308C94CCA492046F8F77DFF20467D
S31508017880F8F74AFF2046F8F75BFF94F8295094F871
S315080178902A30ED1AEDB203212046F9F78AF8C14AD2
S315080178A0D2F82036D2F81C26BF4903A80EF050FF9D
S315080178B003AB002211462046F8F7E1FEBB4BD3F88D
S315080178C09C32002B7FF4ECAEB64CB4F9D025B849FE
S315080178D003A80EF03DFFADB26F00B04E03AB3A46BA
S315080178E085213046F8F7CBFEB4F94C33B14981FB13
S315080178F00321DA17C2EBA10202EB8201A3EB4103D2
S315080179001BB212B2AC4903A80EF022FF03AB05EB7A
S31508017910450285213046F8F7B2FE94F9E03504EBC5
S315080179208303D3F8D41503A80EF044FF03ABAA00CA
S3150801793085213046F8F7A3FE01213046F9F739F8D3
S31508017940B4F9D005F0F7CCFD02460B4600209B4959
S31508017950F0F756FFF1F722F900EE100ABDEEC08ADC
S31508017960F8EEC87A30EE670ADFED957A20EE270A37
S315080179700EF090FAFDEEC07A17EE903A18EE102A3C
S31508017980904903A80EF0E4FE844C03AB3A46AA21BB
S315080179902046F8F774FE03212046F9F70AF88A4FBC
S315080179A02C460026DFF8F491DFF800B295E67B4D08
S315080179B07B492846F8F7E0FE2846F8F7ADFE284643
S315080179C0F8F7BEFE95F8294095F82A30E41AE4B28C
S315080179D003212846F8F7EDFF724AD2F82436D2F881
S315080179E01C267A4903A80EF0B3FE03AB0022114602
S315080179F02846F8F744FE6D4B93F94E33002B7FF773
S31508017A008DAE684A02EB8303D3F80C26704903A8A6
S31508017A100EF09EFEA4B203AB224687215F48F8F713
S31508017A202EFE624B93F94D33002B7FF780AE5D4AEC
S31508017A3002EB8303D3F80C26664903A80EF088FEE9
S31508017A406500DFF8588103AB2A4687214046F8F7D7
S31508017A5016FE544F554E96F94D3307EB8303D3F86B
S31508017A600C1603A80EF074FE03AB2A46872140467E
S31508017A70F8F705FEB7F9D025C6F8AC2296F94D33C5
S31508017A806BB996F94E33002B40F08280474B93F938
S31508017A904E337BB90121454BC3F8B0120AE0434B7B
S31508017AA00221C3F8B01293F94E331BB103213F4BA0
S31508017AB0C3F8B0123D4FD7F8B03202FB03F3C7F84B
S31508017AC0B432364E44493046F8F756FE012130465F
S31508017AD0F8F76FFF3046F8F71FFE3046F8F730FE25
S31508017AE0D7F8AC32D7F8B0223C4903A80EF030FEDD
S31508017AF003ABA20037213046F8F7C1FD294DD7F867
S31508017B00B432D5F85424364903A80EF021FE03AB46
S31508017B1004EB84023C213046F8F7B1FD2049304692
S31508017B20F8F72AFE3046F8F7F7FD3046F8F708FE6B
S31508017B3003213046F8F73DFF05F2F455264604279A
S31508017B40DFF85890DFF864B0AA4629684846F8F77E
S31508017B50FDFDC0F182001FFA80F803214846F8F7B7
S31508017B6028FF9BF94C33BB423FF4EAAD0435DAF8FA
S31508017B700030324641464846F8F781FD013726442A
S31508017B80B6B2062FE0D111B0BDEC028BBDE8F08F7D
S31508017B900221064BC3F8B01278E700BF50D3002084
S31508017BA0A0A3020894000020A4080308D80F002007
S31508017BB03407030867666666C803030800807640CB
S31508017BC00000C8428408030878060020B4080308A0
S31508017BD09008030898080308D4F702087C060308E6
S31508017BE090060308334B93F8C4323F2B00D07047F5
S31508017BF0304B93F89832002BF9D12E4B93F86E320D
S31508017C000A3B042BF3D8DFE803F0030B301E4200CE
S31508017C100123284A82F89832274A82F8CE357047D6
S31508017C20244AD2F8C8320133C2F8C832D2F8182326
S31508017C30013A9342C4BF1F4BC3F8C82201221E4B07
S31508017C4083F8CE2570471B4BD3F8C832013B07D4BE
S31508017C50184AC2F8C8320122174B83F8CE25704755
S31508017C600022144BC3F8C822F5E7124BD3F8C832E1
S31508017C70053B07D40F4AC2F8C83201220E4B83F8D6
S31508017C80CE25704700220B4BC3F8C822F5E7094AEF
S31508017C90D2F8C8320533C2F8C832D2F81823013AE5
S31508017CA09342C4BF034BC3F8C8220122024B83F88F
S31508017CB0CE259CE7D80F002094000020334B93F87B
S31508017CC0C4323F2B00D07047304B93F89832002BC3
S31508017CD0F9D12E4B93F86E320A3B042BF3D8DFE821
S31508017CE003F0030B301E42000123284A82F898321A
S31508017CF0274A82F8CE357047244AD2F8C83201336A
S31508017D00C2F8C832D2F81823013A9342C4BF1F4BAE
S31508017D10C3F8C82201221E4B83F8CE2570471B4B98
S31508017D20D3F8C832013B07D4184AC2F8C83201222F
S31508017D30174B83F8CE2570470022144BC3F8C82287
S31508017D40F5E7124BD3F8C832053B07D40F4AC2F8F8
S31508017D50C83201220E4B83F8CE25704700220B4B01
S31508017D60C3F8C822F5E7094AD2F8C8320533C2F87A
S31508017D70C832D2F81823013A9342C4BF034BC3F859
S31508017D80C8220122024B83F8CE259CE7D80F002092
S31508017D90940000202DE9F04F91B0AD4B93F9503383
S31508017DA0032B40F36581072B40F3D8810A2B40F357
S31508017DB055820D2B40F3048111B0BDE8F08FA54B18
S31508017DC0D3F8B034324600214046F8F758FC04355A
S31508017DD0DAF80030324649464046F8F750FC013792
S31508017DE02644B6B2042FE7D0AA4629684046F8F7D2
S31508017DF0ADFCC0F187001FFA80F903214046F8F768
S31508017E00D8FD9BF95033BB42E1D19BF89832002B40
S31508017E10D5D000948723324600214046F9F7BFF8AA
S31508017E2000214046F8F7C5FDD1E78A4BD3F8B034AF
S31508017E302A4600214846F8F722FC0434DAF80030CD
S31508017E402A4641464846F8F71AFC01373544ADB289
S31508017E50082FB1D0A24621684846F8F777FCC0F149
S31508017E603C001FFA80F803214846F8F7A2FD9BF962
S31508017E705033BB42E1D19BF89832002BD5D00096FE
S31508017E803C232A4600214846F9F789F80021484645
S31508017E90F8F78FFDD1E703AC6F4B0FCB84E80F00E2
S31508017EA06E4C03AB72008A212046F8F7E8FB694D50
S31508017EB0674B93F9513305EB8303D3F8341603A8BB
S31508017EC00EF046FC03AB06EB46028A212046F8F77C
S31508017ED0D6FB05F5CB6534460827DFF88091DFF830
S31508017EE070B115E05B4BD3F8B03422460021484601
S31508017EF0F8F7C5FB0435DAF800302246414648460C
S31508017F00F8F7BDFB01373444A4B20B2F3FF454AF45
S31508017F10AA4629684846F8F719FCC0F187001FFAEE
S31508017F2080F803214846F8F744FD9BF95033BB42D4
S31508017F30E0D19BF89832002BD4D0009687232246AD
S31508017F4000214846F9F72BF800214846F8F731FD94
S31508017F50D0E7404BD3F8B034224600214846F8F71B
S31508017F608EFB0435DAF80030224641464846F8F7D2
S31508017F7086FB01363C44A4B20E2E3FF41DAFAA4639
S31508017F8029684846F8F7E2FBC0F187001FFA80F82E
S31508017F9003214846F8F70DFD9BF95033B342E0D16A
S31508017FA09BF89832002BD4D00097872322460021CC
S31508017FB04846F8F7F4FF00214846F8F7FAFCD0E7F7
S31508017FC0264C27492046F8F7D7FB2046F8F7B8FB91
S31508017FD003212046F8F7EDFC224B0522F92120461C
S31508017FE0F8F74DFB20492046F8F7C6FB2046F8F777
S31508017FF093FB2046F8F7A4FB94F8297094F82A30E5
S31508018000FF1AFFB203212046F8F7D3FC114DD5F824
S31508018010B424164903A80EF09BFB03AB00221146B4
S315080180202046F8F72CFBD5F8C81103A80EF0C2FBB9
S31508018030BFB203ABBA0028212046F8F720FB05F2A8
S3150801804064653C460B26DFF81490DFF804B096E722
S31508018050D80F002094000020BC08030850D3002044
S315080180602C9A0208EC090308A0A30208D4080308FD
S31508018070A64EA7493046F8F77FFB3046F8F760FB6E
S3150801808003213046F8F795FCA24B0522F921304623
S31508018090F8F7F5FAA0493046F8F76EFB3046F8F7D7
S315080180A03BFB3046F8F74CFB96F8294096F82A3000
S315080180B0E41AE4B203213046F8F77BFC974DD5F86C
S315080180C0B424974903A80EF043FB03AB00221146DB
S315080180D03046F8F7D4FA934F95F87026394603A82F
S315080180E00EF036FBA4B203AB22468A213046F8F7D6
S315080180F0C6FA95F8B823394603A80EF029FB03AB4F
S3150801810062008A213046F8F7BAFA874F97F952334F
S3150801811005EB8303D3F8741603A80EF019FB03AB1A
S3150801812004EB44028A213046F8F7A9FA97F9CE32C8
S3150801813005EB8303D3F87C1603A80EF009FB03AB02
S31508018140A2008A213046F8F79AFA05F5C765264648
S315080181500027DFF8B881DFF8D0B145E66B4D6C49E9
S315080181602846F8F709FB2846F8F7EAFA03212846CC
S31508018170F8F71FFC6D4B0522F3212846F8F77FFA1D
S31508018180644B0522F9212846F8F779FA6249284607
S31508018190F8F7F2FA2846F8F7BFFA2846F8F7D0FAB8
S315080181A095F8296095F82A30F61AF6B20321284679
S315080181B0F8F7FFFB594CD4F8B4245D4903A80EF02F
S315080181C0C7FA03AB002211462846F8F758FA94F97C
S315080181D0103004EB8303D3F8841603A80EF0B8FA1B
S315080181E0B6B203AB324641212846F8F748FA94F964
S315080181F0113004EB8303D3F8841603A80EF0A8FA0A
S3150801820003AB720041212846F8F739FA94F912307E
S3150801821004EB8303D3F8841603A80EF099FA03AB8B
S3150801822006EB460241212846F8F729FA94F9133054
S3150801823004EB8303D3F8841603A80EF089FA03AB7B
S31508018240B20041212846F8F71AFA04F5C9643546F9
S315080182500427DFF8B890DFF8D0B0FBE52B4C2C49A2
S315080182602046F8F789FA2046F8F76AFA03212046E4
S31508018270F8F79FFB2D4B0522F3212046F8F7FFF966
S31508018280244B0522F9212046F8F7F9F92249204617
S31508018290F8F772FA2046F8F73FFA2046F8F750FA47
S315080182A094F8296094F82A30F61AF6B20321204682
S315080182B0F8F77FFB194DD5F8B4241E4903A80EF02B
S315080182C047FA03AB002211462046F8F7D8F9164FAC
S315080182D097F93C3005EB8305D5F8941603A80EF0FB
S315080182E037FAB6B203AB32468A212046F8F7C7F900
S315080182F097F85323002A3FF4CEAD02EB8202C2EB74
S3150801830002120D4903A80EF023FAC9E550D300203D
S315080183102C9A0208BC060308A0A3020894000020B0
S31508018320D8080308DC080308D80F0020EC0903085D
S31508018330E4080308E8080308CC080308084B93F87F
S31508018340983263B9064B93F86E320A2B07D1072286
S31508018350034B83F86E220122024B83F8CE25704720
S31508018360D80F002094000020084B93F8983263B97F
S31508018370064B93F86E320A2B07D10722034B83F873
S315080183806E220122024B83F8CE257047D80F0020B2
S315080183909400002070B40E4B93F854530D4A0024F0
S315080183A00923012602E012F8033F3BB19842FAD1AC
S315080183B053788B4204BF95783446F4E724B9044BC5
S315080183C093F8540370BC7047014B83F85453F6E78E
S315080183D0D80F0020A8FF02082DE9F04F87B0364BC9
S315080183E093F8544383F8C4420121344A82F8CE15DE
S315080183F0002283F8982293F8556316B12F4B83F818
S31508018400CF152D4B93F856B393F857A393F8589372
S3150801841093F8598393F85AC393F85BE3284800F114
S31508018420EC0300F50770002505950495039502955B
S3150801843001952F46012102E00833834217D01A78A5
S31508018440A242F9D193F801B09E7893F803A093F864
S31508018450049093F8058093F806C093F807E0012580
S31508018460059104910391029101910F46E4E7FFB941
S31508018470019B13B1104B83F85563029B13B10E4B45
S3150801848083F857A3039B13B10B4B83F85893049BAB
S3150801849013B1094B83F85983059B13B1064B83F82E
S315080184A05AC315B1044B83F85BE307B0BDE8F08FF7
S315080184B0014B83F856B3DBE7D80F00209400002060
S315080184C0A8FF020808B5274B93F8823063B94FF421
S315080184D080612548F4F712FF90B100224FF48061BC
S315080184E02148F4F711FF0BE04FF480611E48F4F7B9
S315080184F005FFD0B901224FF480611B48F4F704FF48
S31508018500184B93F88130B3B94FF400711648F4F754
S31508018510F5FE48B100224FF400711348F4F7F4FE52
S315080185200022104B83F85C2308BD0E4B93F882306A
S31508018530002BE5D1CBE74FF400710B48F4F7DEFECB
S3150801854050B901224FF400710748F4F7DDFE012204
S31508018550044B83F85C2308BD024B93F88130002B4A
S31508018560E2D1D1E7D80F0020000C024010B5064C25
S315080185702046F4F70DF90A212046F4F785F9204635
S31508018580F4F7DDF910BD00BF38130020F8B5F4F78C
S3150801859023F8534BC3F83C031C46FF2603F56A75BB
S315080185A0F4F71AF8D4F83C33C01A7C280DD884F8A5
S315080185B06462002384F8653284F86632012384F8FC
S315080185C069322846F3F7CAFEEAE7454C002504F561
S315080185D06A76F4F701F8D4F83C33C01AF9280CD8AE
S315080185E084F8645284F8655284F86652012384F843
S315080185F069323046F3F7B2FEEBE7394CFF2504F54D
S315080186006A76F3F7E9FFD4F83C33C01AB0F5967FDA
S315080186100DD284F8645284F86552002384F86632D0
S31508018620012384F869323046F3F798FEE9E72C4CC2
S31508018630002504F56A77F3F7CFFFD4F83C33C01A5F
S31508018640B0F5FA7F0FD284F8645284F8655284F83B
S315080186506652012684F869623846F3F77FFE30468A
S31508018660F3F7C0FFE7E71E4C40F2252604F56A77C3
S31508018670F3F7B2FFD4F83C33C01AB04211D800233D
S3150801868084F86432FF2284F8652284F8663201256B
S3150801869084F869523846F3F761FE2846F3F7A2FFD4
S315080186A0E6E70F4C40F2ED2604F56A77F3F794FFF7
S315080186B0D4F83C33C01AB04210D8002384F8643287
S315080186C084F8653284F86632012584F86952384699
S315080186D0F3F744FE2846F3F785FFE7E7F8BD00BF41
S315080186E0D80F002008B5424B93F8C432302B18D066
S315080186F03F4B93F84033002B52D13D4BB3F812331D
S315080187005BB13C4AD2F8FC22934206DB384A002187
S3150801871082F84013062182F86E12374AA2F8B63E4D
S3150801872008BD334B93F84033002B39D1304BD3F87E
S315080187303C33002BE1D12E4BB3F81233002BDCD19D
S31508018740F9F796FB2B4B93F9082303EB4203B3F88E
S31508018750003300EE103AB8EE400AF9F7D9F8FFF7F8
S3150801876015FFF3F739FF224BC3F83C03B3F812237D
S3150801877003EB0211D3F88800C1F86404D3F8CC00DE
S31508018780C1F86804D3F81001C1F86C04D3F8540190
S31508018790C1F87004012183F840130A44A3F812238F
S315080187A0154B93F8B43E002BA7D00022124B83F841
S315080187B0B42EF9F75DFB0E4BB3F8122303EB021146
S315080187C0D3F88800C1F86404D3F8CC00C1F868046A
S315080187D0D3F81001C1F86C04D3F85401C1F8700438
S315080187E00132A3F812230122024B83F8CE2584E72E
S315080187F0D80F00209400002088B90020000000004E
S315080188002DE9F04F2DED048B8FB08D4B03F6B86132
S3150801881000220A6003F6BC610A6003F56C610A600E
S3150801882003F6C4631A60874BD3F8F003EFF76AFEC1
S3150801883081A3D3E90023EFF7B9FEF0F7AFF9824B2D
S31508018840D3F81853AA1E40F63E339A4200F2EA803C
S3150801885008EE100A7C4CD4F8B800EFF731FECDE9E2
S315080188600201D4F8FC00EFF72BFECDE90401D4F898
S315080188704001EFF725FECDE90601D4F88401EFF7AB
S315080188801FFECDE9080104F2644405F1805808F198
S31508018890FF3804EB081800230D934FF000090C93D9
S315080188A0CDF804900B93CB460A93CA46012503E0FB
S315080188B01034444500F0A380636962689B1A002B53
S315080188C0B8BF5B4207EE903AF8EEE77AC7EE889AA8
S315080188D0FDEEE99AA369A2689B1A002BB8BF5B4211
S315080188E007EE903AF8EEE77A87EE889ABDEEC99ACE
S315080188F0E369E2689B1A002BB8BF5B4207EE903A20
S31508018900F8EEE77AC7EE888AFDEEE88A23692268D7
S315080189109B1A002BB8BF5B4207EE903AF8EEE77A4E
S3150801892087EE887AFDEEC77A17EE900AEFF7D8FD3B
S31508018930DDE90223EFF764FF06460F465046EFF7D7
S31508018940E1FD02460B4630463946F0F7BFF828B135
S3150801895030463946F0F722F982460A9519EE900A09
S31508018960EFF7BEFDDDE90423EFF74AFF06460F469A
S315080189705846EFF7C7FD02460B4630463946F0F72B
S31508018980A5F828B130463946F0F708F983460B951C
S3150801899019EE100AEFF7A4FDDDE90623EFF730FF1C
S315080189A006460F460198EFF7ADFD02460B463046DF
S315080189B03946F0F78BF828B130463946F0F7EEF824
S315080189C001900C9518EE900AEFF78AFDDDE9082368
S315080189D0EFF716FF06460F464846EFF793FD0246A0
